:020000040002F8
:1070000070560020DD730200E5730200E773020092
:10701000E9730200EB730200ED7302000000000050
:10702000000000000000000000000000EF730200FC
:10703000F173020000000000F3730200F573020018
:1070400039760200F773020029780200F773020014
:10705000F7730200F773020095750200F7730200E0
:10706000F7730200F7730200F7730200F773020070
:10707000F7730200F7730200F7730200F773020060
:10708000F773020089760200F7730200F7730200BB
:10709000F7730200F773020099760200F77302009B
:1070A000F7730200F7730200F7730200F773020030
:1070B000F7730200F77302000000000000000000F8
:1070C000F7730200F7730200F7730200F773020010
:1070D000F7730200F7730200F7730200F773020000
:1070E000F773020000000000000000000000000034
:1070F00000000000F773020000000000F7730200B8
:10710000000000000000000000000000000000007F
:10711000000000000000000000000000000000006F
:10712000000000000000000000000000000000005F
:10713000000000000000000000000000000000004F
:10714000000000000000000000000000000000003F
:10715000000000000000000000000000000000002F
:10716000000000000000000000000000000000001F
:10717000000000000000000000000000000000000F
:1071800000000000000000000000000000000000FF
:1071900000000000000000000000000000000000EF
:1071A00000000000000000000000000000000000DF
:1071B00000000000000000000000000000000000CF
:1071C00000000000000000000000000000000000BF
:1071D00000000000000000000000000000000000AF
:1071E000000000000000000000000000000000009F
:1071F000000000000000000000000000000000008F
:10720000DFF80CD000F088F90048004771BE02009A
:107210007056002000B583B002900091019244F2B4
:10722000010071466A4600F0D7FC03B000BD0000C3
:1072300030B450E8012F93B2C48923448489A34217
:1072400028BF1B1B0489A34202BFBFF32F8F00205E
:1072500007E0C3EA020340E80134002CE9D14FF013
:1072600001000A6030BC704750E8012FC2EA0242B8
:1072700040E801210029F7D1704730B450E8022FCF
:107280001FFAA2F3C488A34202BFBFF32F8F0020CE
:107290000DE0C48923448489A34228BF1B1BC2EA92
:1072A000034340E80234002CE8D14FF001000A60AB
:1072B00030BC704750E8022FC2EA224240E8022167
:1072C0000029F7D17047034653E8022FD988B2EB63
:1072D000324F4FF0000017BF92B241EA014142EA3B
:1072E000014104E05A68B2EB324F08BF012043E885
:1072F0000212002AE8D1704730B4044654E8000F67
:107300000D4644E80053002BF8D1156030BC70479F
:1073100030B4044654E8000F40EA010544E8005345
:10732000002BF7D1156030BC704730B4044654E8E8
:10733000000F00EA010544E80053002BF7D1156067
:1073400030BC704730B4044654E8000F80EA0105B1
:1073500044E80053002BF7D1156030BC704730B4BF
:10736000044654E8000F00EB010544E80053002BED
:10737000F7D1156030BC704730B4044654E8000FB4
:10738000A0EB010544E80053002BF7D1156030BC99
:10739000704770B404464FF0000054E8006F0D6869
:1073A000AE4207BF44E80023012044E800630E60BA
:1073B000002B1CBF0020F0E770BC704730B40446BF
:1073C00054E8000F88422CBF451A054644E8005394
:1073D000002BF5D1156030BC70470000064880478F
:1073E00006480047FEE7FEE7FEE7FEE7FEE7FEE7AA
:1073F000FEE7FEE7FEE7FEE79D760200017202006F
:107400002DE9F05F0546002092469B4688460646D9
:10741000814640241BE0284641464746224600F06C
:107420006BF853465A46C01A914110D3114618467C
:10743000224600F016F82D1A67EB01084F46224647
:107440000120002100F00DF817EB00094E41201E2D
:10745000A4F10104DFDC484631462A464346BDE834
:10746000F09F202A04DB203A00FA02F10020704746
:107470009140C2F1200320FA03F319439040704772
:1074800000487047542D030040EA01039B0703D0D6
:1074900009E008C9121F08C0042AFAD203E011F853
:1074A000013B00F8013B521EF9D27047D2B201E015
:1074B00000F8012B491EFBD270470022F6E710B5F9
:1074C00013460A4604461946FFF7F0FF204610BD52
:1074D000421C10F8011B0029FBD1801A704730B5FF
:1074E00004460020034600E05B1C934203D2E05CAC
:1074F000CD5C401BF8D030BD202A04DB203A21FAB5
:1075000002F00021704721FA02F3D040C2F12002BC
:107510009140084319467047064C074D06E0E06865
:1075200040F0010394E8070098471034AC42F6D3CA
:10753000FFF76AFEA4440300C444030070B58C182E
:1075400010F8015B15F0070301D110F8013B2A1177
:1075500006D110F8012B03E010F8016B01F8016B64
:107560005B1EF9D12B0705D40023521E0DD401F860
:10757000013BFAE710F8013BCB1A921C03E013F829
:10758000015B01F8015B521EF9D5A142D8D300205E
:1075900070BD00002DE9FC410025DFF894800095C6
:1075A0004FF4807601242F460195304605F0AAFE5F
:1075B00038B1D8F80403204203D0304605F098FED5
:1075C0002543361D64007F1CB6B2082FEDD34FF45F
:1075D000BE74204605F096FE48B1204605F088FEB0
:1075E00045F000456A460221002005F0E9FD15F04E
:1075F000FF0F16D0012600242E420ED008EB840186
:10760000D1F81005D1F81015C0F30520094AC1F3CF
:10761000014152F8242002B190477600641C082CE6
:10762000EAD3002D02DA684608F0B6FEBDE8FC8118
:1076300000600040A02D002070B54FF480763046E9
:1076400005F086F80F4DB40540B1304605F087F8D7
:107650000120C4F808032968002088474FF4827687
:10766000304605F075F800280AD0304605F077F866
:107670000220C4F808032968BDE8704001200847CB
:1076800070BD0000D023002002490248091F09688C
:10769000006808474024002006F036BC10B54FF0C3
:1076A00080520023D2E94C100D2906D18C07C4F872
:1076B0000C31C4F81031534C23600D2955D1524B75
:1076C0001B68524C2360504B1B1D1B68241D2360FC
:1076D0004D4B08331B68241D23604B4B0C331B6838
:1076E000241D2360484B10331B68241D2360464B28
:1076F00014331B68241D2360434B18331B68434C11
:1077000020342360404B1C331B68241D23603E4BF8
:1077100020331B68241D23603B4B24331B68241D2E
:107720002360394B28331B68241D2360364B2C33D0
:107730001B68241D2360344B30331B68334C4034AA
:107740002360314B34331B68241D23602E4B3833A8
:107750001B68241D23602C4B3C331B68241D2360B5
:10776000294B40331B68241D23600D2906D128486E
:107770000168C90702D06FF0010101602548016866
:1077800041F470010160BFF34F8FBFF36F8FD2E9F7
:107790004C104FF010220D2907D130B1012804D030
:1077A000D2F80802174920310860D2F800020028F8
:1077B00003DBD2F8040200281FDA012007F074F876
:1077C0001221C2F8001214480368002BFCD0C2F842
:1077D000041201680029FCD0002007F065F8BFF30F
:1077E0004F8F0C487C3801680C4A01F4E06111436A
:1077F0000160BFF34F8F00BFFDE70A4908480860EA
:1078000010BD0000380500400404001020C50040F1
:107810000004004088ED00E000E401400400FA05A7
:107820000090D00320250020014800680047000098
:10783000D823002002E008C8121F08C1002AFAD18C
:1078400070477047002001E001C1121F002AFBD1E0
:10785000704700000121202803DA814005480140DB
:1078600003E0402802DA2038814009B10120704746
:1078700000207047FC06FFBD2DE9F843804643F227
:10788000020669B9694607F041FFB04204D018B159
:10789000284AB221FFF7BEFC9DF80000800746D4BD
:1078A0000021404607F03CFF050040D0112D3ED09E
:1078B00021482249401AC708022000EB07440D2D39
:1078C0000AD00B2D1DD0B5421FD11D49204642467E
:1078D000BDE8F84305F01CBF20464246194905F0B3
:1078E00017FF1321404676DF002820D006F0E0FB8A
:1078F000024601B020464346BDE8F04312A105F020
:107900000EBF204642461E49E2E7284606F0D0FB5D
:107910000246012000EB074043461AA105F0FFFE96
:107920002846BDE8F843034AE121FFF773BCBDE8F0
:10793000F8830000EC3503000C450300D444030039
:107940001C350300A834030073645F626C655F67D5
:1079500061705F646973636F6E6E6563742829205C
:1079600072657475726E6564202573206F6E206376
:107970006F6E6E5F68616E646C652025642E00001A
:1079800068350300417373657274696E672E2070E9
:107990006D5F636F6E6E5F73656375726528292016
:1079A00072657475726E6564202573206F6E206336
:1079B0006F6E6E5F68616E646C652025642E0000DA
:1079C00010B560B159B102780B785208B2EB530F81
:1079D00005D10622401C491CFFF781FD08B100209B
:1079E00010BD012010BD800701D00020704701208C
:1079F0007047C3688B4206D811440069491E814212
:107A000001D8012070470020704790F82400012819
:107A100001D01F207047EE20704710B501220221CF
:107A2000002001F0E7FD08B1072810D1072202214C
:107A3000012001F0DFFD08B1072808D100210A224A
:107A4000084601F0D7FD08B1072800D1002010BD7D
:107A500010B504462C21FFF730FD012020714FF4B2
:107A60009670206144F25060606110BD10B588B11D
:107A70000F481049401AC008032101EB00400EA135
:107A800005F042FE08F018FC002810D00E4A4FF412
:107A90002E7108E003210D4800F091FD002806D06A
:107AA000094A40F23231BDE81040FFF7B3BB10BDC8
:107AB0007C450300D4440300457261736520626F06
:107AC0006E6473210000000000C0020058250020F1
:107AD00070B58CB015460E4600236C46C3F10F01FD
:107AE000415CE1545B1C102BF8D30D2104F1100014
:107AF000FFF7E3FC0020C0F10F02315C2244401C80
:107B000011740328F7D3684646DF0020C0F10F0147
:107B1000214491F820102954401C0328F6D30CB0BE
:107B200070BD022001F056BC0149C97800F014BFB5
:107B30009823002070B50024064D06E068680121F6
:107B400010F8340006F026FB641C28788442F5D334
:107B5000002070BDE0230020F8B516460C4605460F
:107B60000A2A01D20720F8BD06F00AFC18B906F06F
:107B7000CDFB0028F7D1134F202113487D603C70C6
:107B8000BE60FFF79AFC0020C7E904000F4E0DE02D
:107B900005EBC4003168009181788DF80110007800
:107BA0000B4A694606F042FB0028DCD1641EE4B2B1
:107BB000EED2BDE8F84005480021064A001D00F05D
:107BC0003DB90000E0230020582E0020AC2903001E
:107BD0004DB10200D19F0200FEB515460E46074684
:107BE00072B605F049FE00BF05F072FC0028FBD11B
:107BF0002249234A0120891AC90800EB0144012FB8
:107C000022D06FF48050381821D0B0F5405F23D0D7
:107C10006FF44051C842204605D1D5E9003219A180
:107C200005F07DFD03E032461DA105F071FD2248FF
:107C30000068C00700D000BE2A4603B0314638466F
:107C4000BDE8F04000F07AB820461CA101E02046D3
:107C500022A105F059FDEAE7A86806F029FA0346D3
:107C6000D5E90001CDE900100296204624A1AA68BA
:107C700005F070FD20462CA1EBE700007C450300D9
:107C8000D4440300415353455254494F4E2046417A
:107C9000494C45442061742025733A257500000045
:107CA000554E4B4E4F574E204641554C5420617413
:107CB0002030782530385800F0ED00E0534F46541E
:107CC0004445564943453A20415353455254494F40
:107CD0004E204641494C454400000000534F465455
:107CE0004445564943453A20494E56414C49442063
:107CF0004D454D4F525920414343455353000000D9
:107D00004552524F52202575205B25735D206174CA
:107D10002025733A25750D0A50432061743A2030AE
:107D20007825303878000000456E64206F66206545
:107D300072726F72207265706F72740008B50123E1
:107D40008DF800309DF80030144B186059609A602F
:107D50006FF48041401807D001280FD1DA60D8684D
:107D600000689861D86807E01A61186980685861EE
:107D700018690068986118694068D861186858687F
:107D80009868D868186958699869D86972B600BF48
:107D90009DF800000028FBD162B608BD782E0020B7
:107DA00010B502280ED108480849401AC10803201E
:107DB00000EB0140044606A105F0A6FC204610A1F8
:107DC00005F0A2FC012010BD7C450300D444030053
:107DD000506F776572206D616E6167656D656E7459
:107DE0002077616E747320746F20726573657420E0
:107DF000746F20444655206D6F64652E00000000AE
:107E0000506F776572206D616E6167656D656E7428
:107E100020616C6C6F77656420746F207265736588
:107E20007420746F20444655206D6F64652E0000E9
:107E3000014802F04EB900002024002010B55AB1CC
:107E400000684FF0FF3401294261C0E9024400D0CC
:107E500000210161002010BD072010BD38B5114878
:107E600008235822416800910F49006804F01BFA6A
:107E7000002815D10D4A69460D4802F02FF904007B
:107E80000ED101210A4802F0A4F90123094A19463A
:107E9000074802F0F6F80649012008390870204624
:107EA00038BD0000B4290300A82E0020910A030069
:107EB00020240020FFFF7F00F8B504460026174667
:107EC0000D468DF80060684600F042F8D4E90201E2
:107ED000C04370EA010005D09DF8000000F05CF896
:107EE0000020F8BD03F018F940197141C4E90201FE
:107EF0009DF8000000F050F8A761206900B12561ED
:107F00002146BDE8F840002009F0B4BE38B504466B
:107F100000208DF80000684600F01AF8D4E902014C
:107F2000C04370EA01000DD04FF0FF30C4E90200F9
:107F30009DF8000000F030F82146BDE838400120EF
:107F400009F098BE9DF8000000F026F8002038BD2A
:107F500030B5EFF3108172B60D4A9468012324B155
:107F60000370002900D162B630BD93604FF0E0236A
:107F7000D3F88051074C25401560C3F88041D3F8F1
:107F8000844154605A17C3F8842100220270E8E744
:107F9000002F0020FC06FFBD0B498A68002A11D083
:107FA00000280FD1EFF3108072B60B684FF0E0227B
:107FB000C2F800314B68C2F8043100228A60002800
:107FC00000D162B670470000002F002070B5054652
:107FD00008680C46411C04D005F063F9206805F0E0
:107FE000C3F86068411C02D0002105F0ABF8296895
:107FF000A069C1F82405607D227D29681043C1F87D
:108000006C05D4E900122868C0F81425C0F80C15D6
:10801000207D012814D1A068411C02D0002105F068
:1080200091F8E068411C04D005F03BF9E06805F0E8
:108030009BF8D4E902122868C0F80825C0F810158A
:1080400070BD70B5054608680C46411C04D005F0AB
:1080500032F9206805F092F86068411C02D00021D6
:1080600005F079F82968A069C1F82405607D217DB3
:108070002A680843C2F86C05D4E900122868C0F8E1
:108080000C15C0F81425207D012814D1A068411CCE
:1080900002D0002105F05FF8E068411C04D005F033
:1080A0000AF9E06805F06AF8D4E902122868C0F815
:1080B0000825C0F8101570BD03F0A0BD2DE9F047EC
:1080C000814605884A484FF000088AB00178424648
:1080D000284600F059FC99F80500400701D400211A
:1080E00076E005F58077B8B205AB0122072106F0EE
:1080F00055FF04003F48404A4FF00101A0EB020049
:108100004FEAD00001EB00460AD0204605F0D0FF30
:10811000024630462B46394905F001FB214629E04D
:10812000284603F001FB4FF6FF71044688422BD12D
:108130008A46069803F062FA0446504510D001467C
:10814000284603F0D1FA2846FFF7EEFCE0B92846AE
:1081500008F064FF2846FFF7E7FC0028BFD013E0D3
:1081600007F0F2F80446504508D1304624A105F046
:10817000CBFA0421284608F07FFFB0E701462846E5
:1081800003F0B2FA4FF00108B8B22246072106F018
:108190007DFF07001BD0862F1ED005F089FF024609
:1081A00030462B462349009405F0C1FA394628464B
:1081B00008F062FF0021484606F0E8FDB8F1000F24
:1081C00002D0204603F09AFA0AB0BDE8F0870121F8
:1081D000484606F0DBFDF7E7142217496846FFF72B
:1081E00053F9ADF80250684602F014FAEFE70000C8
:1081F0009823002014450300D4440300AC38030046
:10820000436F756C64206E6F7420616C6C6F63617A
:108210007465206E657720706565725F696420669D
:108220006F7220696E636F6D696E6720626F6E6436
:108230002E000000C8390300302903002DE9FC4757
:10824000002517880646158090F82D0014468946AB
:1082500030B13A462146484600F0BCFB051E09D124
:10826000B0784FF00C0A18B32088C846001DB842F9
:1082700002D95046BDE8FC87684679DF0028F9D16D
:108280002088032108F8001020881921401C80B2A2
:10829000208008F800102088401C80B2208000EB6D
:1082A0000801BDF8000009F0B8FE218808442080CC
:1082B000F0780222C8B1218896F9033001F1030C4D
:1082C0004846BC45D5D8425421884FF0010C491C82
:1082D00089B2218000F801C02188491C89B221801F
:1082E00009F801302088401C20807068B8B12188CE
:1082F00090F9003001F1030C4846BC45B9D842540E
:1083000021880A22491C89B2218042542188491CB3
:1083100089B2218009F801302088401C20803089F2
:1083200050B1CDE900474B460622022106F1080074
:1083300009F062FF051E9DD1308A50B1CDE900479A
:108340004B460722032106F1100009F055FF051ED8
:1083500090D1308B50B1CDE900474B461522142106
:1083600006F1180009F048FF051E83D1306A30B1CC
:108370003B462246494601F0D2FC051EDBD1706A1D
:1083800030B13B462246494603F068FE051ED2D175
:1083900096F82C0038B13B4622464946304608F054
:1083A000ABFF051EC7D1307838B13B46224649465F
:1083B000304603F0E1FE051EBDD128465AE718B548
:1083C00004460020ADF8000013466A46204600F03F
:1083D00006F8002802D0BDF80000204418BD70B592
:1083E000E0B1DAB1002402E0045D2C44A4B2651CC3
:1083F0008D4206D21688A642F6D8061976789E4295
:10840000F2D18C420AD2A31C005D9BB200B1401E87
:108410000004000C02D01C188C4201D9002070BD51
:10842000138070BD80F8301070472DE9F0410D00C9
:10843000044606D02CB195F87A000026012803D016
:1084400006E00E20BDE8F08195F89800012821D0C3
:108450004FF00108A6702C2205F17801201DFFF7CE
:1084600013F884F83060D5F8A4006063D5F8A8004C
:10847000A0634FF6FF70A4F8240404F58260C4F8EA
:108480002004C4F82664A4F82A6484F82C642078B4
:1084900010B104E00720D5E7FF2084F8540004F170
:1084A00055072046C4F81074FFF7AFFAA4F8140477
:1084B00004F2144239462846FFF7C0FE0028C1D115
:1084C00004F23120C4F818042046FFF79EFAA4F8FD
:1084D0001C0404F21C4205F13C00D4F81814FFF708
:1084E000ADFE0028AED184F85180208BA4F848005E
:1084F00084F83C80266484F85060606900216064E0
:10850000454604F13C02781E72DF00289AD125709E
:1085100098E72C22001DFEF7B7BF10B50288102A7D
:108520001BD0112A20D0262A1DD1007A0C46012802
:1085300001D0022817D1A0780521401CB0FBF1F230
:1085400001FB1201204600F03AF800280BD0A16B85
:10855000002908D0BDE810400847C27B012A02D19B
:108560008088A1F8240410BD0C46002184F82E1444
:108570008088B4F824148842F5D120790028F2D1FB
:108580000121DFE710B5044690F8540074DF0120A4
:1085900084F82E04002084F8300484F8500006216A
:1085A000204602F072FA002808D1A178204600F097
:1085B00006F810B1A16B01B18847002010BD2DE96C
:1085C000F05F044600780F4698B1A7700025C4F804
:1085D0002654A4F82A5484F82C54A079012608B112
:1085E000012F09D0E07980B1012F05D0022F03D0EF
:1085F0000BE00820BDE8F09F616B21B184F82D6489
:108600000820884701E084F82D5404F22741002017
:108610000A5C0AB1304603E0401C0628F8D300206B
:108620004FF002084FF0030B012F06D0022F0CD0A1
:10863000032F0FD0042F15D110E0A17929B194F8A0
:10864000241011B908B130460DE0E17911B108B13B
:10865000404608E0207A08B1584604E0607A08B144
:10866000042000E02846A070616B41B1032801D0CE
:10867000042804D1607910B194F82E0498B184F8DC
:108680002F5404F13C0018210746FEF716FF84F82A
:108690003C6004F12C0006F095FF58B194F82C00D2
:1086A00084F8510008E084F8305484F82F640720DF
:1086B0008847E6E784F8516094F8240058B104F143
:1086C000280006F07FFF20B194F8280084F85200BB
:1086D00001E084F8526084F85050A27804F22641F8
:1086E00004F582694FF0060A052A64D2DFE802F039
:1086F0007C030F22420084F83160C4F82054C4E99E
:10870000101584F83C808020A4F8480055E084F8D7
:10871000318094F82420384612B10722027001E01B
:1087200080F800B0228A8281C4F820544160E16858
:10873000B96042E06069B860208BB88194F8240089
:108740003D460028204602D084F83CA001E084F891
:108750003C6009F01DFD50B185F8148004212046CD
:1087600002F093F938BB052184F8311021E084F838
:1087700031B01EE0E069B860208CB88194F8240024
:108780003D460028204602D084F83CA001E084F851
:108790003C6009F0FDFC48B185F8148004212046B6
:1087A00002F073F938B984F831A002E0042084F8AB
:1087B0003100C4F82094A07878B13A4604F154000E
:1087C000D4F8201472DF00287FF414AF94F830102E
:1087D00094F8540073DF0028F6D1616B11B194F85E
:1087E00031008847002005E784F83150F5E70000A4
:1087F00070B5040012D001461C221448FEF744FE56
:108800001248134D0560206850B17ADF002806D168
:108810002068016829604068686005E00E2070BD2E
:108820000B487BDF0028FAD108484FF6FF71143857
:10883000084A20F8041B0549343901600021FFF77C
:10884000FDFA0028EBD0032070BD0000CC290020E9
:10885000F02200202921030010B5044600F0B0F8F2
:10886000002805D02146BDE81040024803F09ABD1B
:1088700010BD0000F82900200346034880680A461E
:10888000194602F02FB90000E829002070B51546FE
:108890000E46044609F088FC002809D0054800EB84
:1088A0008400C0692A463146BDE8704002F01AB91A
:1088B00070BD0000E829002010B5044600F080F8E3
:1088C000002805D02146BDE81040024803F06ABDEB
:1088D00010BD0000002A002010B5044600F070F81A
:1088E000002805D02146BDE81040024803F05ABDDB
:1088F00010BD0000FC29002070B50546002400F0E2
:108900005FF838B12946044803F04CFD08B1022451
:1089100000E00124204670BDF429002070B5054612
:10892000002400F04DF838B12946044803F03AFD20
:1089300008B1022400E00124204670BDF029002087
:1089400010B51821034803F008FD182800D0C0B264
:1089500010BD0000E829002070B505460C46084609
:1089600009F022FC60B1284600F02AF840B1054821
:10897000294600EB8400BDE870401C3003F012BDB6
:10898000002070BDE829002070B5054616460C464B
:10899000084609F009FC00280ED0284600F010F81F
:1089A000002809D00548324600EB84002946BDE87E
:1089B00070401C3002F064B870BD0000E82900204F
:1089C000142801D3002070470146014803F0EABC97
:1089D000EC2900207CB5054608880C4609309042F9
:1089E00001D90C207CBD68466DDF0028FAD12188B2
:1089F0000820685420881B21401C80B22080295404
:108A00002088401C80B220802844DDF801100160DD
:108A1000BDF8051081802088801D80B220809DF8DF
:108A20000010490800D0012129542088401C2080D2
:108A300000207CBD10B503F09BFE002809D105483D
:108A40004FF0030C00DF002803D1BDE8104003F015
:108A5000FDBE10BD642D002018B103490860002040
:108A600070470E2070470000B823002010B54FF06B
:108A7000FF3100203DDF00280BD1B1213CDF002871
:108A800007D10448416901208847022005F01CF8FD
:108A9000002010BD482D0020044810B50068416931
:108AA00000208847BDE81040FFF7E0BFB823002052
:108AB00010B588B0044620216846FEF7FEFC03206E
:108AC000ADF8000020788DF802009DF80D00172108
:108AD00040F028008DF80D0001208DF810008DF871
:108AE0001300ADF804108DF812008DF80C008DF80D
:108AF00011006088A21D694600F0DCFF08B010BDBF
:108B000010B5184C86B01ECC8DE81E0048B1164C2E
:108B10004FF6FF71A180006800216061217618B1D5
:108B200004E00E2006B010BD104860610E48FFF74B
:108B300093FF0028F6D101208DF812004FF65960FE
:108B4000ADF81000A21C04A90120A8DF0028E9D17B
:108B50000549684662DF0028E4D10348FFF7A8FF13
:108B6000E0E700008C290300482D0020D1A202007C
:108B700010B5002823D003881C4C102B17D0214699
:108B8000112B8A8815D0C988512B19D0532B16D197
:108B9000C088884213D1207E002810D0FFF77CFFC8
:108BA00000280CD06169BDE8104002200847808889
:108BB00004E08088824202D14FF6FF70A08010BD91
:108BC00083889342FBD110F8062F022AF7D14288FE
:108BD0008A42F4D1017A0429F1D00629EFD005297F
:108BE000EDD0BDE81040801C05F0F6BE482D0020F9
:108BF0002DE9F0410546007B042601272E4C012873
:108C000011D002282CD00226287B314600F08EF8A5
:108C100018B1206841690320884720684169022013
:108C2000BDE8F041084720684FF00008417E49B197
:108C30000621012000F07AF800283BD02068416925
:108C40000320EDE707760121084600F06FF80028C1
:108C500030D02268112882F81880D5D10626D3E7B3
:108C60006A7B142A22D80AB3DFF8508005F10E017E
:108C700008F10400FEF708FC697BC8F818102168A9
:108C80004046497E0029BFD1A0F10C010A68011FAE
:108C9000904768B10F28B7D109480A49401AC0085F
:108CA00007EB0040084904F02FFDADE70526ABE7D0
:108CB00020684776BDE8F081B8230020702D0020A1
:108CC0007C450300D4440300003C030070B5154903
:108CD00000250A68002A24D04A68002A21D00831D9
:108CE000904708281DD0104C0028206845760ED0EB
:108CF0000621022000F01AF818B12068416903200B
:108D00008847206841690220BDE87040084701217A
:108D1000022000F00BF8002803D0206841690320EE
:108D2000F2E770BD642D0020B823002086B0032335
:108D3000ADF8003020238DF814308DF81500002296
:108D40000E48019202928DF81610C188ADF80410F9
:108D500002218DF8061005A90491ADF80820CDF880
:108D60000CD0808801A9AEDF002804D1BDF8001026
:108D7000032900D00C2006B070470000482D0020C9
:108D800030B51F491F4B01250322C91AC9088BB0F2
:108D900002EB014478B1012825D0194A1946511A2D
:108DA000C908012202EB014202281FD00328104605
:108DB0001FD015A11EE020461DA104F0A5FC6846A9
:108DC000FEF746FE8DF8005069462548FFF7A1FBE7
:108DD00000212448FFF750FD0246204622A104F05E
:108DE00097FC0BB030BD204625A103E010462DA115
:108DF00000E03BA10BB0BDE8304004F085BC0000B2
:108E00007C450300D4440300556E6B6E6F776E2073
:108E10006576656E742066726F6D20626C655F6446
:108E200066755F627574746F6E6C6573732E000087
:108E3000446576696365206973207072657061723C
:108E4000696E6720746F20656E74657220626F6F43
:108E5000746C6F61646572206D6F64652E00000034
:108E60005825002019A00200446973636F6E6E6577
:108E700063746564202564206C696E6B732E00003A
:108E80004465766963652077696C6C20656E7465EE
:108E90007220626F6F746C6F61646572206D6F64B5
:108EA000652E00005265717565737420746F2065BE
:108EB0006E74657220626F6F746C6F61646572208E
:108EC0006D6F6465206661696C6564206173796E9D
:108ED0006368726F6E656F75736C792E00000000A9
:108EE0005265717565737420746F2073656E6420AC
:108EF0006120726573706F6E736520746F20636C90
:108F000069656E74206661696C65642E00000000FE
:108F100038B504460088212827D016DC102830D127
:108F2000072000F089FB20B11BA240F24A21FEF786
:108F300071F91D48A18801801C4803F091FB0028AD
:108F40001FD015A240F24D210BE03B281AD0562825
:108F500017D1A088132176DF002812D00EA240F28C
:108F60006A21BDE83840FEF755B900200090A0887E
:108F700069468FDF002804D007A240F25921FEF78E
:108F800049F938BDA088132176DF0028F9D002A264
:108F900040F26221E5E700002E2E5C2E2E5C2E2E84
:108FA0005C6D61696E2E6300702200204C250020EC
:108FB00010B51A4C0188606810290ED011292BD1E8
:108FC000401E606028D1FEF728FD002824D02168CB
:108FD000002921D0BDE810400847D0B90021012266
:108FE000084600F007FB08B107280FD1072202212D
:108FF000012000F0FFFA08B1072807D1042202215E
:10900000002000F0F7FA20B1072802D0216801B152
:1090100088476068401C606010BD0000E8220020A6
:109020002DE9F04701883B4E40F2F3194FF6FF75EA
:1090300010291BD011293ED0122954D0502946D1D5
:10904000C188F289841D914241D1618902293ED1B2
:109050008688304602F014FC050038D004F10C007C
:1090600000F04EF9A8B3294630464EE0C17B878810
:10907000044601292BD1A846284602F001FC050030
:1090800017D02F8000202872234843464A460168A3
:10909000C5F80A104068C5F80E0004F1100105F18A
:1090A0000A0002F0B1FC6872F08900280FD129464D
:1090B0002AE0042013E0808802F0E2FB040006D0DE
:1090C0006068FEF723FF08B107F0BAFF2580BDE80E
:1090D000F087FFE76868FEF719FF0028F7D0BDE8C2
:1090E000F04707F0ADBF87880646384602F0C8FB58
:1090F0000400ECD02B464A4606F1080104F10A00B0
:1091000002F082FC607221463846BDE8F04700F06C
:1091100059BE0000CC290020F02200202DE9F04F9C
:10912000044686880188434897B0834610290CD0AE
:10913000112952D0103019296CD01A2976D1217AF0
:109140000C09042C4FD301224EE03A4D083DA8688B
:10915000C0430B9069680BA803F048F90B990CA861
:1091600000F0BEFD2C220CA96846FEF78DF9002701
:10917000E946A84610E000BF09EB47005FF0000594
:10918000B0F804A008EB85005146001D03F0CAF8B2
:109190006D1C1E2DF6D37F1C0098B842ECD8142EFF
:1091A00007D317B0F021BDE8F04F23A20420FEF74B
:1091B00031B83146584603F000F9314608F1040051
:1091C00003F0FBF8E07B022830D117B03146BDE850
:1091D000F04F1848001D03F0F0B817B03146BDE855
:1091E000F04F03F09FB80022314601F049FC032CF8
:1091F00001D3012200E000220E4831460C3001F07C
:109200003FFC022C01D3012200E000220948314634
:10921000083006E0217A002908D1617AC1F3C00242
:10922000314617B0BDE8F04F01F02ABC17B0BDE8D9
:10923000F08F0000F02900202E2E5C2E2E5C2E2EAA
:109240005C2E2E5C2E2E5C2E2E5C636F6D706F6E0E
:10925000656E74735C626C655C636F6D6D6F6E5C84
:10926000626C655F636F6E6E5F73746174652E63AD
:109270000000000070B51F4E044686B070780028CC
:1092800036D02088A588102811D031782846FFF7DD
:1092900063FB00282CD1204602F022F9204608F07A
:1092A000EDF806B02046BDE8704001F071BD002029
:1092B0008DF80000142101A8FEF7FFF801208DF8B9
:1092C00004004FF6FF70ADF8080004F108000390A9
:1092D000ADF80650CDF810D001A801F085F99DF841
:1092E000002031782846FFF74FFB9DF80000D0E7BB
:1092F00006B070BD282300200078C0F340007047FE
:10930000007800F00100704708B504F0C3FD20B1FB
:109310000D4A40F27D21FDF77DFF00200090694657
:10932000012004F025FC20B1074A40F28321FDF71B
:1093300071FF684604F09CFC002804D0024A40F209
:109340008721FDF767FF08BD00C002000149085CE6
:1093500070470000C8270300084908B5085C009062
:10936000684603F045FFD0F810050099C84010F09A
:10937000010000D0012080F0010008BDC8270300D3
:109380002DE9FC410646C0074FF000050ED0104FF6
:1093900000240122385D009500231146019503F059
:1093A0005BFE641C042CF4D300F04EF8B0070DD51E
:1093B000074E0024361D0022305D03230095114620
:1093C000019503F049FE641C042CF4D3BDE8FC8134
:1093D000C4270300094908B5085C0090684603F0FB
:1093E00007FFD0F80425009B0121994021EA0203E0
:1093F000C0F808351140C0F80C1508BDC42703009B
:109400000249085C012103F060BF0000C42703008B
:109410000249085C002103F058BF0000C427030084
:10942000084908B5085C0090684603F0E1FED0F8F2
:1094300004050099C84010F0010000D0012080F020
:10944000010008BDC427030010B500242046FFF723
:10945000D7FF641C042CF9D310BD10B5002420469E
:10946000FFF7D6FF641C042CF9D310BD10B50246DB
:10947000064B4FF0FF3000215C5C944201D108465E
:1094800010BD491C0429F7D310BD0000C8270300F4
:1094900070B50C4E0C004FF0000530600BD0012071
:1094A00000F06AF808B1022004E0002000F064F83F
:1094B00000B10B202070706810B9FEF7AEFA0546B7
:1094C000284670BDE822002010B5002000F0EEF91B
:1094D00008B1062806D1012000F0E8F908B10628F5
:1094E00000D1002010BD00002DE9F0470D46814657
:1094F000FFF7BCFF0446042836D2DFF874801B480F
:109500001C4EA8F10C0725B3012D0ED0022D2BD136
:1095100004EB440030444578002D25D0B96800297B
:1095200022D02846BDE8F047084704EB4401755CAB
:109530000E44717849B10E4A4FF48041093A80686F
:10954000FEF7BAFC08B987F80390B17808F8041060
:10955000E2E78068FEF7DAFC04EB4401314418F8D6
:1095600004008D78A842D7D0BDE8F087CC2703004F
:10957000842200208C290020042801D2FFF7ECBEB1
:10958000002070470146154810B50088042907D00F
:1095900007290FD00A291FD1BDE8104007F048BFA6
:1095A000132176DF082817D0002815D00CA240F22E
:1095B000CF210DE0A0F57F41FF390DD10C48FEF71A
:1095C000E1FF082808D0002806D005A240F2D921E2
:1095D000BDE81040FDF71EBE10BD00007022002047
:1095E0002E2E5C2E2E5C2E2E5C6D61696E2E63001D
:1095F0005825002070B50023042810D20D4D00EB33
:109600004004012A02D101290CD00022094E00EBAE
:109610004000304461B1012906D0022906D0072359
:10962000184670BD0E30C2B22A55F9E74270F7E70E
:109630008270F5E78C290020044A01460020127947
:10964000D20702D0084600F04DB8704778220020BB
:1096500070B506461E480024C0E90161B00720D558
:109660000025012211462846FFF7C4FF6D1C044661
:10967000042D02D2002CF4D013E094B940F233321E
:1096800004211448FEF768FA04000AD1FEF752FAE2
:10969000040006D10F48104A0021001FFEF7CEFB40
:1096A0000446F00712D00120FFF76AFE74B909489A
:1096B0000A4A00210C38FEF7C1FB040006D1054818
:1096C000074A01210838FEF7B9FB0446204670BD61
:1096D00078220020D8270300B99902009DBA020021
:1096E000237B02002DE9F05F6E4C05460026607872
:1096F000B34618B184F801B002F0B8F96A4F4FF4DC
:109700007A694FF4C87A4FF00108182D69D2DFE862
:1097100005F00C1313384754696E727B727BC58455
:1097200084848484B3B6B9BCC5C502F09FF9386897
:10973000FEF7ECFB06465CE00020FFF771FE002818
:109740004FF0000008D0FFF75BFE022D02D14FF46E
:10975000E16008E0484606E0FFF75AFE022D01D11D
:10976000C82000E05046410CC0034FF47A728018C4
:1097700041F10001257052000023FDF741FE014632
:109780002AE00020FFF74CFE00284FF0000004D034
:10979000FFF736FE4FF44870E5E7FFF739FEDFE7E5
:1097A0000020FFF73DFE00284FF0000002D0FFF739
:1097B00027FECFE7FFF72CFED4E70020FFF730FEAF
:1097C00000284FF0000002D0FFF71AFE01E0FFF77B
:1097D0001FFE257040F6CD4100223868FEF76CFB75
:1097E000064646E00020FFF7F5FD257008E0002062
:1097F00051E025703DE084F801800120FFF7EAFD8B
:10980000002240F26661E8E784F801800120FFF75A
:10981000E1FD00224FF40051DFE77868FEF776FBA8
:109820000646D5F1110000D02EB10220FFF7E8FD69
:1098300084F802B01DE0012816D980B2C82148433F
:10984000C117C90341EA5041C0034FF47A7280182E
:1098500041F1000152000023FDF7D2FD0146002234
:109860007868FEF729FB06460220FFF7D1FD84F851
:1098700002803046BDE8F09F02F0F8F8B9E702F048
:10988000F5F8B4E702F0F2F804E002F0EFF8002097
:10989000FFF7BEFD0120FFF7BBFDAAE7FFF7DDFDE7
:1098A000A7E7000078220020CC270300012108F060
:1098B0000BBD00002DE9F84F0546861C00208DF8F1
:1098C000000091460F464FF0010A6846FEF740FB44
:1098D0001B4C04F21C4860683860D4E90101194F40
:1098E000401A3968081A0EE00121404602F078FD5E
:1098F00002F06CFA0146404602F072FDD4E9010123
:10990000401A3968081A401C8642EDD8B9F1000F98
:1099100003D0052065F3891002E0062065F39F500F
:1099200061683A68114004EB8101C86060683044A6
:1099300060609DF80000FEF72FFB5046BDE8F88FF1
:1099400050320020C824002070B50D4604460A2974
:1099500002D10D21FFF7F8FFA0682268411CA16029
:109960001554D4E90101814204D32046BDE870407A
:1099700003F037B870BD0000044881684068814238
:1099800001D10120704700207047000050320020B4
:10999000034630B5074800210478426806E000BF5E
:1099A00002EBC10005789D4203D0491CA142F7DBC0
:1099B000002030BDE023002000780221FFF794BD95
:1099C000032805D10349A9200860002004F07CB8D1
:1099D00070470000200500401CB5044601F0A4FEBD
:1099E00000236A46092105F01BFC052805D1034820
:1099F000012241792046FEF7C7FF1CBDF822002056
:109A00001CB504460020009042F6A620ADF80000E8
:109A100001208DF80200084801AA694600680190FB
:109A20002046A0DF002805D1044801228179204684
:109A3000FEF7AAFF1CBD0000F8270300F822002053
:109A400005494FF0FF32082841F8202002D308448E
:109A500080F8522070470000A02D0020F0B54FF094
:109A6000FF3512B10023082601E008230C260C4C18
:109A700005E000BF54F823707F1C04D05B1CB34288
:109A8000F8D32846F0BD26185DB286F8305044F869
:109A90002310002AF5D1E11881F85200F1E7000007
:109AA000A02D00200249084490F9300070470000C2
:109AB000A02D00202DE9F0438146887891B0904692
:109AC0000C4600B901208DF83E002088ADF83C001E
:109AD00000250095607C694607F052FC6E46A07C2C
:109AE000711C07F04DFCE07B00289DF8020002D0BD
:109AF00040F0080001E020F008008DF80200217C11
:109B000011B140F0100001E020F010008DF80200CB
:109B1000217B11B140F0010001E020F001008DF83F
:109B20000200217D09B1022100E0012161F3420020
:109B30008DF802001C2102A8FDF7BFFC607BC10666
:109B400001D4800617D50E950EAFE07C791C07F086
:109B500017FC9DF83800079720F00F00401C20F0FC
:109B6000F00010308DF838009DF83A0020F0060023
:109B7000801C8DF83A00607B8DF80800A07B8DF882
:109B80000900142109A8FDF798FC0FA8CDE90906E2
:109B9000A088ADF83000A06820B1E088ADF82C00B6
:109BA000A0680D90A06998B301950088ADF81000E9
:109BB000A06901AD01A94088ADF81200A069406814
:109BC00006950390A069007B07F0DAFBA069691C89
:109BD000407B07F0D5FBA069807A00289DF806003D
:109BE00002D040F0080001E020F008008DF80600E7
:109BF000A169C97A11B140F0100001E020F0100015
:109C00008DF80600A169097A19B140F0010002E05F
:109C10000DE020F001008DF80600A169897B09B1F3
:109C2000022100E0012161F342008DF80600E069A5
:109C300000B10590434609AA02A94846AADF11B01F
:109C4000BDE8F08370B504464FF6FF750A46284616
:109C5000AC4209D14FF480742146104602F07DFBDE
:109C600080B2A0420BD070BDFF2CFCD8214610461C
:109C700002F063FB90F0010F01D0204670BD284632
:109C800070BD000070B5084C050009D01034216883
:109C9000002907D008682060496828468847F6E709
:109CA0000834F4E770BD00008C2D0020054A012126
:109CB00020B1012805D19170FFF7E4BF5170002059
:109CC000FAE770478C2D002010B5D0E90234D1E9B5
:109CD0000220D11AA04101D3012010BD002010BDE7
:109CE00073B58CB00646002000900D9880B100241A
:109CF0006D4621460DA802F055FB30B1009805EBEA
:109D0000400084800098401C0090641C142CF0D308
:109D10002C2269463046FDF7B7FB0EB070BD2DE929
:109D2000F04117880646B81D14460D46984202D9E0
:109D30000C20BDE8F0813188072206290AD34FF4B0
:109D4000486C4FF6FF73614501D9994202D1708882
:109D5000062801D21046ECE7604501D99842F9D1B6
:109D6000994203D0984201D08142F3D80520E855AA
:109D700020881221401C80B2208029542088401C59
:109D800080B220804119308808F047F921880844C2
:109D900080B220804119708808F03FF9218808447A
:109DA00020800020C5E7000002A240F2E311FDF789
:109DB00031BA00002E2E5C2E2E5C2E2E5C6D616959
:109DC0006E2E630038B54A7A0F4B62B100220A72D8
:109DD0005969002906D001228DF80020ADF8020053
:109DE0006846884738BD0A7A62B19B684C6802466B
:109DF00019462046FEF760F80028F3D0BDE8384049
:109E000007F01EB95B68F1E7CC290020F0B585B0FA
:109E100016460F4604461D4614220B496846FDF7B8
:109E200033FB0A488DF80870ADF80240ADF80A60BF
:109E30008DF80C50017800222046FEF7A5FD6846FB
:109E400000F0E8FB05B0F0BD442903009823002092
:109E5000FDF712BD70B588B006460020059006904B
:109E6000ADF81410ADF816100190029001AA05A9E2
:109E7000304690DF050021D004F01AF9034611485E
:109E800011493246401AC108012000EB0140044646
:109E90000E4903F044FCBDF8042012B9BDF80600D9
:109EA00028B1BDF80630204609A103F038FCBDF802
:109EB00008201AB12046164903F02AFC08B02846AB
:109EC00070BD0000EC440300D4440300DC30030008
:109ED00054686520726571756573746564205458A3
:109EE0002F5258207061636B6574206C656E6774C7
:109EF0006820697320746F6F206C6F6E67206279C1
:109F00002025752F2575206F63746574732E0000EE
:109F10002831030070B504460948012102F07BFA9C
:109F2000BFF35F8F0025002808D1204601F0C2FE54
:109F3000002803D1BFF35F8F0148056070BD0000AA
:109F4000042300202DE9FF410C4620B14FF40640C8
:109F500004B0BDE8F0812079002748F2096538B1E6
:109F600041F61D5601281BD0022826D0681DEFE7B8
:109F70000220207102970397E0680190694601A8CA
:109F800006F09CFC50B102988188E1800088208115
:109F9000BDF80010029806F00FFDD9E72846D7E774
:109FA0000A4B6A460021A01D06F040FC38B1074963
:109FB00018398F61CF61A842CAD13046C8E703483B
:109FC0008188019806F0F8FCF5E700006024002085
:109FD00070B500240F4D10E0686800EBC4063078BF
:109FE00004F08CF97178012901D0012100E00021F1
:109FF0004140307800F062FA641C28788442EBDB40
:10A00000D5E90401084303D0BDE8704007F04EBE17
:10A0100070BD0000E023002030B40446132176DF39
:10A0200003000BD0064807492246401AC008022107
:10A0300001EB004030BC044903F071BB30BC7047F9
:10A040007C450300D4440300582D030010B50021C3
:10A05000024802F0E0F980F3100010BD6C360020D9
:10A060004FF480328A400168C1F848230068C0F884
:10A07000082370474FF4A07202EB810189B200F00F
:10A080008DBA2DE9F04105460E464FF4A07000EB65
:10A09000860081B228684FF48034B440984622F09C
:10A0A0007F47C0F808432868C0F84843286803F091
:10A0B0004FFD286800EB8600C0F840752868C0F89E
:10A0C0004443B8F1000F02D02868C0F80443BDE84B
:10A0D000F0810068D0F804057047000070B543793E
:10A0E000234C44F823204279231D03EBC202224C67
:10A0F0001579204A121BD4082DB10825022000EB47
:10A1000004401EA130E005680A88C5F8082590F9CA
:10A1100004208978002A4FEA411104DB02F1E02291
:10A1200082F8001405E002F00F0202F1E02282F84A
:10A13000141D90F904100122002909DB01F01F050C
:10A1400002FA05F54909890001F1E021C1F8005141
:10A150004179002503EBC1010A71417943F83100CF
:10A16000032000EB04400EA103F0CEFA284670BD98
:10A170003C2400205C450300D44403005254432097
:10A18000696E7374616E636520616C726561647978
:10A1900020696E697469616C697A65642E000000DB
:10A1A0005254433A20696E697469616C697A6564D6
:10A1B0002E00000090F90400002809DB00F01F02C7
:10A1C000012191404009800000F1E020C0F8001218
:10A1D00070470A46022100F067B94FF4827100F01F
:10A1E000DDB900680121016070470068012141600C
:10A1F00070472DE9F05F07460C464FF4A07000EB66
:10A2000084001FFA80FA38684FF48036A6409B46D7
:10A2100022F07F45C0F848633868C0F808633868A2
:10A22000D0F8048500EB8402D2F84095C2F840854E
:10A230005146386803F08CFCA9EB080020F07F4001
:10A24000012806D1102003F09DFF5146386803F025
:10A250007FFC3868D0F80485C0F84463A5EB08019A
:10A2600021F07F413868012900EB840010D0C0F84C
:10A2700040553868D0F804156FF07F4C6A1A521EAA
:10A2800022F07F42ACEB0B03934217D362B118E08C
:10A290006D1CC0F84055102003F074FF3868D0F8EA
:10A2A000040540450AD10CE000EB84006D1CC0F8A9
:10A2B00040553868D0F80405884202D00D20BDE82A
:10A2C000F09F01223146384600F0EEF80020F6E714
:10A2D000704713460A460021FFF798BD2DE9F84361
:10A2E000104D0F4680461E4691466946286801F08B
:10A2F000EDFF040014D01C21FDF7DFF801202071D0
:10A30000C4F81490380BC4F80080C4E902606946B0
:10A31000286801F0FCFF06F0F5F90020BDE8F8839D
:10A320000420FBE7602A030010B503780022072B06
:10A3300006D2DFE803F005040610202930000A7079
:10A3400010BD01230B7003898B818388CB81C0688A
:10A3500088600A7410BD02220A7002898A8182888C
:10A36000CA81C2688A60807D062802D000200874F5
:10A3700010BD0120FBE703220A70C2888A8102898E
:10A38000CA81C068886010BD04230B70C0888881B2
:10A39000CA818A6010BD0520087010BD70B5064DD9
:10A3A0000646002455F8241009B130468847641C3D
:10A3B000042CF7D370BD0000282F002030B50446D0
:10A3C000006887B00D46806800281FD018216846B5
:10A3D000FDF773F80195A0680590207910B1012868
:10A3E00010D107E001208DF8000020690290E0689C
:10A3F000039005E002208DF80000E0680003029061
:10A4000060690490206881686846884707B030BD5D
:10A41000F0B585B017460C0005463AD0112C38D05F
:10A42000082C36D01C481D49401AC6080D2C11D0E6
:10A43000204603F03DFE0246012000EB06402B467D
:10A44000174903F06CF92A460821684601F0F2FE2C
:10A4500002941BE0022000EB06402A46114903F05B
:10A4600057F92A460421684601F0E4FE27B13878FE
:10A47000C00701D0012000E002208DF80800002074
:10A480008DF80C0041F20110ADF80A00684600F0AA
:10A49000CFF805B0F0BD00001C450300D444030014
:10A4A000943B0300843A03000368C3F84413002A72
:10A4B00002D00068C0F80413704700002DE9F84F7F
:10A4C0000E463449804601EB5001C007097801D09F
:10A4D0000F0901E001F00F074FF00009424601208B
:10A4E0004946FCF7BEFFDFF8B0A004460D46052F35
:10A4F0004ED2DFE807F003161B282C00002E47D0B1
:10A500000121404607F090FA8DF800906846FDF76B
:10A510001FFD5046D0E904120C431543CAE9044517
:10A5200032E00EB1022114E0002112E04EB103210D
:10A53000404607F079FA4046BDE8F84F012107F0A0
:10A540004BBE012105E0002E22D1042101E02EB1F5
:10A5500003214046BDE8F84F07F066BA00214046A7
:10A5600007F062FA0021404607F036FE8DF80090B1
:10A570006846FDF7EDFC5046E243D0E904341A404A
:10A5800024EA0501CAE904219DF80000FDF704FD55
:10A59000BDE8F88F582E0020E023002010B5006899
:10A5A00042581AB103F0D4FA012010BD002010BDAA
:10A5B00010B50446408801F0B7F8A0800248016851
:10A5C0002046BDE8104008470023002010B504468F
:10A5D000808800F0F3FF6080024801682046BDE8F3
:10A5E00010400847102300202DE9F04107460024C1
:10A5F000064E074D05E000BF56F824103846884740
:10A60000641C28798442F7DBBDE8F081FC2C002033
:10A610002823002010B50446408801F085F8A0806A
:10A62000024801682046BDE810400847042903009D
:10A6300001490968084700008029030070B586B009
:10A64000044614216846FCF738FFA0890125A0F5CF
:10A650004040ADF8040020782F4E062833D2DFE8C2
:10A6600000F0320303032C4AA08900F0EDF930B961
:10A67000E08943F6FE71A0F54040884223D8A07BD4
:10A680008DF80800207803280FD000208DF80900ED
:10A69000A0680390606850B10A208DF800006068DF
:10A6A0000490684604F00EFD0DE00120EEE709205D
:10A6B0008DF800008DF81050F3E7A08900F0C4F980
:10A6C00008B1E08930B17078002801D004F04EFE66
:10A6D00006B070BD606830B10C208DF80000606875
:10A6E00002907570DDE70B208DF80000BDF80400C6
:10A6F00004F0E0FEF5E7606848B115208DF8000031
:10A70000606802904FF6FF70ADF80400C9E71420AE
:10A710008DF80000F6E700001423002038B5044649
:10A720000F480078B0B1A4F57F40FF380FD06846DD
:10A7300005F018FF88B10521017001210171C48065
:10A74000684605F01DFF05F0CFFF002038BD48F238
:10A75000036038BD48F2016038BD48F2076038BD7B
:10A76000682400200D4808B5007888B1684605F0D7
:10A77000F9FE80B106210170684605F001FF084826
:10A78000017809B10121017305F0AEFF002008BD79
:10A7900048F2016008BD48F2076008BD6824002047
:10A7A000EC2F0020F0B587B014216846FCF785FE39
:10A7B000314C207818B16846FFF7F0FD5AE0201DB3
:10A7C00001F00BFEA0BB40F6F8700168481C02D1F6
:10A7D0004FF0102041694FF08050026940694B1CD6
:10A7E00001D100FB02F1254800220161A1F5405191
:10A7F000C160234902F08AFA002826D122481C238E
:10A800008C222049006801F04EFD04F0E7F90500B4
:10A810004FF0000615D0022D13D00127062D16D0BB
:10A8200005A805F09FFEA8B107700C2D1DD200E011
:10A8300020E0DFE805F01A121A121A191A191A1470
:10A8400016142670666048F20A6007B0F0BD2770E3
:10A850006660B0E748F20760F7E7067105E003219C
:10A8600000E00221017100E0077105A805F088FEF3
:10A8700005F03AFF0020E8E76824002024250020A6
:10A88000702A0300382F0020D829030038B50400AF
:10A8900014D0694606F012F8B0B1BDF8000000EB24
:10A8A00080010B4800EB8100C16851B1A17A41B130
:10A8B000C168491EC1600020A07238BD48F2046022
:10A8C00038BD48F2056038BD48F2096038BD000067
:10A8D000C42F00201FB501A9684605F0A7FF04B0EA
:10A8E00010BD07B513460A466946002005F09EFFD5
:10A8F0000EBD07B513460A460021684605F096FFCF
:10A900000EBD20B119B1006808600020704748F200
:10A9100004607047F8B50D46040018D0BDB1694613
:10A9200005F0CCFFB0B1BDF800000C4900EB800091
:10A9300001EB800001210C30666801F051FD2E60B2
:10A9400060680C3068600120A0720020F8BD48F2F9
:10A950000460F8BD48F20960F8BD0000C42F002073
:10A9600018B10323002207F0FBBD48F204607047D2
:10A970000223002207F0F4BD094910B50A69042A30
:10A980000AD0084A096942F821000548012110301F
:10A9900001F026FD002010BD48F20B6010BD000044
:10A9A00048240020282F00202DE9F84F0446244891
:10A9B0000078D8B1F4B112212046FCF77EFD0320C7
:10A9C000DFF880902080002504F1100804F10E0AC1
:10A9D00005EB850109EB810630897189084487B24E
:10A9E000706804F085F8032807D009E048F2016098
:10A9F000BDE8F88F48F20460FAE72088401E208006
:10AA00006088F16808446080208971890844208149
:10AA1000608938446081C7F58060A18980B2814235
:10AA200000D2A0815346A21D211D2846CDF80080EA
:10AA300005F0E0FF6D1CADB2022DC9D30020D7E7B1
:10AA400068240020C42F002043F6FE71A0F540408A
:10AA5000884201D8012070470020704710B5044695
:10AA60000078182802D1FDF76BFF207010BD10B5DB
:10AA700004460078182802D1FDF762FF207010BD4F
:10AA80000AB101F09ABC01F04DBC70B50D46044608
:10AA9000B0F81414D0F810040122FDF790FC00B1B6
:10AAA000057004F13C0204F5826104F1540072DF88
:10AAB00070BD000070B5134600220546112900D173
:10AAC0000122074C33B12179FDF75EFF0022617846
:10AAD000284600E06178BDE87040FDF755BF0000F2
:10AAE000A0230020F7B517460E0011D000980025CE
:10AAF00060B100242146684601F054FC18B1A0B2B0
:10AB00003946B0476D1C641C142CF3D32846FEBD97
:10AB10000020FEBD406805F045BD00000EB516A141
:10AB20009DF8080020F00F00401C20F0F0001030CD
:10AB30008DF808000D2202A87CDF20B1124A40F2F5
:10AB40006111FCF767FB0020009001905021ADF8E7
:10AB50000400ADF800104FF4C870A021ADF8060055
:10AB6000ADF8021068467ADF002804D0064A40F2A9
:10AB70006F11FCF74FFB0EBD4E6F726469635F642B
:10AB800066755F4F4B00000000C0020070B510B149
:10AB90004FF4064070BD1C4C0025207B08B1257386
:10ABA00001E000F0A5F8207808282AD2DFE800F0BC
:10ABB0002904080C10291422BDE8704000F026B8C2
:10ABC000BDE8704000F082B8BDE8704000F064B8A5
:10ABD000BDE8704000F040B80620207060880A4947
:10ABE00000EB8000283901EB80004068BDE8704030
:10ABF00003F0D4BF072020706560BDE8704003F00B
:10AC0000DBBF48F20E6070BDEC2F00201149F0B49C
:10AC10008A1C00200346A1F128050C18A67A4EB123
:10AC2000A37200EB800405EB8404E66816B9247C6B
:10AC3000012C0AD0401C80B20228EED30B704B804E
:10AC40004B60F0BC41F61D5070471080F0BC00F026
:10AC50003DB80000EC2F00200C48418801EB810238
:10AC6000A0F1280101EB8201CA6852B105210170EF
:10AC7000074802218180016800230122054801F074
:10AC8000A9BF042202704968F6E70000EC2F0020FB
:10AC9000702400202425002038B50A4908480324E0
:10ACA0000B684268898803EB810153880470DB1CC0
:10ACB00000201B0400909B0B034802F0DFF838BD16
:10ACC000EC2F00207024002024250020074910B517
:10ACD0004888091D05F042FE18B1BDE81040FFF795
:10ACE000DBBFBDE81040FFF7B7BF0000EC2F00202E
:10ACF00070B5194C0121207808281AD2DFE800F03D
:10AD00000419191C252929182089134A401C20815F
:10AD1000002060802073283A00EB800312F8233073
:10AD200043B100232518401C80B2AB720228F3D334
:10AD3000217070BD0123F5E76068084940888A8862
:10AD4000C01C10448880022004E000F009F80620AE
:10AD500000E00720207070BDEC2F00207024002040
:10AD60000A4909484988026801EB810307492839E3
:10AD700001EB83014B6803604A6082880A810222EA
:10AD8000828000200874704770240020EC2F00207F
:10AD90002DE9F043064680883288DFF85C8185B073
:10ADA0000746502A37D010DC5449554B06F10A05A6
:10ADB000A1EB03014FEAD1014FF0020303EB014481
:10ADC000352A3AD0362A07D168E0522A02D0542ACE
:10ADD000F9D102E000F012FF82E0142249496846EE
:10ADE000FCF752FBADF80270384600F09DFCADF860
:10ADF000040000F0C9F90022444698F804103846CF
:10AE0000FDF7C2FD0022E1783846FDF7BDFD68463A
:10AE1000FFF7CEFB64E0307B012861D1B07A0128D6
:10AE20005ED13089A0F52451023959D1012138462B
:10AE300000F038FF07F060F952E098F80610FDF7CF
:10AE40008BFD00284CD0002298F806103846FDF7FC
:10AE50009BFDF288B2F5857F17D012B120462AA15A
:10AE60000BE02A88012A03D0204636A102F050FCCC
:10AE70006A88012A04D0204641A102F049FC04E07E
:10AE8000A98800223846A1DF08B1002125E001226F
:10AE900098F807103846FDF777FD21E04FF00009DC
:10AEA00098F80710FDF758FDD0B1002298F8071068
:10AEB0003846FDF769FDF28812B1204612A104E080
:10AEC000AA88012A04D020462DA102F021FC03E02B
:10AED000A87900B1012081464946384606F008FEAF
:10AEE0000022364998F80200FDF7D0FC05B0BDE815
:10AEF000F04306F0F9B80000F8220020D444030023
:10AF0000D444030050280300556E6578706563745F
:10AF100065642047415454207374617475732077BD
:10AF200068696C652067657474696E672043415277
:10AF300020636861722076616C75653A20307825EF
:10AF4000780000004D756C7469706C65202825646C
:10AF5000292043415220636861726163746572699C
:10AF6000737469637320666F756E642C20757369E2
:10AF70006E67207468652066697273742E00000025
:10AF8000556E657870656374656420434152206333
:10AF90006861726163746572697374696320766154
:10AFA0006C7565206C656E67746820282564292C93
:10AFB0002073746F726520302E000000B98002008B
:10AFC00070B504460078002814D1608800F016FEA1
:10AFD0006588284600F0E8F928B107480122C178C1
:10AFE0002846FDF7D1FC6088FEF7F6FCBDE870400E
:10AFF00007F082B870BD0000F822002070B5204C28
:10B0000000252570FDF79CFC6070FDF799FCA07091
:10B01000FDF796FCE070FDF793FC2071FDF790FCC6
:10B020006071FDF78DFCA071FDF78AFCE07162781C
:10B030000121182A18D0A278182A15D0E278182AE7
:10B0400012D02279182A0FD06279182A0CD0A2794E
:10B05000182A09D0182807D004F10C000560BFF3A6
:10B060005F8F2170002070BD0648074A801AC00813
:10B0700001EB0040054902F047FB032070BD0000D2
:10B08000F8220020D4440300D44403009C2D030084
:10B090007CB504460078092837D1607A58BB207AFD
:10B0A0001C4E4FF6FF75012811D0072802D0082842
:10B0B0002BD121E0A08800F081FA0446A84224D0D8
:10B0C000012100F0EFFD2046FEF786FC1DE0A08880
:10B0D0006A46012103F018FF68B90198007850B161
:10B0E000A08800F06BFAA8420FD00122F178FDF79A
:10B0F0004BFC05F0F9FF08E0F068012805D1BFF32B
:10B100005F8F044900200C310860BDE87C4006F0E8
:10B11000F3BF0000F822002010B50B48FEF7D9FF5E
:10B12000094A083AD2E90434C018D2E9063244F197
:10B130000001C31A71EB020204D24FF08072801832
:10B1400041F1000110BD00002024002010B5C0B264
:10B15000FEF71EFC0446007803F0D0F80146607844
:10B16000012801D0012000E0002090EA010F08D062
:10B170000449D1E90401084303D1BDE8104006F0B9
:10B1800095BD10BDE02300201CB5054AD2E902128E
:10B19000CDE900120022694604F07CF81CBD0000D5
:10B1A0006828030003484FF6FF7181800121017078
:10B1B00000207047082300202DE9FC41804600F064
:10B1C000B3FA002403250127A0F57F412646FF3965
:10B1D00008D06A46082103F097FE18B90198841D2B
:10B1E0008688056832462B4621464046B1DF042852
:10B1F00004D0082804D00B2808D002E0112000E079
:10B200000020002F00D10B20BDE8FC810027A807FB
:10B2100001D50125E6E7344303D000242646032563
:10B22000E0E7064806494246401AC008012101EB02
:10B230000040044902F06CFAE5E70000DC4403003A
:10B24000D4440300643003002DE9FF47824600F038
:10B250006BFAA0F57F418146FF3916D03B493C4A45
:10B260000127891AC90807EB014600BF3A467F1C2F
:10B270004FF00008BFB202AB0821484603F08EFE33
:10B28000040007D0072C5ED05EE043F2020004B059
:10B29000BDE8F087039D03232A1DA91D50462B609E
:10B2A000B2DF040004D00C2C37D0052C38D038E0A5
:10B2B0006A460821484603F027FE58B1052814D0F5
:10B2C00002F0F6FE02463046534622A102F027FA6B
:10B2D0000320DCE70198AA888088824205D1019981
:10B2E000A81D891DFCF7FBF830B14A46082110461D
:10B2F00003F0CCFE044627E00821484603F0BCFEDC
:10B3000048B102F0D5FE034630464A461F4902F0D6
:10B3100006FA032418E00B2416E04FF0010800E0C1
:10B3200000240821484603F0A7FE40B102F0C0FE09
:10B33000034630464A46154902F0F1F90324B8F1B4
:10B34000000F93D100E00C242046A0E7DC4403006A
:10B35000D44403007064625F706565725F646174F9
:10B36000615F7074725F67657428292072657475F7
:10B37000726E656420257320666F7220636F6E6E37
:10B380005F68616E646C653A20256400E42F0300F9
:10B3900004488088A0F57F41FF3901D005F0AEBE9A
:10B3A00070470000082300200EB502A9019100F0AB
:10B3B000BBF96A46012103F0A7FD08B100200EBDCC
:10B3C000019800780EBD00002DE9F04107464FF6C8
:10B3D000FF761048B3DF78B102F06AFE02460E48ED
:10B3E0000E49401AC008012101EB00400C4902F04F
:10B3F0008FF90320BDE8F081064C43F20305A41E3B
:10B40000324661883846AFDFA842F3D16088401CDD
:10B410006080F5E70A230020DC440300D4440300E5
:10B42000982F0300428800EB82020C328A4201D935
:10B43000022070478188A1F57F42FF3A06D001883B
:10B4400021B18068401C01D0002070470120704766
:10B45000884204D20068401C01D0012070470020BF
:10B4600070473EB5027802230C46B3EB520F17D15A
:10B47000B0F80110ADF80010C1788DF80210818885
:10B48000ADF8041080798DF8060002AA01A92046C3
:10B49000FCF71EFB032202A96846FCF720F808B15E
:10B4A00000203EBD01203EBD70B50D460446142867
:10B4B00010D2FDF785FA68B1084904EB840001EB6E
:10B4C0004000D0F802102960C188A980007AA871D4
:10B4D000002070BD43F2020070BD0000642A00200D
:10B4E00070B5018890B0102961D1011D2C226846E9
:10B4F000FBF7CAFF9DF804004FF6FF7603213446A0
:10B50000B1EB500F2BD003F083FE9DF804006D4685
:10B5100040080ED001280CD0022820D118E00D9947
:10B52000281D1131FCF74CFA18B100BFBDF82C40B2
:10B5300015E00CAA0BA9072003F03EFE0028EED16F
:10B540000DE00D99281D491CFFF78BFF0028EDD158
:10B550000CAA0BA9072003F02FFE0028F1D1BDF89B
:10B560000000B44200EB8001124820F8114000EBCB
:10B5700041000199C0F80210BDF80810C1809DF883
:10B580000A10017213D0BDF80000ADF82E000020A3
:10B59000ADF83040084E8DF82C000BAD044600BFCE
:10B5A00056F8241028468847641C022CF8D310B0A3
:10B5B00070BD0000642A00207C2803002DE9F041C2
:10B5C0004FF6FF760546B04213D00B4F002400BF64
:10B5D00004EB840037F81000A84206D12046FDF79E
:10B5E000EFF910B12046BDE8F081641CA4B2142C20
:10B5F000EED33046F7E70000642A00203EB50C4643
:10B60000054603F005FE0BE0BDF80000A04207D0A0
:10B610002846029900F00EF810B1BDF800003EBDBA
:10B6200001AA6946072003F0C7FD0028ECD14FF6B8
:10B63000FF703EBD2DE9F0410C46054600F11107B3
:10B6400001F111061022491C401CFBF748FF48B9C4
:10B65000681C00F0FBF928B1601C00F0F7F908B194
:10B66000012400E0002431463846FCF7A9F93B7874
:10B670000222B2EB530F0CD00321B1EB530F08D0D1
:10B680003378B2EB530F04D0B1EB530F01D001214B
:10B6900000E00021084201D18C4302D00120BDE826
:10B6A000F0810020FBE7018811B9421892780AB1B5
:10B6B00001207047491C0829F7D30020704710B5B6
:10B6C0000C460346FFF7EFFF00280AD018882188B0
:10B6D000884205D10822A11C981CFBF700FF08B185
:10B6E000002010BD012010BD142804D2024A00EB36
:10B6F000800022F810107047642A002070B50546BB
:10B70000FFF75CFF0446284603F002FC002808D13E
:10B71000142C06D2034B04EB84024FF6FF7123F87E
:10B72000121070BD642A002010B50446142808D2F7
:10B73000FDF746F928B1044904EB840031F8100004
:10B7400010BD4FF6FF7010BD642A00203EB50446C0
:10B7500003F05EFD0EE0019920464631FFF7AFFF92
:10B7600028B9019920462A31FFF7A9FF10B1BDF889
:10B7700008003EBD6A4602A9072003F01DFD00280F
:10B78000E9D14FF6FF703EBD10B50A4941600A4845
:10B7900000F023FE58B902F0C9FB07491C238C2294
:10B7A000087404488C39001F006800F07CFD0020FC
:10B7B00010BD0000642A0300983000202DE9F041FC
:10B7C0002C4D002420B16C604FF40640BDE8F081A0
:10B7D0000879012250B1284B01280BD0254A0226B6
:10B7E0000832022821D0032829D12CE00A7103F065
:10B7F000E3F922E05FF0000000EB800113F8211074
:10B80000022908D0401C80B20228F5D32A706C604F
:10B8100041F61D50DAE700EB800003F8204003EB0F
:10B820008000406803F0BAF907E00C719680116857
:10B8300000230122114801F0CDF90028C6D06C6028
:10B8400048F20D60C2E70C480C712830418810683E
:10B8500001EB810703EB8701D1F804C0C2F800C0F7
:10B860004860B2F804C0A1F808C0968003F82740E9
:10B87000D8E7000068240020C42F002024250020E1
:10B880000146034802888A4200D000207047000029
:10B89000B82900202DE9FC5F0E008346DDE90C4746
:10B8A000C6F1000098469246814600D4084601251C
:10B8B00003E000BF90FBFAF06D1C5045FADAA84592
:10B8C00000D9454624B1002E01DB780700D5641E5F
:10B8D000B80702D5B8F1000F0AD0F80708D13CB17B
:10B8E000A54205D220215846641EFEF72DF8F6E742
:10B8F000002E02DA4E462D2102E0780703D52B21D7
:10B900005846FEF721F807F0030002280BD1B8F1E2
:10B91000000F08D13CB1A54205D230215846641E23
:10B92000FEF712F8F6E7CDE90047434652463146A6
:10B93000584606F087FBBDE8FC9F000070B50D4639
:10B94000044600684FF4887102F0D2FB4FF4907106
:10B95000206802F0CDFB4FF49271206802F0C8FB22
:10B960004FF4A271206802F0C3FB4FF4AC71206861
:10B9700002F0BEFB20681249C0F804132068690772
:10B9800040F30730090E002804DB00F1E02080F8C6
:10B99000001405E000F00F0000F1E02080F8141D15
:10B9A000206840F30730002809DB00F01F02012166
:10B9B00091404009800000F1E020C0F8001170BD06
:10B9C00010034200024600201268530713D502F00C
:10B9D0000300012802D002280CD105E0C2F3831035
:10B9E0000B68801C184404E00223086803EB9252A1
:10B9F00010440860012070470248007A002800D0F7
:10BA00000120704798300020F0B58488A518944232
:10BA100000D82246A41AC288D6189A4200D81346E3
:10BA2000D21A4B880788BB420CD34088834209D87E
:10BA30008888A04206D3A84204D8C888904201D37F
:10BA4000B04201D90020F0BD0120F0BD0021425CD0
:10BA50000AB101207047491C1029F8D30020704713
:10BA6000800701D000207047012070470A4810B5B8
:10BA7000807860B1002401E0022C06D02046FDF75A
:10BA8000BFFC641C042CF7D310BD0324F6E7BDE80B
:10BA90001040FDF7D9BC000078220020034801794E
:10BAA000C90702D00078FDF71DBE7047782200203C
:10BAB0001721018041800021017141711B21817199
:10BAC000C17170472DE9FE4F2E4F984692460D00EA
:10BAD000814601D000260DE0684600F0A1FB6A46D1
:10BAE0000021484603F06CF93878009E10B99DF8A3
:10BAF000090098B152463146484605F06DFE0446AD
:10BB0000014600224846FEF7D5FF0D2C37D008DC51
:10BB1000A4B3082C33D00B2C09D130E00520BDE8AC
:10BB2000FE8F112C1ED0A4F54050023827D020469D
:10BB300002F0BEFA0246144814494B46401AC008A7
:10BB4000012101EB0040124901F0E9FD5FF003051E
:10BB5000B8F1000F04D0324621464846FEF758FCA3
:10BB60002846DCE72A46F9784846FCF70DFF52469E
:10BB7000B9784846FCF708FF0025E9E7FFE72546C6
:10BB8000E6E70000A02300201C450300D444030086
:10BB90003C3B030070B50E460C4915460446097837
:10BBA000FCF7DAFE00280FD0204603F0AFF800289B
:10BBB0002A463146204603D0BDE8704003F0ACB8B9
:10BBC000BDE87040FEF785BB70BD000098230020E3
:10BBD00070B5094D0646A978FCF7BEFE0446E97823
:10BBE0003046FCF7B9FE014622463046BDE87040BB
:10BBF0000123FFF767BF0000A0230020F0B585B048
:10BC00000546002714216846FBF757FCA5F57F4041
:10BC1000ADF80250FF3825D02846FFF7CDFA0400D2
:10BC200022D01B481B49401AC6080B2C22D0112CCD
:10BC30001ED0A4F5405002380ED0204602F038FA4B
:10BC40000246012000EB06402B46134901F067FD38
:10BC50002146284605F0FCF910483A4681782846E6
:10BC6000FCF792FE05B0F0BD0F208DF800000BE050
:10BC70000127F1E710208DF80000022000EB0640BC
:10BC80002A46074901F044FD6846FEF791FCE3E7C8
:10BC9000D4440300D44403006C2E0300F822002097
:10BCA000C02E03000A4602494978FCF76DBE000029
:10BCB000F82200202DE9F041002786B080463E465C
:10BCC000FFF7C2FA04461F481F49401AC508112C45
:10BCD00023D003DCFCB10B2C06D114E0862C1ED043
:10BCE000A4F5405002380ED0204602F0E1F9024699
:10BCF000012000EB0540434614A101F010FD214650
:10BD0000404605F0A5F939464046FFF7CBFF06B09F
:10BD10003046BDE8F0810126F5E70127F3E714225C
:10BD20001A496846FBF7B0FB0220ADF8028000EB31
:10BD30000540424616A101F0EBFC6846FEF738FCD0
:10BD4000E1E70000D4440300D44403006773636D4B
:10BD50005F6C6F63616C5F64625F63616368655FA2
:10BD600075706461746528292072657475726E65DA
:10BD70006420257320666F7220636F6E6E5F68614A
:10BD80006E646C653A2025640000000028280300DA
:10BD9000466C6173682066756C6C2E20436F756C01
:10BDA00064206E6F742073746F72652064617461B7
:10BDB00020666F7220636F6E6E5F68616E646C6583
:10BDC0003A20256400000000704700002DE9FF4183
:10BDD0000026244800F0FEFA2248001F074600F023
:10BDE000F9FA214C2149A06800900D6800E0009804
:10BDF0006946284004EB80000C30FFF7E3FD002883
:10BE0000F5D101AA009901EA050304EB8303491C5B
:10BE1000DB6842F82030401C00910228F2D30198E0
:10BE200000F0030001280BD0022810D10198032153
:10BE300001EB90500099BDF80A6001EB900005E01D
:10BE40000198BDF80A60C0F383100844009038469A
:10BE500000F0BDFA08B10098A06004B03046BDE81B
:10BE6000F08100006836002050320020C8240020F5
:10BE7000ACB04FF48041002001F0D2FC20B160A2B0
:10BE800040F21631FBF7C6F901F014FBFCF7D2FDC6
:10BE900020B15BA240F25731FBF7BCF9FBF7DEFFA4
:10BEA00020B157A240F24311FBF7B4F901F0C2FDF3
:10BEB00020B153A240F23B31FBF7ACF954490320C7
:10BEC000FDF7C6FB20B14EA24FF44271FBF7A2F979
:10BED00069460020FDF7DCFA20B149A240F20B319F
:10BEE000FBF798F99DF80000022877D05FF0000575
:10BEF000FDF70AFA03F024FBFEF710FE0021454887
:10BF000000F0F4FA20B13EA240F22231FBF782F9B0
:10BF1000AC216846FBF7D1FA02208DF80000012021
:10BF20008DF802000621ADF810008DF803103A4894
:10BF300005901EA8FBF78CFD3848299035486946C6
:10BF40002030FCF772FA20B12DA24FF43E71FBF7BE
:10BF500061F9304801212030FCF764FA30480024B0
:10BF6000CDE900402B4801A9143000F084FB20B13A
:10BF700023A24FF4D371FBF74DF92A48009068468D
:10BF8000FCF7BEFD20B11EA240F2AB11FBF742F957
:10BF90001C216846FBF791FA4FF4A030CDE9004030
:10BFA0004FF4F02002902048059003261F488DF89A
:10BFB0000C600690ADF80E408DF810406846FCF716
:10BFC00017FC20B10EA24FF4FD71FBF723F91848BE
:10BFD0001849401AC00806EB004000E00DE016A129
:10BFE00001F092FB2846FBF741FD00BF01F070FA1B
:10BFF0000028FBD101F046FDF8E7012578E70000B5
:10C000002E2E5C2E2E5C2E2E5C6D61696E2E6300D2
:10C01000859502003825002072220020C1E8020028
:10C0200019DB0200818D0200FDE80200A99D0200DB
:10C030007C450300D4440300427574746F6E6C65D4
:10C04000737320444655204170706C696361746954
:10C050006F6E20737461727465642E0070B514463F
:10C0600082880E4605462088111D0144921C994283
:10C0700001D8FE2A01D90C2070BD521C32542088F0
:10C08000FF21401C80B2208031542088401C80B2A7
:10C0900020808119288805F0C0FF2188084480B2DB
:10C0A0002080AA8842B1A96841B13044FBF7ECF97D
:10C0B0002088A98808442080002070BD072070BD1A
:10C0C0002DE9F047C5881E1DB6FBF5F78946B6FB7E
:10C0D000F5F1044605FB176C407916686843DDF8F6
:10C0E00020A0F718001F874200D9C61A166001E089
:10C0F0002468491E0029FBD1A5EB0C078846B742EE
:10C1000016D818E004EB0C00001D09EB0803BAF187
:10C11000000F3A4602D00146184600E01946FBF7E8
:10C12000B3F92468F61B4FF0000CB844B54201D9AE
:10C13000374600E02F46002EE4D1BDE8F08700002E
:10C1400030B5024651B101F07FFB0021074C08E0F9
:10C1500034F821301568AB4202D11160002030BDA7
:10C16000491C8142F4D3052030BD000000000000CE
:10C17000BFF35F8F00F016B9F8B50F46017814468B
:10C180000546012901D1687830B12088821C9A4285
:10C1900032D8012902D006E00720F8BD69780144B1
:10C1A000891C994228D8181A801E86B2ADF8006002
:10C1B0002188B81C084469467DDF0028EDD1297824
:10C1C000022904D06878BDF80020904205D3BDF85C
:10C1D0000000B04201D809200AE00820012905D159
:10C1E0006978B14202D8ADF8001001E0ADF8006006
:10C1F000BDF80010FE2901D90C20F8BD2288491C89
:10C20000B9542188491C89B2218078542088401C67
:10C210002080BDF80010084420800020F8BD0000F8
:10C22000034A00219268C0E9002181607047000044
:10C23000A023002070B586B00D4606461446142192
:10C240006846FBF73AF98DF80050ADF802402046F9
:10C25000FFF76AFAADF80400142269463046FBF78E
:10C2600013F906B070BD70B54FF6FF750E46A842C3
:10C2700001D1002000E0401C84B208E02146304695
:10C2800000F090F808B1204670BD641CA4B2FF2CE9
:10C29000F4D9284670BD10B5FBF715F808B1002099
:10C2A00010BD112010BD10B531B1B2FBF3F403FB8A
:10C2B00014241CB1092010BD0E2010BD0160002106
:10C2C000416081608281C381084610BD70B50C4613
:10C2D0000546FAF7ADFF002802D0218828680844F7
:10C2E00070BD10B50A8849888A4203D1FAF7E2FF87
:10C2F000012010BD002010BD70B50C460546FAF7B0
:10C30000BCFF002802D061882868084470BD10B5C1
:10C310000A8849888A4203D1FAF7A6FF012010BD96
:10C32000002010BD01F01F0301229A40D2434909A9
:10C3300000EB8100114600F059B80A4601F01F03D6
:10C340000121994010B552090C4600EB820000F023
:10C350005DF8204000D0012010BD2DE9F04180465D
:10C360000D460024481E012101EB501716E058F835
:10C370002400C04390FAA0F0B0FA80F020280CD23C
:10C3800000EB4416AE4208D231464046FFF7D5FFD7
:10C390000028ECD13046BDE8F081641CA742E6D805
:10C3A0002846F8E74A0950F8220001F01F0201214F
:10C3B0009140084000D00120704701F01F03012286
:10C3C0009A40490900EB8100114600F029B800218C
:10C3D00000F017B8012100F023B8012100F016B8D1
:10C3E00008B56A46FAF7BBFF009808BD08B56A466B
:10C3F000FAF79BFF009808BD08B56A46FAF7AFFF49
:10C4000008BD08B56A46FAF790FF08BD08B56A4648
:10C41000FAF77EFF08BD08B56A46FAF76DFF08BD5A
:10C4200008B56A46FAF774FF009808BD08B56A4671
:10C43000FAF7A2FF009808BD38B5044600258DF82C
:10C4400000506846FBF784FD2168626808689042E6
:10C450000ED9401E08600178238AE26801FB03259B
:10C46000227A2168101AC0B20A79824200D2087179
:10C470009DF80000FBF790FD284638BD38B505460D
:10C4800000208DF800000C466846FBF761FDE86867
:10C49000298A201AB0FBF1F12A681068431C136046
:10C4A00001709DF80000FBF777FD38BD10B530B185
:10C4B000017A42680368891AC9B21A6006E00E2040
:10C4C00010BD03681A68541C1C601170491EC9B263
:10C4D000F7D2006800210171084610BDC20800F0C3
:10C4E00007030120895C98400840704710B560B18F
:10C4F0000161172120F8021B20F8021B1B2100F804
:10C50000021BFFF7D5FA002010BD0E2010BD000061
:10C51000F0B5858893B00C46002D39D101880026EE
:10C520003F4F24293BD006DC102909D011290CD01B
:10C53000232958D14FE03A290BD0552953D129E06E
:10C540000146204602F0F4F94DE0A01DFFF7B0FAD5
:10C5500049E02246408934F8061F814200D8084647
:10C560006080172800D217206080106970B1607950
:10C5700060B1D7E90001CDE90301ADF80E50608844
:10C58000ADF81000136903A910469847667126712B
:10C5900013B0F0BD0146204602F054FA23E0011D1D
:10C5A0002C2206A8FAF770FFBDF81800BDF81C2071
:10C5B00004EBC0014A732269AAB1D7E90423CDE98B
:10C5C0000423ADF81200487B8DF814002269204640
:10C5D00004A9904707E0017A207B884200D20146F7
:10C5E0002846FDF737FCA07A0028D1D0E1882846FC
:10C5F000A5DF012580B11128CAD001F059FD0246FE
:10C600000848094913B0401AC00805EB0040BDE8CE
:10C61000F04006A101F07CB8A672E572B8E7000010
:10C6200084280300EC440300D444030073645F6275
:10C630006C655F67617474635F65786368616E677A
:10C64000655F6D74755F72657175657374282920F7
:10C6500072657475726E65642025732E000000008B
:10C6600020B10278DE2A03D0082070470E207047E0
:10C6700041800020704760B159B10278DE2A0AD0AB
:10C6800009684160DE2101704FF6FF714180002092
:10C6900070470E207047082070477FB50546002977
:10C6A0004DD0002D4BD008780C46DE2847D1A88805
:10C6B0006188884202D1204605F07CFD2888012847
:10C6C00025D002283BD011283AD0512837D135F84F
:10C6D000040F6188884232D1A978A81C02292ED182
:10C6E000017A042903D0062901D0052927D1002188
:10C6F000009102228DF8002001914FF4C072029146
:10C700000391ADF80420007A05280FD010E0297AB3
:10C710002046012913D1A988428891420FD10121D5
:10C72000017204B0BDE8704005F044BDADF80410DE
:10C7300028886946B0DF002801D0616888477FBD3E
:10C74000A88861888842FAD14FF6FF7060807FBD6B
:10C7500000F180400068002800D00120704708B533
:10C7600000F18040002101600068009008BD0000D9
:10C7700070B540F6F8700468601C02D14FF01020CC
:10C7800044691248124B4FF00102A3EB00004FEA3C
:10C79000D000611C02EB004512D0032101EB0040E8
:10C7A00022460CA100F0B4FF204613DF040005D0A0
:10C7B000284613A100F0A8FF204670BD002070BDE0
:10C7C00028461CA100F0A0FF042070BDD444030043
:10C7D0007C45030053657474696E672076656374E5
:10C7E0006F72207461626C6520746F20626F6F7469
:10C7F0006C6F616465723A203078253038780000BB
:10C800004661696C65642072756E6E696E6720732F
:10C81000645F736F66746465766963655F7665638C
:10C82000746F725F7461626C655F626173655F7380
:10C83000657400004E6F20626F6F746C6F61646589
:10C84000722077617320666F756E640070B50C4856
:10C850000C490D4A401AC508032000EB05400BA106
:10C8600000F056FF084813DF040007D0012000EB5A
:10C87000054011A100F048FF204670BD002070BDAA
:10C880007C450300D44403000070020053657474B7
:10C89000696E6720766563746F72207461626C657F
:10C8A00020746F206D61696E206170703A2030785D
:10C8B00025303878000000004661696C656420729C
:10C8C000756E6E696E672073645F736F66746465FE
:10C8D000766963655F766563746F725F7461626CBD
:10C8E000655F626173655F736574000070B50D4CC0
:10C8F0000125207808B185260EE00020A060606048
:10C900002061E060084801F017FC064601F00EFBCC
:10C9100008B901F0FBFB257001F0F0FB00B1A57038
:10C92000304670BD8C2D0020AD9C020038B500252E
:10C930008DF800506846FBF70BFB084CE068401E82
:10C94000E060E06828B901F0D9FB10B901F002FC01
:10C95000A5709DF80000FBF71FFB38BD8C2D002053
:10C96000F0B505460478154889B0164640F82420ED
:10C97000124A08690832A2F10C0742F82400487FE5
:10C98000385520226846FAF77FFD04942878385CF1
:10C9900048B10EB10A4A00E000226946281D01F0A4
:10C9A00065FE09B0F0BD0EB1064A00E000226946FE
:10C9B00005F10C0001F024FDF3E70000C023002086
:10C9C000D91E0300191D03000FB408B503990029EF
:10C9D00004D004AA00926A4600F00FF801B05DF896
:10C9E00014FB10B582680446002A05D0D4E904037C
:10C9F000216898470020A06010BD2DE9FC479146B2
:10CA00000C00804676D014F8011B39B125290ED0D0
:10CA10004046FCF799FF20780028F4D198F80C00E4
:10CA2000002867D04046BDE8FC47FFF7DABF00208A
:10CA3000012221782B291BD02D2902D0302908D1A1
:10CA400002E040F0010001E040F00200641C002A16
:10CA5000EFD100252A290ED02178A1F130020A2A2F
:10CA600011D205EB850201EB4205641C303DF1E774
:10CA700040F00400EAE7D9F800100B1DC9F80030B7
:10CA80000968641C0D44217800232E290BD114F869
:10CA9000011FA1F130020A2A05D203EB830201EB48
:10CAA0004203303BF3E76C290DD068290BD069298C
:10CAB00021D00BDC252918D0582931D063290ED07C
:10CAC000642915D117E014F8011FECE7702969D02B
:10CAD000732932D075291BD0782909D120E0D9F8E3
:10CAE0000000011DC9F8001001784046FCF72CFF3A
:10CAF000641C90E76CE0D9F800100A1DC9F800200A
:10CB00000968CDE900500A224046FEF7C3FEEFE770
:10CB1000D9F800100A1DC9F8002009680A2206E0A9
:10CB2000D9F800100A1DC9F8002009681022CDE9C3
:10CB30000050404605F086FADAE7D9F800100027E1
:10CB40000A1DC9F800200E68C00705D112E0404652
:10CB5000761C7F1CFCF7F8FE31780029F7D104E041
:10CB6000202140466D1EFCF7EFFEBD42C0D9002DCE
:10CB7000F6D1BDE74EB13046FAF7AAFC074604E00D
:10CB8000202140466D1EFCF7DFFEBD4206D9002D78
:10CB9000F6D103E04046761CFCF7D6FE317800293A
:10CBA000F8D1A5E7D9F80000011DC9F80010056803
:10CBB00030214046FCF7C8FE78214046FCF7C4FE11
:10CBC00008200021CDE90001034610222946B0E7E4
:10CBD000BDE8FC872DE9F843884605002C482D491F
:10CBE0009946A0EB01004FEAD0004FF00101164634
:10CBF00001EB004424D0286800282CD0002E34D02B
:10CC0000696840464FF010070A68511E11EA080F84
:10CC100011D1014672432846FAF7EBFE00282ED0C8
:10CC200028684B463246046901B041462846A4466E
:10CC3000BDE8F04360472046174B18A2009722E05A
:10CC40000E2000902046144B1EA220A100F06FFD84
:10CC50000E20BDE8F8830820009020460E4B26A247
:10CC60001AA100F064FD0820F3E709200090204697
:10CC7000094B24A215A100F05AFD0920E9E7064B53
:10CC8000214A2046009711A100F051FD1020E0E755
:10CC900064450300D44403004B2A030061646472BA
:10CCA0005F69735F706167655F616C69676E65641A
:10CCB00028705F66732C20706167655F61646472C1
:10CCC00029000000705F6673000000002573206378
:10CCD0006865636B206661696C656420696E2025F8
:10CCE00073282920776974682076616C7565203017
:10CCF0007825782E00000000705F66732D3E705F0F
:10CD0000617069006C656E00D03C030038B50300AB
:10CD10001148124D4FF00E04A0EB05004FEAD00071
:10CD20004FF0010505EB004009D061B119600C68B6
:10CD300001B0A446BDE83040114618466047084B94
:10CD400008A2009402E0064B08A2009409A100F09A
:10CD5000EEFC0E2038BD000064450300D4440300FF
:10CD6000002A0300705F667300000000705F61704E
:10CD700069000000257320636865636B2066616944
:10CD80006C656420696E2025732829207769746892
:10CD90002076616C756520307825782E00000000C3
:10CDA000044801214174007A08B100207047012035
:10CDB0007047000098300020012801D0032808D1D6
:10CDC0000449002201284A7400D00020087403F0AE
:10CDD0003BBC70479830002070B50246022801D055
:10CDE000032A45D1234C207A002841D0012833D092
:10CDF000022831D120480023022A006802D0032AE9
:10CE00002AD11BE0E360017911B1012924D10DE0A1
:10CE1000D0E90565711B4FF48056B14200D331460D
:10CE2000294481614569A9420ED015E00169491C78
:10CE30000161426991420FD1237213E0E168491CFC
:10CE4000E160082908D9E3602372022A0AD00D2183
:10CE5000FDF7B4FA03F09CFB607C28B1BDE870409C
:10CE600001F06AB80021F3E7BDE8704003F0ECBBC5
:10CE700070BD000098300020782400202DE9F84F84
:10CE800090468A463A493B4A0500A1EB02014FEA27
:10CE9000D1014FF00102DDF828901E464FF00E0040
:10CEA00002EB01441AD0B8F1000F1CD0286800280A
:10CEB00022D00920002E29D069684968B6FBF1F21A
:10CEC00001FB1261002926D000902B4B20462BA29B
:10CED00035A100F02CFC0920BDE8F88F0090204619
:10CEE000254B3CA203E00090234B20463BA22EA101
:10CEF00000F01DFC0E20EFE70820009020461E4B9E
:10CF000038A229A100F013FC0820E5E70090204694
:10CF1000194B37A2DCE75046FAF765FD102798B1A8
:10CF20004046FAF760FDA0B1324651462846FAF76E
:10CF300060FD98B1CDF80090286833464246C46839
:10CF400051462846A047C7E720460B4B29A2009729
:10CF500008E02046084B2DA2009703E0064B204630
:10CF600033A2009710A100F0E2FB1020B4E700000C
:10CF700064450300D4440300382A030021286C656B
:10CF80006E202520705F66732D3E705F666C617346
:10CF9000685F696E666F2D3E70726F6772616D5F5C
:10CFA000756E697429000000257320636865636BE2
:10CFB000206661696C656420696E202573282920CC
:10CFC000776974682076616C756520307825782ED5
:10CFD00000000000705F667300000000705F7372F5
:10CFE00063000000705F66732D3E705F61706900C2
:10CFF0006C656E00616464725F69735F616C696720
:10D000006E656433322864657374290061646472E8
:10D010005F69735F616C69676E6564333228287578
:10D02000696E7433325F7429705F73726329000014
:10D03000616464725F69735F77697468696E5F6267
:10D040006F756E647328705F66732C2064657374EB
:10D050002C206C656E2900002DE9FF411C46DDE99E
:10D060000A7815460E46684600F0C2F846EA4501C1
:10D0700041EA840141EA072242EA0841009A00EBB2
:10D080008200C0F80017BDE8FF812DE9FF411C4672
:10D09000DDE90A7815460E46684600F0B7F846EA1C
:10D0A000450141EA840141EA072242EA0841009A27
:10D0B00000EB8200C0F80017BDE8FF812DE9FF41B9
:10D0C0001C46DDE90A7815460E46684600F0ACF8C5
:10D0D00046EA450141EA840141EA072242EA084161
:10D0E000009A00EB8200C0F80017BDE8FF812DE92F
:10D0F000FF411C46DDE90A7815460E46684600F0F9
:10D10000A1F846EA450141EA840141EA072242EAE0
:10D110000841009A00EB8200C0F80017BDE8FF81CB
:10D120001CB5002100910B4601220191FFF7C6FFBB
:10D130001CBD1CB5002100910B4601220191FFF797
:10D14000D6FF1CBD1CB500220B4600921146019271
:10D15000FFF7B4FF1CBD1CB500220B460092114620
:10D160000192FFF7C4FF1CBD1CB5002100910B46C6
:10D17000012201911146FFF7A1FF1CBD1CB5002142
:10D1800000910B46012201911146FFF7B0FF1CBD33
:10D1900013B50C46684600F039F8009900EB8101A0
:10D1A000D1F8002722F44032C1F80027009900EBA3
:10D1B0008100D0F8001741EA0441C0F800171CBDF7
:10D1C0003CB50A4CD4E90034CDE900346B46441830
:10D1D00008E000BF53F82010D1F8205520C2C1F854
:10D1E0002055401C8442F5D83CBD00009C2903001A
:10D1F0000168202902D24FF0A040704701F01F01C2
:10D2000001600148704700000003005001682029B8
:10D2100002D24FF0A040704701F01F0101600148A9
:10D2200070470000000300500168202902D24FF02F
:10D23000A040704701F01F010160014870470000E5
:10D24000000300500168202902D24FF0A04070472F
:10D2500001F01F0101600148704700000003005009
:10D2600042094FF0000102D0012A05D102E04FF03F
:10D27000FF3101E040F2FF3100F01F000122824047
:10D280000A4201D0012070470020704701B568466E
:10D29000FFF7BCFFD0F810050099C84000F001006E
:10D2A00008BD01B56846FFF7BFFF009A0121914014
:10D2B000C0F8081508BD01B56846FFF7C3FF009A1E
:10D2C00001219140C0F8081508BD38B5012400902F
:10D2D000684631B1FFF78CFF00998C40C0F80845D3
:10D2E00038BDFFF785FF00998C40C0F80C4538BD6C
:10D2F000034908B50844002101600068009008BD9A
:10D300000060004002494058012800D000207047CA
:10D310000060004030B5154A01460020D2F81044A4
:10D3200023460AE0DB681D79854205D1401C0A28A6
:10D33000F6DB4FF0FF3030BD1B68002BF2D1431CF1
:10D34000F9D0CB681871D2F8103443B1DB68CC68DF
:10D350001B682360D2F81024D268116030BDC2F877
:10D360001014C96800220A6030BD0000503200204D
:10D37000F0B595B01C4615460F4608461A9E00F0BB
:10D3800033FB182109A8FAF798F80E96CDE909544D
:10D390000023082203A9384600F03BFB05980690BD
:10D3A000BDF81000ADF81C00BDF81200ADF81E006D
:10D3B00000208DF821000398082600F003000128C2
:10D3C00002D0022818D032E003983346850AC0F311
:10D3D000C2008DF8200003980FA9C0F38314A200A7
:10D3E000384600F016FB09A8009006AB22460FA9AC
:10D3F000284600F055FA1AE00398840DC0F3C200E5
:10D400008DF82000082C01D2254600E0082533467F
:10D410002A460FA9384600F0FCFA2E44641B09ABDB
:10D4200006AA29460FA800F0A3F9002CEAD1384635
:10D4300000F0E0FA15B0F0BD7047012004F08ABC9E
:10D44000084810B50178084A515C19B1001D01F077
:10D45000A7F902E00C3001F0A1F8BDE8104000206F
:10D4600004F078BCAC240020BC23002008B5034A9B
:10D4700000924023024AFFF77BFF08BDA110030082
:10D48000B83000200A4A012902EBC00007D0022967
:10D4900007D0032907D0042907D0002070470220B5
:10D4A000704704207047007970474079704700004A
:10D4B000D444030010B5FFF7C0FF04210348FFF771
:10D4C00029FF02490120C968487110BDC444030006
:10D4D0002DE9F04F8DB0FCF74FFA18B100200DB0D8
:10D4E000BDE8F08F7E4C4FF0000BC4F818B4BFF3CA
:10D4F0004F8F7C49A06802900D68D846284004EB05
:10D5000080000BE0D4F8180470B961680298814279
:10D5100001D8A160E2E7284004EB80000C3002A9AA
:10D52000FEF750FA0028EDD1002005AA029901EA81
:10D53000050304EB8303491CDB6842F82030401CE0
:10D5400002910228F2D3059800F00300022802D0CD
:10D5500001284DD0AAE005985022810D8946B2EBF2
:10D56000905F00D850210E4666F39F500590083119
:10D570005D4800F0F0F9070078D000F035FA434636
:10D58000082205A9384600F04CFA029908F1080A69
:10D590002940681A8000001D864222D9504D0C3562
:10D5A00030B1C2B204EB8101301A90460C3104E074
:10D5B0002946F2B2002590462846C6B25346384660
:10D5C00000F02FFA0AEB080325B132462946384607
:10D5D00000F027FA029909F1030001EB9000029094
:10D5E0003BE004EB81015346324638460C31EFE70D
:10D5F0000598C0F38310062800D30620059960F330
:10D600008911C1F38310801C05918100364800F018
:10D61000A2F907004AD000F0E7F94346082205A91D
:10D62000384600F0FEF908F1080800260FE00298DD
:10D63000434600EA0501401C04EB810102900422EC
:10D6400038460C3100F0EDF908F10408761C059815
:10D65000C0F38310B042EAD847B1D4F81054D4F8DC
:10D66000180478B1384600F0C5F934E01EE0E868E7
:10D670004079012804D12A68284639461268904723
:10D68000E8680568002DF2D1384600F0B3F98DF84E
:10D6900000B06846FAF75CFCD4F8180408B90298A0
:10D6A000A0609DF80000FAF777FC14E0D4F810446D
:10D6B00005E02168204689688847E0680468002CF6
:10D6C000F7D10A480A49401AC008022101EB00407C
:10D6D00008A100F019F8FCF74FF980F00100FEE610
:10D6E00050320020C82400209C4503007C450300E4
:10D6F000D44403004261636B656E647320666C758D
:10D70000736865640000000000231A4604F0A4B9A1
:10D7100008B5012300926A4604F09EF908BD1CB5C5
:10D72000CDE9002302236A4604F096F91CBD3EB5FC
:10D73000069C8DE81C0003236A4604F08DF93EBD6B
:10D740007FB5DDE908458DE83C0004236A4604F016
:10D7500083F97FBD70B586B00DF1280C9CE8700090
:10D760008DE87C0005236A4604F076F906B070BDAA
:10D770002DE9F0470E4680461C469246082940D8BF
:10D7800094F80C90002020731946104602F092FE87
:10D790000025B54206D218F805201BA12046FFF748
:10D7A00013F903E01AA12046FFF70EF96D1C082DAE
:10D7B000EFD318A12046FFF707F90025B54212D292
:10D7C00018F805707E2F08D8F9F75AFE0068C05D7A
:10D7D00010F03E0F01D03A4600E02E220EA1204666
:10D7E000FFF7F2F803E00DA12046FFF7EDF86D1CFE
:10D7F000082DE3D301222146504602F03DFE84F875
:10D800000C90BDE8F0870000202530327800000041
:10D81000202020007C000000256300002000000084
:10D82000064910B500200870054800F0E1F800280E
:10D8300003D1044800F07EF9002010BD50320020D2
:10D840009C450300202C030002480349401AC008ED
:10D85000704700009C450300D444030013B568469C
:10D86000FEF76EFC08B100201CBD0248009950F87C
:10D8700031001CBDD444030070B508480125D0F820
:10D880001044057007E0E06845712168204649684A
:10D890008847E0680468002CF5D170BD5032002044
:10D8A0002DE9FF4781460C9D00200C462F7B2873F5
:10D8B000984616462946184602F0FCFD072E42D22D
:10D8C000DFE806F004090F161F2A360049462846ED
:10D8D000FFF77AF837E0494628462268FFF774F8E0
:10D8E00031E0D4E9002349462846FFF76DF82AE0E5
:10D8F000A0680090D4E9002349462846FFF764F861
:10D9000021E0D4E90201CDE90001D4E90023494630
:10D910002846FFF759F816E004F1080007C88DE81B
:10D920000700D4E9002349462846FFF74DF80AE0EE
:10D9300004F108000FC88DE80F00D4E90023494620
:10D940002846FFF741F800222946404602F094FDA0
:10D950002F73BDE8FF872DE9F041058A80462D1F12
:10D960004819C01CB0FBF5F0C6B24046FEF764FD96
:10D97000041E19D00020207101206071E58000276D
:10D980002546761EC4F800800BE04046FEF754FDA5
:10D9900060B16179491C6171286005467F1CC0F83F
:10D9A0000080B742F1D32046BDE8F081204600F068
:10D9B00002F80020F8E72DE9F041457901466B1E99
:10D9C000002201E00968521C9A42FBD30F6801460D
:10D9D000002605E038460C68FEF750FD2146761C0F
:10D9E000AE42F7D3BDE8F0810121001DFEF7F8BC7F
:10D9F000FEF75CBD10B504460121001DFEF716FDC3
:10DA000010F0FF0F04D12046BDE81040FFF7D3BF50
:10DA100010BD1CB501920122009201AAFEF750FB35
:10DA20001CBD1CB501920022009201AAFEF748FB22
:10DA30001CBD00000F4910B500204870091D08608A
:10DA4000BFF35F8F0C490D4800F0C4FA0A480C4A36
:10DA50000121001FFAF7F2F9002809D10648002237
:10DA6000001F4FF480410068BDE81040FAF724BA67
:10DA700010BD0000A0240020AC2A0300AC30002020
:10DA800005DB020008B500208DF800006846FAF7B3
:10DA90005FFAF1EE100A20F09F00E1EE100ABFF3EA
:10DAA0005F8F08494020C1F880029DF80000FAF716
:10DAB00073FA00F03BFA08B141DF08BD20BF40BF58
:10DAC00020BF08BD04E000E070B504460C48012109
:10DAD000FEF7A1FCBFF35F8F0025002809D10120CC
:10DAE000074E042C08D0311F4A781AB1BFF35F8F5C
:10DAF000356070BD0C70487003F05AFCF6E700000A
:10DB0000A424002003484078002802D00420FFF716
:10DB1000DBBF7047A024002002A24FF4BE71F9F7CA
:10DB200079BB00002E2E5C2E2E5C2E2E5C6D616962
:10DB30006E2E6300826800219160826811618268A4
:10DB400051618268D160826851608068016070476D
:10DB500008B5002242504058009008BD20B103494A
:10DB600009680160002070470E207047A42C030054
:10DB7000FEB502460E460846FFF7F0FF002867D1C3
:10DB8000002500950195012706208DF80020ADF8AD
:10DB9000040002958DF8027069462020326869DF22
:10DBA0002C492D4A891AC908012202EB014430B1DF
:10DBB00000F07EFA024620462849FFF7A9FD0095AD
:10DBC0008DF801708DF80250019502958DF8035083
:10DBD00069464020326869DF30B100F069FA0246D8
:10DBE00020461F49FFF794FD0095019502958DF899
:10DBF000007069460120326869DF30B100F058FAE0
:10DC0000024620461749FFF783FD4FF4B0600090AD
:10DC1000019502956946A120326869DF30B100F0B4
:10DC200047FA024620461049FFF772FD009501951C
:10DC300002958DF800706946A020326869DF30B126
:10DC400000F036FA024620460849FFF761FD002041
:10DC5000FEBD00008C450300D4440300B042030025
:10DC6000F8420300104203005C420300BC41030081
:10DC70002DE9F0410546076860DF804619491A48DA
:10DC80002A68081AC608BA4219D9022000EB0644CD
:10DC900016A12046FFF738FD20463A461FA12B6803
:10DCA000FFF73DFD4FF08050D0F80C01296880024D
:10DCB00000F10050421A204625A1FFF729FDB8F1D6
:10DCC00000004FF001040AD000F0F2F9024604EB24
:10DCD00006402AA1FFF71CFD4046BDE8F0812F4811
:10DCE0000470F9E78C450300D4440300496E737552
:10DCF0006666696369656E742052414D20616C6C83
:10DD00006F636174656420666F7220746865205368
:10DD10006F66744465766963652E00004368616EC2
:10DD20006765207468652052414D20737461727478
:10DD3000206C6F636174696F6E2066726F6D203046
:10DD400078257820746F20307825782E0000000028
:10DD50004D6178696D756D2052414D2073697A650A
:10DD600020666F72206170706C69636174696F6E98
:10DD700020697320307825782E00000073645F627C
:10DD80006C655F656E61626C6528292072657475CB
:10DD9000726E65642025732E000000001F25002090
:10DDA00030B5154891B00078002822D05FF03404D7
:10DDB000ADF8404010A903A861DF48B1052818D08C
:10DDC00011B00EA2BDE8304040F23B11F9F722BA83
:10DDD00003AD1A49684600F0FDF806E0D0E90021DD
:10DDE00028469047684600F00CF902980028DFD0DA
:10DDF000F4E711B030BD00001F2500202E2E5C2E50
:10DE00002E5C2E2E5C2E2E5C2E2E5C2E2E5C636FD6
:10DE10006D706F6E656E74735C736F667464657637
:10DE20006963655C636F6D6D6F6E5C6E72665F7368
:10DE300064685F626C652E6300000000A82C03001C
:10DE4000F8B5134C2078C0B10120A07002F038FF63
:10DE5000112814D0022002F04BFF00258DF800504D
:10DE60006846FAF775F811DF064625709DF8000040
:10DE7000FAF792F82EB13046F8BD0820F8BD002020
:10DE8000F8BDA57003F03EFD032002F031FFF6E778
:10DE90001C2500207CB5194C207808B108207CBDD9
:10DEA0000120A070002002F00BFF112819D00020E3
:10DEB00002F01EFF12480026006801908DF80060F5
:10DEC0006846FAF745F80F4901A810DF05000AD0A7
:10DED000002020709DF80000FAF75EF82DB128466A
:10DEE0007CBD00207CBD0120F3E7A670667003F0C6
:10DEF00049FD012002F0FCFEF3E700001C25002094
:10DF00003C2C0300D97B02000EB50749684600F09F
:10DF100061F805E0D0E900108847684600F071F824
:10DF200002980028F6D10EBD582C03000148007855
:10DF3000704700001C2500200548817819B1007841
:10DF400018B1FFF77DBF08207047FFF7A3BF00009F
:10DF50001C2500201FB568464BDF40B1052816D0B0
:10DF600004B00BA2BDE810406B21F9F753B9184972
:10DF700001A800F02FF806E0D0E9002100989047B2
:10DF800001A800F03EF803980028E4D0F4E71FBD94
:10DF90002E2E5C2E2E5C2E2E5C2E2E5C2E2E5C2EBB
:10DFA0002E5C636F6D706F6E656E74735C736F66FD
:10DFB000746465766963655C636F6D6D6F6E5C6ECE
:10DFC00072665F7364685F736F632E6300000000A6
:10DFD000C42C0300016009684160AFF3008010B5F4
:10DFE000D0E900215368994201D1002104E0D1E930
:10DFF0000034A34202D01946816010BD083141604F
:10E00000F0E7816800290BD0026892680A448260B8
:10E0100041684B689A4203D108314160FFF7DFBF86
:10E02000704770B50D460646446804E0B26829465C
:10E03000904718B1246820680028F7D1206828602C
:10E04000256070BD40680068704741680868002816
:10E0500001D002680A60704702460020526806E05C
:10E060008B4203D108681060012070471A4613687C
:10E07000002BF5D1704700000C4A10B502F59473DF
:10E080000EE0991AC91001EBD171491002EBC101E0
:10E090000C68844201D90B4602E005D201F1080266
:10E0A0009A42EED3002010BD486810BDCC2A030070
:10E0B00000B5FFF7E1FF002800D1014800BD0000D6
:10E0C000B82A03004058002800D00120704708B546
:10E0D000002242504058009008BDD0F80403084088
:10E0E00000D0012070474058002800D00120704720
:10E0F00008B5002242504058009008BD0248006810
:10E10000002800D001207047000401400848006842
:10E11000012110F0010F06D14FF0E020C02280F85D
:10E1200000248430C1670349012008607047000063
:10E1300000E100E0180500400549024600200B7987
:10E140000BB1852070470A6001220A7170470000F8
:10E15000D0230020022010B54107C1F808034FF476
:10E160008270FEF7FCFA0549012008600448016846
:10E17000C1F300410029FAD110BD00000C0000409D
:10E1800018040040002802D0014980010847704768
:10E19000D12903002DE9F0410D46064601F02CFA85
:10E1A0000028304615D0FBF77DFC083802F05CF9FA
:10E1B000032802D001280AD003E03046FFF766F8B2
:10E1C00028B103213046BDE8F041FEF7E1BF02214E
:10E1D000F8E701F01DFA002822D03046FBF762FC78
:10E1E00004464FF4807000EB84000E4F81B207EBC1
:10E1F0008400D0F8102542F00102C0F8102508462E
:10E20000FFF776F8002D0BD03046FBF74BFC0649A4
:10E2100051F82000002803D00120A040C7F80403D3
:10E22000BDE8F08100600040A02D00202DE9FC41F8
:10E23000DFF8BC80044608EB0400002790F93000AA
:10E240001346C0170E46401C01D008274DE0B07899
:10E250001946C0F340022046FBF700FC0546401C6F
:10E2600042D0B07841071AD4C0070DD06846009458
:10E27000FEF7CCFF009900EB8101D1F8000720F0F8
:10E280000200C1F8000707E00021737820460091E2
:10E290000A460191FEF7F9FE204601F09FF9B07899
:10E2A000800718D51348317800EB8500D0F8102589
:10E2B000114B1A40C0F810254FF47C524FF44033F4
:10E2C00002EA042203EA01410A43D0F810150A4386
:10E2D000C0F8102509E008EB0500327810F8521F4D
:10E2E00041EA8211017000E004273846BDE8FC8154
:10E2F000A02D002000600040FFC0FCFF10B5FEF71D
:10E30000C5FF002800D0012010BD000070B5194DD8
:10E3100095F8640008B1082070BD0024661E2046F0
:10E32000FEF79EFF10B1281980F83060641CE4B23B
:10E330002A2CF4D300242046FBF782FB641CE4B2B1
:10E340000C2CF8D3002045F85E0F0C49A8800A4C2D
:10E35000C02081F8000401264020891FC1F8000177
:10E360004FF4BE70FEF7C4FFA004C4F80403AE71FE
:10E37000002070BDA02D00200060004006E000E0FD
:10E38000034890F86400002800D001207047000086
:10E39000A02D00200121B1EB507F01D10120704759
:10E3A0000020704738B50D4602F0D0F8040014D0B4
:10E3B00000208DF800006846F9F7CAFD207928B1E1
:10E3C0009DF80000F9F7E8FD112038BD0120256017
:10E3D00020719DF80000F9F7DFFD002038BD10B571
:10E3E00002F0B4F8002802D000210160017110BDD4
:10E3F0000149024803F0DABC082E0020002000404A
:10E400002DE9F0410546007916460F4600EB400124
:10E410002D4A01EBC00102EB810494F82A1011B1DE
:10E420000820BDE8F081294951F820102868FFF73D
:10E43000B9FF08B11120F4E739462846F9F7C6FDBF
:10E4400066603869206030004FF001062FD03F7FB2
:10E450004FF48E712868FFF73AFE4FF4A2712868D6
:10E46000FFF735FE28681A49C0F8041328684FEAF8
:10E47000471140F30730002804DB00F1E02080F86A
:10E48000001405E000F00F0000F1E02080F8141DFA
:10E49000286840F30730002809DB00F01F0106FA66
:10E4A00001F14009800000F1E020C0F80011286867
:10E4B0000421C0F800150020A061E06184F8290063
:10E4C00044F8140FA675ACE7082E0020A429030019
:10E4D000800002002DE9F05F054600790B4600EB55
:10E4E000400101EBC000244901EB8004284600F004
:10E4F00045F810B11120BDE8F09F62614FF00009AE
:10E50000C4F82090A36084F828904FF48E784E468B
:10E5100041462868FFF7DBFD28684FF0010AC0F884
:10E5200008A02146286803F0CDFB606808BBD5F839
:10E5300000B067690FE000BF94F8280008B10F260B
:10E5400015E041465846FFF7BDFD0028F4D02146AE
:10E55000584603F0B7FB206AB842F2D3574641460B
:10E560002868FFF7AFFD0028F9D02868C760C4F815
:10E5700014903046BFE70000082E0020007900EB21
:10E58000400101EBC000044901EB80004069002814
:10E5900000D0012070470000082E00202DE9F04730
:10E5A000044600794FF0000900EB400101EBC00088
:10E5B000284901EB80072068C0F800957868B0B161
:10E5C00020682549C0F80813206840F30730002868
:10E5D0000DDB00F01F02012191404009800000F195
:10E5E000E020C0F88011BFF34F8FBFF36F8F20681A
:10E5F000D0F80C25D0F81485D0F80865D0F810555F
:10E600004FF0FF31C0F81415C0F80C152068C0F8A1
:10E610000815C0F81015501C02D01046FEF780FDFA
:10E62000B8F1FF3F02D04046FEF77AFD681C02D0E9
:10E630002846FEF775FD701C02D03046FEF770FDCF
:10E640002068FFF7CCFE87F82A90C7F80490BDE851
:10E65000F0870000082E00208402020001490248D1
:10E6600003F052BC342E0020002000402DE9F04180
:10E670000546164600790F46154A00EBC00102EB2D
:10E68000810494F8201011B10820BDE8F0811149EF
:10E6900051F820102868FFF785FE08B11120F4E733
:10E6A00039462846F9F7CDFC6660386920601EB10E
:10E6B000397F2846FDF742F928680821C0F800157F
:10E6C0000020A061E0616061012184F82010DCE796
:10E6D000342E0020A82903002DE9F04704460E46F9
:10E6E0000079274900EBC00001EB80051746304652
:10E6F000FFF750FE30B1204600F044F820B1112061
:10E70000BDE8F0871020FBE76F61AE604FF49077B3
:10E710004FF0000839462068FFF7EAFC4FF4AC766A
:10E7200031462068FFF7E4FC2068AA686969C0F8F0
:10E730004425C0F8481520684FF00109C0F808903A
:10E740006868D0B9BA4651462068FFF7CCFC074646
:10E7500031462068FFF7C7FC0743F4D010B14FF0F3
:10E760000F0808E02068C0F80C9031462068FFF7D9
:10E77000BAFC0028F9D0002068614046C0E70000DC
:10E78000342E00200079054900EBC00001EB800029
:10E790004069002800D0012070470000342E00207E
:10E7A0002DE9F047064600793D4900EBC00001EB3A
:10E7B0008005346868680127A8B13A49C4F808138D
:10E7C000306840F3073000280DDB00F01F0107FA26
:10E7D00001F14009800000F1E020C0F88011BFF392
:10E7E0004F8FBFF36F8FD4F8000220F02000C4F8E1
:10E7F0000002A8694FF4A27820B141462046FFF7F5
:10E8000077FC67604FF4AC7949462046FFF770FC0F
:10E81000E760474649462046FFF765FC0028F9D0E7
:10E82000A86928B139462046FFF75DFC0028F1D0E1
:10E830004FF0000AC4F800A53068D0F80C25D0F8D5
:10E840001495D0F80885D0F810754FF0FF31C0F856
:10E850000C15C0F814153068C0F80815C0F810156C
:10E86000501C02D01046FEF764FCB9F1FF3F02D005
:10E870004846FEF75EFC781C02D03846FEF759FC8D
:10E88000B8F1FF3F02D04046FEF753FC2046FFF7A9
:10E89000A6FD85F820A0C5F804A0BDE8F08700001B
:10E8A000342E002010034200034908600348016829
:10E8B0000029FCD07047000004E5014000E401405D
:10E8C00010B568B103280FD10220FAF7B5FE002871
:10E8D0000AD0BDE8104005A24FF40B71F8F79ABCBE
:10E8E000BDE8104002F0A4BD10BD00002E2E5C2E2D
:10E8F0002E5C2E2E5C6D61696E2E63000078002800
:10E900000AD106483B21008876DF002804D004A203
:10E910004FF4EC71F8F77EBC7047000070220020C5
:10E920002E2E5C2E2E5C2E2E5C6D61696E2E630089
:10E9300070B58D88027900EBC5042273C97BA41DD4
:10E94000012902D0022904D101E0008800E04088BA
:10E95000208021886088814211D92846A5DF0126C0
:10E96000B0B1112816D0FFF7A3FB02460B480C49A3
:10E97000401AC00806EB00400AA1FEF7C9FEA179C3
:10E98000E079814208D92846BDE87040FBF762BAB9
:10E990006671F4E72671F2E770BD0000EC440300F5
:10E9A000D444030073645F626C655F676174746371
:10E9B0005F65786368616E67655F6D74755F7265CA
:10E9C000717565737428292072657475726E65643B
:10E9D0002025732E0000000070B588B00025064683
:10E9E000009502208DF800001448019502950395CA
:10E9F00000680490124C07A805906189A08804AAB9
:10EA0000ADDF48B907A8FAF777FC28B101208DF8E7
:10EA10000600ADF8045003E040F2FD10ADF804002C
:10EA2000A0886946B0DF1128FAD0BDF8040000289C
:10EA300002D13046FAF7DCF808B070BD8429030033
:10EA4000482D00207CB506468D88C88806EBC50495
:10EA5000A41D172800D217202188814200D808461B
:10EA600060800020207121882846B5DF60B1FFF763
:10EA70001FFB02460F481049401AC008012101EB54
:10EA800000400EA1FEF744FE6079002810D13069E5
:10EA900000280DD01549D1E90201CDE90001ADF8FA
:10EAA00002506088ADF804003269694630469047EC
:10EAB0007CBD0000EC440300D444030073645F6237
:10EAC0006C655F67617474735F65786368616E67B6
:10EAD000655F6D74755F7265706C79282920726549
:10EAE0007475726E65642025732E000084280300FF
:10EAF00048B1064A0168914205D14068044940186E
:10EB000002D0012800D0032070470000DEC0ADDE37
:10EB100002FEE10E8A7D022A04D90289CB881A44BA
:10EB2000D21C02814289C988511AC91E418170478D
:10EB30002DE9F0410D460221904600F580562980CE
:10EB400000F10804144F1BE031462046FCF76AFC34
:10EB500040B1B8F1000F02D0012288F8002002284D
:10EB600016D004E0A0687969884200D978612888C5
:10EB700061880844C01C2880608804EB80040C3441
:10EB800031462046FCF764FC0028DDD1BDE8F08169
:10EB90004FF480602880F9E74824002008B5002160
:10EBA000009101460823024A0248FEF767F908BDB2
:10EBB000E82903002425002008B50020009004481F
:10EBC0000823044A01680448FEF758F908BD00000C
:10EBD00070240020E0290300242500202DE9F05FA7
:10EBE0000026DFF81891DFF818B134464FF003081B
:10EBF000B2463746D9F80C0000EB07352846FFF738
:10EC000077FF98B301284BD0032869D12868411CAD
:10EC100002D03C49884205D10120820255F82010DB
:10EC2000491C0ED004EB84010BEB8102A8F101001A
:10EC3000556003221FFA80F80BF82120641CA4B24F
:10EC40004EE0401C9042E9D32F48016879B104EBB3
:10EC5000840002210BF820100BEB8000456001813D
:10EC6000274828304480641CA4B205E007E0022154
:10EC7000056081804FF0010A46F0010630E004EBA8
:10EC8000840100220BF821200BEB810101F110021D
:10EC90004D6028460831FFF74BFF46F00206CDE7EE
:10ECA000BAF1000F0FD004EB84000221164A0BF8D2
:10ECB00020100BEB80001268426001811048283060
:10ECC0004480641CA4B210480022011D056028463F
:10ECD000FFF72EFF0C48808802280CD0082006433E
:10ECE0007F1CBFB2032F85D3B8F1020F00D20026DC
:10ECF000F0B2BDE8F09F0420F1E7000024250020D9
:10ED0000C42F0020DEC0ADDE702400200149497808
:10ED1000F9F722BE982300202DE9F04188461749D3
:10ED2000174604468978F9F717FE08B1012600E076
:10ED3000022604F5807080B2072100F09DF90500DD
:10ED400013D0052D11D0FFF7B3F902460C480D4939
:10ED50002346401AC008012101EB00400A49FEF792
:10ED6000DEFC2946204602F087F93B464246314602
:10ED70002046BDE8F041FBF749B800009823002089
:10ED800014450300D44403004038030000B585B0A7
:10ED900003228DF800200288ADF802204079400758
:10EDA00001D5012000E002208DF808008DF809103F
:10EDB0006846FBF72FFC05B000BD002102F076BDD0
:10EDC00030B5154685B00C46024606216846FDF76B
:10EDD00031FA6846CDE90245FBF72AFC05B030BDA3
:10EDE00070B5054D06460024304655F82410884776
:10EDF000641C042CF8D370BDB42803007CB5164DF8
:10EE0000002400BF04EB440005EB800003F084FB0A
:10EE1000641C042CF6D3502104208A00CDE90001A3
:10EE20000F490E4B01F5A07000F030FC012468B1D1
:10EE3000FFF73EF902460B480B49401AC00804EBA5
:10EE400000400AA1FEF764FC03207CBD0348001FBC
:10EE5000447000207CBD00008C2C00202423002066
:10EE60003C2B0020FC440300D4440300504D5F427F
:10EE700055464645525F494E4954282920726574CB
:10EE800075726E65642025732E00000070B504460F
:10EE90000025C1681A4A284600EB400302EB8303B1
:10EEA0005B688B4204D100EB400002EB800003E082
:10EEB000401C0428F0DB00202178092904D00A290D
:10EEC00008D0142914D112E0617A89B980B103F015
:10EED00031FB0DE0617A59B950B100214160817A6E
:10EEE00041F00201817207490120087003E0012509
:10EEF0002046FFF775FF2846BDE8704001F042BC90
:10EF00008C2C002020230020002300F089B9000071
:10EF10007CB506460020019001A9304603F0E4FAD2
:10EF200004461A481A49401AC008012101EB00455D
:10EF300019E0A178304600F09FF860B105280AD0AA
:10EF4000FFF7B6F80246A0780090284633461149EC
:10EF5000FEF7EDFB18E0019801A9401C0190304636
:10EF600003F0C2FA0446002CE3D1304600F0F0F979
:10EF700000280AD0072808D0FFF79AF80346284649
:10EF800032460549FEF7CBFB03207CBDFC44030061
:10EF9000D4440300DC320300343303002DE9F0478E
:10EFA0001F00154681460E4604D0072E05D0082EB8
:10EFB00006D102E00E20BDE8F0870DB1042D01D985
:10EFC0000720F8E74FF00008484603F073FA041EE4
:10EFD00004D0207AA8420BD00F20ECE7FF214FF697
:10EFE000FF7003F067FA041E06D0A0F80090A67028
:10EFF000607AFF2802D00CE01120DCE729461A488D
:10F0000000F012FB014620466172FF2913D04FF039
:10F0100001082572617A144800F04AFB02000DD005
:10F02000ABB23146384600F01FFAB8F1000F19D0E4
:10F03000082E10D016E003F06FFADDE70B480C49FC
:10F04000627A401AC008012101EB00400949FEF72D
:10F050005FFB0320AFE738886FF0050101EB80000C
:10F06000796888800020A6E77C2C0020FC440300FF
:10F07000D44403006832030010B503F01BFA18B142
:10F0800003F058FA002010BD052010BD70B50C46E5
:10F0900006461546072901D0082C0ED1104600F06F
:10F0A00062F950B12146304603F004FA38B10580C8
:10F0B0008470BDE8704003F057B9072070BD05208B
:10F0C00070BD00004FF6FF71418001490968084793
:10F0D0009C28030070B588B02048FBF74DFC020067
:10F0E0001F4820494FF00105A0EB01004FEAD00076
:10F0F00005EB004406D020461B49FEF709FB032020
:10F1000008B070BDFBF74EFB020005D0204617A1EA
:10F11000FEF7FEFA8620F3E700F0F8F900200290EF
:10F120004CF2070603900EE0694604A8FBF7F2FBD9
:10F1300000988088A0F5404084B204A8FBF7A6FBA5
:10F14000204600F09FF902AA04A93046FBF7C9FB4C
:10F150000028E9D0154805700020D1E73DA602003F
:10F16000F4440300D444030080310300436F756C02
:10F1700064206E6F7420696E697469616C697A6568
:10F1800020666C6173682073746F726167652E20EE
:10F190006664735F696E697428292072657475727C
:10F1A0006E656420307825782E000000142300203E
:10F1B00000F08EB900F092B970B586B014460E46D4
:10F1C000054600F03FF940B105F5404080B20F4AD6
:10F1D0006946FBF786FB40B902E0012006B070BD2E
:10F1E00003A96846FBF796FB08B10020F6E7A57077
:10F1F0000398408820800498606003988088A0F578
:10F20000404030806846FBF741FBE6E718230020CA
:10F2100002480021416081607047000014230020F3
:10F22000F0B587B01F46154606460C46FF280AD89B
:10F23000084600F007F930B104AA2146304600F034
:10F24000E9F840B902E0072007B0F0BD02A904A820
:10F25000FBF760FB08B10520F6E7AC700298408828
:10F2600028807FB1840039682646B1EB800F00D238
:10F270000C46039922466868F8F706F9B44203D2AF
:10F280000C20E1E70398686004A8FBF7FFFA002070
:10F29000DAE7000070B586B016460D460446FF2832
:10F2A00028D8A87800F0CEF820B304F54040ADF897
:10F2B0000000A87803AA00F54040ADF80200686895
:10F2C000019028880290A978204600F0A3F805282C
:10F2D000694603A811D0FBF743FB024648F20661DA
:10F2E000401A8A4226D00BDCDAB1A2F50640023879
:10F2F0000AD121E0072006B070BDFBF739FBECE72F
:10F30000012815D0072813D00C480D492346401A70
:10F31000C008012101EB00400A49FEF700FA032072
:10F32000E9E71EB1314603A8FBF7EBFA0020E2E75C
:10F330001120E0E78620DEE71020DCE7F44403003C
:10F34000D4440300C43103004FF6FF7000F09AB8B4
:10F3500010B5FF2801D9072010BD00F099F800F082
:10F3600005F8002010BD00F0D7B80000F0B5244E1D
:10F370008DB00020707002904FF6FF750390284604
:10F3800000F0A6F8044648F2096706E0204600F0BF
:10F3900091F8204600F09CF80446AC422BD004F5CE
:10F3A000404080B202AA04A9FBF7A3FAB842EDD00C
:10F3B00004F5404080B2FBF7B1F905460120A5F500
:10F3C0000641073919D0002D15D00E490E4A2346A3
:10F3D000891AC90800EB01402A460C49FEF79FF93B
:10F3E00014220B4907A8F8F74FF8ADF8204007A8FA
:10F3F0000995FFF767FE0DB0F0BD7070FBE70000E8
:10F4000014230020F4440300D44403001C320300FE
:10F41000A02803007CB5054616460C46084600F0B9
:10F4200011F80020009005F54045019004F5404496
:10F43000A8B2A1B26B463246FBF74CFA002800D0C6
:10F4400005207CBD07280DD001280BD0082809D045
:10F45000052807D0062805D0092803D0042801D0A4
:10F46000002070470120704710B503EB83034FF66F
:10F47000FF7404EA03138170DB1C99084260018069
:10F4800010BD00000149FAF7DDBB0000BC2C0020D4
:10F4900010B50446A0F57F40FF3807D00449204648
:10F4A000FAF7D0FBA04201D1012010BD002010BD11
:10F4B000DC2C002010B50446044901F0DFFA0349B2
:10F4C0002046BDE81040203101F0D8BABC2C002005
:10F4D0000149FCF7C8BE0000DC2C002070B50A49C9
:10F4E000FCF7C1FE04464FF6FF7507E000F01EF87A
:10F4F00038B105492046FCF7B6FE0446AC42F5D1CA
:10F5000070BD204670BD0000BC2C00200148402189
:10F51000F7F7D3BFBC2C0020FF2803D801460248D0
:10F52000FCF740BF00207047BC2C0020FF2803D808
:10F5300001460248FCF736BF00207047DC2C002053
:10F540001CB500F041FC20B11C4A40F29521F7F7B0
:10F5500061FE0020009001909DF8000020F07E00E8
:10F5600040F00100303020F080008DF800000720CE
:10F570008DF8010010208DF802009DF8030040F086
:10F5800003008DF803009DF8040040F003008DF89F
:10F590000400684600F0F0FE20B1084A4FF42A71DA
:10F5A000F7F738FE064800F0D1FE002804D0034AE1
:10F5B00040F2AB21F7F72EFE1CBD000000C0020098
:10F5C0003DF702000068012805D0022803D0042876
:10F5D00001D00020704701207047000010B5054998
:10F5E000C20800F00703885C01249C402043885433
:10F5F00010BD0000FE2D00200449084490F93000A1
:10F60000082801DB0120704700207047A02D002052
:10F610000449084490F93000082801D201207047BD
:10F6200000207047A02D00202DE9F0410F46060074
:10F630002AD0306840B3706830B3FF24002520E042
:10F6400029467068FCF779FE80F00100BFF35F8FF8
:10F6500048B1FF2C00D12C46281B401CB8420ED1CB
:10F660002046BDE8F081FF2C06D108E02146304657
:10F6700000F032F8641CE4B2AC42F7D3FF246D1CF6
:10F68000EDB2B068A842DBD8FF20EAE770B5DDE94B
:10F69000044558B151B14BB104FB05F6964205D86B
:10F6A00024B11DB180E83A00002070BD072070BD74
:10F6B00070B504000D460DD0206858B1606848B19F
:10F6C000FF2D07D0FCF754FD20B1E168206805FB51
:10F6D000010070BD002070BD70B504000D4613D050
:10F6E0002068002810D0606800280DD0FF2D0BD0B6
:10F6F000FCF73EFD002807D060682946BFF35F8F06
:10F70000BDE87040FCF70EBE70BD0000034A5278A1
:10F710000AB101F0C9BE082070470000282300206C
:10F72000054A10B552782AB101F03CFF082800D1F3
:10F73000112010BD082010BD2823002010B504465C
:10F7400000F088F9204600F009F82046BDE8104096
:10F7500000F03EB8FAF748BFFAF746BF10B50446C6
:10F76000007804281CD10F480F496288401AC0084D
:10F77000022101EB00400DA1FDF7CAFF60881321B3
:10F7800076DF08280CD0A0F54051023908D00028B7
:10F7900006D0BDE810400D4A40F27921F7F73ABD96
:10F7A00010BD00000C450300D4440300446973639A
:10F7B0006F6E6E656374696E6720636F6E6E5F68EF
:10F7C000616E646C652025642E000000EC3503003A
:10F7D0002DE9F04105460178694C0020012686B0EC
:10F7E00004F1500716297DD2DFE801F00B8E8E2B35
:10F7F0008E8E8E368EA08EA08E8E8E8E8E8E8E8E5D
:10F80000A2BBA88800F056FC86280DD011280BD08A
:10F81000062879D0072877D0132875D0002873D010
:10F82000584A4FF4AE7144E06068A98827F8101078
:10F83000401CC11700EB517121F00701401A6060B4
:10F8400098E0287A012801D000285DD1A88806B068
:10F85000BDE8F04100F068BF2078002854D14A4844
:10F860004A49401AC708032000EB0740804648A1D8
:10F87000FDF74AFF607888B96846FBF795F8051EE2
:10F8800004D0404A40F28111F7F7C4FCBDF80600ED
:10F8900000B10120607088B1002D35D1FAF762FF08
:10F8A000002841D0A0F5064107392DD0354A4FF444
:10F8B000D37106B0BDE8F041F7F7ACBC00236A464F
:10F8C0001946184600F084FC050013D14046BDF8E7
:10F8D000002036A1FDF71CFFBDF8000000F0E0FBA2
:10F8E000051E00E010E012D0264A4FF4C671F7F76B
:10F8F00091FC6670052D0CD0062D0ED02846214AAD
:10F9000040F29911F7F786FC06B0BDE8F081667009
:10F91000C4E706EB074030A103E0022000EB0740FC
:10F9200035A1FDF7F1FEEFE72670EDE76670EBE736
:10F9300020706070656800244FF6FF766019C1176B
:10F9400000EB517121F00701401A07EB40010888D4
:10F95000B04202D00E8000F0E7FE641C082CEDDB04
:10F96000D2E72070A868A0F506410D3902D0B0F5A5
:10F97000064FC9D106B0BDE8F04100F05DB8000007
:10F9800038230020EC3503000C450300D444030069
:10F99000417474656D7074696E6720746F20636C58
:10F9A00065616E20666C6173682E000044656C654D
:10F9B00074696E67206C6F776573742072616E6B0B
:10F9C000656420706565722028706565725F696482
:10F9D0003A20256429000000546865726520617230
:10F9E00065206E6F20706565727320746F2064658A
:10F9F0006C6574652E000000506565722072616E42
:10FA00006B732066756E6374696F6E616C6974796F
:10FA10002069732064697361626C65642C20736F64
:10FA2000206E6F2070656572732061726520646559
:10FA30006C657465642E000000B585B0142204491D
:10FA40006846F7F721FD6846FFF7C2FE05B000BD26
:10FA5000F028030010B5044600F02CF82078A8B177
:10FA6000082819D10D480E49401AC008012101EBA0
:10FA700000400CA1FDF748FEA06800280CD0BDE8AE
:10FA800010400B4A40F22711F7F7C4BB6088BDE86D
:10FA900010400021FAF7DCB910BD00000C4503004E
:10FAA000D4440300417373657274696E672E00005D
:10FAB000EC3503002DE9FC5F044602785148524BB7
:10FAC0000321C01AC00801EB0047DFF834A102216E
:10FAD00001EB00450121AAF108080AF10C0B01EB2A
:10FAE000004608F12009162A71D2DFE802F0191940
:10FAF000190B1B19192A2D3448575B6369197119A1
:10FB00001919197A6088F8F7F7FE217A5AF8202037
:10FB10005BF821000090638838463CA1FDF707FEA2
:10FB2000BDE8FC9F6088F8F7E7FE237A5AF82020AA
:10FB300061895BF82300CDE90001638838464349B9
:10FB40001AE0284642A137E0A068FEF7B1FA024663
:10FB5000304645A14BE0207CC00701D03AA100E02F
:10FB60004CA1627A58F82200CDE90001217AA288DE
:10FB7000384659F821304A49FDF7E2FDD0E72069BF
:10FB8000FEF796FA627A58F82210CDE90010217A31
:10FB9000A288284659F821304249EDE7A28830462C
:10FBA00041A124E0A068FEF783FA0346A28830460C
:10FBB00047A111E0384652A1BDE8FC5FFDF7A4BDA6
:10FBC000A068FEF775FA0246304652A10FE013E036
:10FBD000A3886288284658A102B0BDE8F05FFDF70F
:10FBE0009EBDA068FEF764FA0246284661A102B0F5
:10FBF000BDE8F05FFDF78CBD28466AA1F7E700007D
:10FC0000482300200C450300D4440300436F6E6E6C
:10FC1000656374696F6E20736563757265643A20FD
:10FC2000726F6C653A2025732C20636F6E6E5F686F
:10FC3000616E646C653A2025642C2070726F636578
:10FC4000647572653A2025730000000034360300A5
:10FC5000466C6173682073746F72616765206973A5
:10FC60002066756C6C000000556E65787065637475
:10FC7000656420666174616C206572726F72206FBA
:10FC8000636375727265643A206572726F723A20AE
:10FC9000257300002C206E6F206368616E6765001D
:10FCA0008C37030040370300506565722064656C33
:10FCB00065746564207375636365737366756C6CD6
:10FCC000793A20706565725F69643A2025640000A6
:10FCD000506565722064656C6574696F6E2066613D
:10FCE000696C65643A20706565725F69643A2025C5
:10FCF000642C206572726F723A2025730000000038
:10FD0000416C6C2070656572732064656C65746508
:10FD1000642E0000416C6C20706565722064656C17
:10FD20006574696F6E206661696C65643A206572FE
:10FD3000726F723A202573004C6F63616C204442ED
:10FD400020636F756C64206E6F7420626520617033
:10FD5000706C6965643A20636F6E6E5F68616E6493
:10FD60006C653A2025642C20706565725F69643A81
:10FD700020256400466C6173682067617262616768
:10FD80006520636F6C6C656374696F6E2066616972
:10FD90006C65642077697468206572726F722025C3
:10FDA000732E0000556E657870656374656420502D
:10FDB0004D206576656E742049443A203078257868
:10FDC0002E000000FAF710BC70B5FFF783F9284940
:10FDD000284A891AC908012505EB014430B1FEF70C
:10FDE00067F903462046244A24A130E0FFF706F8CD
:10FDF00030B1FEF75DF9034620461F4A2AA126E0EE
:10FE000001F0A4FB30B1FEF753F9034620461A4A2D
:10FE100030A11CE001F0ACFC30B1FEF749F903461B
:10FE20002046154A36A112E0FBF7E8F830B1FEF79C
:10FE30003FF903462046104A3CA108E0FBF7B2F91F
:10FE400048B1FEF735F9034620460B4A42A1FDF7BB
:10FE500066FC032070BD4B4C4FF6FF70E080002025
:10FE6000A060A0706570F8F76BFD2070002070BD79
:10FE700004450300D4440300C4280300257320660E
:10FE800061696C6564206265636175736520706487
:10FE9000735F696E697428292072657475726E6566
:10FEA000642025732E0000002573206661696C654F
:10FEB000642062656361757365207064625F696E5A
:10FEC000697428292072657475726E6564202573C3
:10FED0002E0000002573206661696C6564206265F0
:10FEE000636175736520736D5F696E69742829207D
:10FEF00072657475726E65642025732E00000000B3
:10FF00002573206661696C65642062656361757341
:10FF10006520736D645F696E697428292072657449
:10FF200075726E65642025732E00000025732066AF
:10FF300061696C65642062656361757365206763E0
:10FF40006D5F696E697428292072657475726E65BB
:10FF5000642025732E0000002573206661696C659E
:10FF6000642062656361757365206773636D5F69A3
:10FF70006E697428292072657475726E6564202517
:10FF8000732E0000282300202DE9F041044686B09E
:10FF900001278088FBF712FB6080207800263F4D08
:10FFA000092808D00A2820D04FF6FF780B2829D03E
:10FFB0000C2853D158E0607A10B1012809D04DE0E7
:10FFC000A86830B1E168814203D1AE60A088E880C2
:10FFD00016E0A878E8B3A088E98888423ED1207A64
:10FFE00006283BD100F0AEFB38E0607A88BBA868F9
:10FFF00078B3E168814231D1AE60E868401EE860C4
:020000040003F7
:10000000E6602BE0E878E8B14046FFF7D3F84146D8
:10001000404517D10846FFF7CBF8404512D1EE70A6
:1000200014216846F7F749FA0D208DF80000ADF865
:100030000480ADF8028000272046FAF7D5FA68461A
:10004000FAF7D2FAA87838B1A088E988884203D1B3
:1000500000E003E000F076FB002F1CD006B0204645
:10006000BDE8F041FAF7C0BAE8780028F6D0EE70A3
:1000700014216846F7F721FA0E208DF80000ADF83C
:100080000480ADF80280A06802902046FAF7ACFA2E
:100090006846FAF7A9FA06B0BDE8F08128230020E7
:1000A0000349497809B1FBF729BB082070470000D4
:1000B00028230020F0B5324C064687B0607838B16E
:1000C0003049D1E90201CDE90501A07818B104E079
:1000D000082007B0F0BD00F035FBA078A168401EF5
:1000E000084301D0112547E0E088002786421CD153
:1000F000E068D0B1002514216846F7F7DEF9092041
:100100008DF800003046FBF759FAADF802000620E2
:100110008DF80800ADF804608DF8097003978DF82C
:1001200010706846FAF760FA26E0E068411C25D0B6
:10013000401C134AE060083205A93046FFF7AAF8D0
:10014000050019D0A760E068401EE060112D13D0B3
:10015000862D11D0072D0FD02846FDF7A9FF0246A6
:1001600009480A493346401AC008012101EB004002
:1001700007A1FDF7D4FA03252846AAE71325FBE7D4
:1001800028230020C428030004450300D4440300AE
:10019000436F756C64206E6F742075706461746554
:1001A0002072616E6B2E207064625F7261775F7384
:1001B000746F726528292072657475726E6564208B
:1001C00025732E20706565725F69643A202564008E
:1001D0002DE9FF4F344885B09946407892468B46CA
:1001E000C0B14FF6FF742046FEF7E4FF80460020C2
:1001F0000421CDE90210009003A8019002AB6A46E9
:1002000006214046FFF70CF800277E1E25460728EA
:1002100004D017E0082009B0BDE8F08F0520FAE708
:100220000398B84201D307464546B04201D206467C
:1002300044464046FEF7BEFF804602AB6A460621B2
:10024000FEF7EEFF0028EBD00528F2D04FF6FF7145
:10025000884519D18D4201D08C4201D1052000E0A2
:100260000020059901B10D80BBF1000F01D0CBF842
:100270000070BAF1000F01D0AAF80040B9F1000FE8
:10028000C9D0C9F80060C6E7FDF712FF024607486B
:1002900007494346401AC008012101EB00400549C7
:1002A000FDF73DFA0320B6E72823002004450300AC
:1002B000D4440300E8330300F0B51F4E85B07078D6
:1002C000D0B101274FF6FF74F7702046FEF772FF9A
:1002D0000546A0422BD10020F07014216846F7F7A4
:1002E000ECF80D208DF80000ADF80440ADF80240A8
:1002F0006846FAF779F91CE0082005B0F0BD00BFA8
:10030000FFF7CEFE78B1FDF7D3FE03460B480C494C
:100310000C4A401AC00807EB00400B490095FDF756
:1003200006FA0320E9E72846FEF744FF0546A54202
:10033000E6D10020E1E70000282300200445030067
:10034000D4440300E028030030340300084A517805
:1003500021B11179032903D3042070470820704785
:10036000044B43F82100491C117100207047000024
:1003700028230020FC2C00200349497809B101F012
:100380004DB908207047000028230020002801D024
:10039000FAF72AB9704700002DE9F84F314F0546AA
:1003A0004FF001090024381990F95A10491C46D021
:1003B00090F85A00294620F0C0063046FCF78EF827
:1003C00070B3204600F050F8824668460096FCF76D
:1003D0001DFF009900EB8100D0F80007C0F3014831
:1003E000B8F1020F1DD002213046FCF7D1FE68465D
:1003F0000096FCF70BFF009A09FA02F1C0F82015ED
:100400003046F9F74FFB57F820204AB15046BAF171
:10041000030F11D0B8F1020F05D0B8F1030F07D0C8
:100420000DE00321E0E75046BAF1010F04D006E0E9
:100430005046BAF1020F02D1014630469047641C83
:10044000042CB0D32A4602210020FCF7B9FE00207C
:1004500055F820100029A5D1401C0228F8D3BDE88A
:10046000F88F0000A02D00200249084490F85A009F
:1004700080097047A02D002010B50C46017A05298F
:1004800008D0407A38B1084808A102682046FCF735
:100490009BFA00E01AB106A12046FCF795FA204627
:1004A000BDE81040FCF79DBAF82400202573000039
:1004B0000D0A000038B5C3880D46044633B114A0B8
:1004C000009015A216A12846FCF77EFA217A05298C
:1004D0001CD0607A48B1A088FCF7D4FF164951F8C7
:1004E000202016A12846FCF76FFAA0880021FDF70E
:1004F000B5F903461049207A143951F8202001B08B
:100500002846BDE830400EA1FCF75EBA38BD0000B9
:100510001B5B306D000000001B5B313B33316D0015
:1005200025734C6F67732064726F70706564202848
:1005300025642925730D0A00F82400202573000086
:100540003C25733E2025733A200000000349884271
:1005500001D1034870470020704700000020004090
:10056000D82300200146054810B50068FBF7AEFE11
:1005700004461C21F6F7A1FF204610BDD829030030
:10058000014602480068FBF7C2BE0000D8290300FC
:10059000034802490068FBF7A4BE00007C24002049
:1005A000602A0300F0B5264D264E85B0044600278C
:1005B000686828B9224930680831FBF79DFE6860F9
:1005C00001460078072817D2DFE800F01604080873
:1005D0000E0E12002046FBF7F1F802E0204602F072
:1005E00039F8040029D009E02046F9F7ABFCF8E718
:1005F0002046FAF7CBFAF4E748F20E641421684675
:10060000F6F75BFFA4F5E8501D3800D100240194F3
:1006100069466868F9F788FE6846F9F7BFFE084939
:100620006F60002408313068FBF75BFE044801214D
:100630000C30FBF7FBFE0028BAD105B0F0BD00007E
:1006400048240020D82903002DE9F041234C00253F
:10065000234E207A012730B92248311D0068FBF76C
:100660004BFE306038B1022020723168087928B121
:1006700001281ED116E06560BDE8F081D1E90503CF
:10068000C01A4FF48052904200D31046B7EB900F3F
:1006900001D2820800E001220869C968184419449F
:1006A00029DF03E0D1E90301084428DF58B111280C
:1006B00012D003213068F9F781FE25726560BDE82C
:1006C000F041FFF765BF207C0028D5D1BDE8F0419F
:1006D00000210220FCF780BB2772CDE79830002074
:1006E00078240020602A030010B501210448FBF79C
:1006F00083FE002803D1BDE81040FFF753BF10BDB3
:100700005424002010B5074C201DFBF766FE00287E
:1007100006D1607C002803D1BDE81040FFF794BFEC
:1007200010BD00009830002010B586B0044614219A
:100730006846F6F7C2FEADF804406846FFF748F891
:1007400006B010BD0A4910B500231A46881FFFF7EE
:100750003FFD07490C39052803D038B100208870C7
:1007600010BD4FF6FF70C8800020C8600120F6E77A
:100770003423002010B510461A46F6F785FE0020F7
:1007800010BD00002DE9F0438146234885B0017873
:10079000002936D00021214F01700D4680460126E8
:1007A00005EB450007EB8004A07A810701D4C1075F
:1007B0002ED088F80060800702D4B9F1000F27D04E
:1007C000204601F0D1FD18B34FF6FF71ADF80210CD
:1007D0002188ADF80410862816D008218DF8001065
:1007E0000290FDF765FC02460D480E492388401A29
:1007F000C00806EB00400C49FCF791FF6846FEF785
:10080000EFFA05B0BDE8F08307208DF80000F5E7AA
:100810006D1C042DC4D3F4E7202300208C2C002071
:10082000FC440300D4440300883303002DE9F0475F
:10083000074620481C46154600780E4670B18DB11B
:1008400084B1DFF874804FF00009A08802282DD20F
:1008500000EB800118F8210020BB1BE048F201608A
:10086000BDE8F08748F20460FAE720681FB181888C
:100870003A8891420ED11EB101883288914209D145
:1008800080682860206868600B48283000892881CB
:100890000020E5E7A088214600F060F80028E4D1B8
:1008A000C4F80090A088401CA080CEE748F2096000
:1008B000D6E7000068240020C42F0020F8B50546C4
:1008C0004068244F0C46002648B32349CA68824238
:1008D00025D80969814222D3FBF7C2F8F8B12889EB
:1008E000398988421BD1D5E900018A68904216D126
:1008F0000020A7F1280200BF00EB800302EB830376
:100900005B688B4205D203F580538B4201D920806E
:1009100011E0401C80B20228EED30020F8BD2680F2
:1009200000960AE0009829688068884205D10098FE
:100930006860388928810120F8BD2088694600F068
:100940000DF80028EED12088401C80B220800228BB
:10095000E6D3E2E7EC2F00202425002070B50E46F8
:1009600000EB8001134800EB81004468306804F517
:10097000805518B1418800EB810411E0083410E083
:1009800029462046FAF74EFD20B1012805D002285D
:1009900007D10DE00120346070BD608804EB800455
:1009A0000C3429462046FAF753FD0028E8D170BDE3
:1009B000002070BDC42F002038B50C4600210091E6
:1009C00001460423084A0948FCF758FA10B148F2D6
:1009D0000D6038BD064A04EB840102EB8101012061
:1009E0000874002038BD0000DC2903002425002005
:1009F000C42F00202DE9F047884600EB80011E48F7
:100A00001D4600EB810016464168DDF8209001F19B
:100A1000080401F580571BE039462046FAF702FD2D
:100A200068B1012802D0022812D119E03088401C98
:100A30003080288861880844C01C288004E0B8F809
:100A40000000401CA8F80000608804EB80040C340F
:100A500039462046FAF7FCFC0028DDD1BDE8F087D6
:100A60003088401C30802988381B01EBA00028808A
:100A7000012089F80000F1E7C42F00200A46FF2872
:100A800003D801461046FBF74DBC70470846704737
:100A900070B50546F9F7A1FB134C40B1D4E9040247
:100AA0004FF08071411842F10000C4E904100021A8
:100AB0002846F9F7DFFA30B1606820B1606801F0CC
:100AC0004DF80020606001212846F9F7D3FA18B1EB
:100AD000FAF722FBC4E90601284601F08BF8284604
:100AE000BDE8704000F038B8182400202DE9F0412E
:100AF00000260E70D0E902740D468046FAF70CFB12
:100B0000381A002364EB01011A461B1A8A4115DAD0
:100B1000B0F5350F04D3F7F78BF90D49421800E013
:100B20003A464FF4960300210A48F9F762FB10B1E8
:100B30000D2807D00AE00120BDE8F081002105481A
:100B4000F9F78EFA404601F009F828700020F3E723
:100B5000FFFFB40020240020F8B5204C06460025F5
:100B60001F48FDF76FFA10B3D0E90210CA4372EACA
:100B7000000224D0626882B16368D3E90223891A33
:100B8000984127D26068D0E90210C94371EA000198
:100B900003D061681248FDF744FA00F03FFF0746B2
:100BA0006946FFF7A3FFB0B1606858B10DE0606817
:100BB00000280FD13046BDE8F840F9F716BB00F029
:100BC0002DFFCDE73046F9F70CFB67609DF800007C
:100BD0000028C5D1F8BD6560C2E7000018240020D8
:100BE000BC29030070B5054688690C4600284FF4FF
:100BF000847128460AD0FDF76AFAD5F81805626AAA
:100C0000E1688854606A401C606270BDFDF75FFA5D
:100C1000D5F8180570BD1FB501238DF80030CDE95A
:100C20000121D0E90012684690471FBD1FB501237E
:100C30008DF80030CDE90121D0E9001268469047D7
:100C40001FBD000010B50446064801792046F7F79D
:100C500083FE002804D12046BDE8104000F098BA79
:100C600010BD0000F822002038B50021012548B150
:100C7000012810D003280DD1FDF748FABDE838400F
:100C8000FBF754BE4FF0E020C0F88051BFF34F8F08
:100C9000BFF36F8F38BD8DF800106846F7F758F92D
:100CA000064C207808B9FBF721FEE068401CE060A4
:100CB000A5709DF80000F7F76FF938BD8C2D002066
:100CC0003EB5044609496846FDF784F908E000BFCF
:100CD000D0E900212046904730B16846FDF791F9F0
:100CE00002980028F4D13EBD11203EBD402C0300E7
:100CF0003EB5044608496846FDF76CF907E000BFB9
:100D0000D0E90021204690476846FDF77AF902981D
:100D10000028F5D13EBD00004C2C03002DE9FE4318
:100D200004460C3000278046FAF710FD4FF6FF7698
:100D30000546B042208803D1FAF7F6FC054602E0EA
:100D40002946FAF7D1FC20880022012100F008F999
:100D5000B54214D001AA07212846FEF7D5F870B98C
:100D6000029EA07D3436C00709D0307CC00705D173
:100D7000414606F11200FAF7A2FC00B13746002303
:100D800020881A46394686DF1649174A0646891AC8
:100D90004FEAD108082811D0BEB1FDF789F9024603
:100DA0000121009501EB084023881049FCF7BFFCA6
:100DB0002088314600F060F9BDE8FE83022101EB96
:100DC00008400B49FCF7A0FCF6E7A07DC007F3D074
:100DD000002FF1D12088002241F20601F9F779FABB
:100DE000EAE7000014450300D4440300D0370300B1
:100DF000583903002DE9FC4788460646274828490C
:100E00001C00A0EB01004FEAD0074FF00100914613
:100E100000EB074515D006F5807080B26B460122C5
:100E20000721FEF7BBF8112809D080B1FDF740F982
:100E30000246284633461B49FCF771FC0320BDE8F7
:100E4000FC872846184A19A1FCF762FCF6E75021F6
:100E50000198F6F732FB019981F800800198C4F8F7
:100E60000C90343020600198183020610198401CAB
:100E700060611B48E061019930461131FAF714FBBB
:100E80000028DCD0FDF714F90246022000EB0740F1
:100E900033461449FCF743FC0820D0E7144503000F
:100EA000D4440300203A03006C290300496E7465A2
:100EB000726E616C206572726F723A2025732072B7
:100EC00065636569766564204E554C4C20666F728B
:100ED00020705F7365635F6B65797365742E0000C6
:100EE000082D002008390300002835D0027891072A
:100EF00001D411062FD4C2F3021104292BD8930771
:100F000003D5032901D1110625D5437881788B4279
:100F100021D8072B1FD310291DD8C1784B071AD40D
:100F20000079430717D40B0715D4030713D4D2074E
:100F30004FEAC17201D042B10FE062B989070AD409
:100F4000C10708D1800706D407E0890705D4C10787
:100F500003D1800701D400207047012070470000B2
:100F6000F0B5154E14460F460A4685B00546317851
:100F7000F7F70AFD002F1AD00CB1012200E0002281
:100F800071782846F7F700FD012C12D00022B178C5
:100F90002846F7F7F9FC142208496846F6F774FA70
:100FA000ADF802508DF808406846F9F733FB05B0FC
:100FB000F0BD0122EBE70000982300200829030080
:100FC000F8B50446144800252E46806808B36088AA
:100FD000F7F742FCA0B100200090207A9DF8002095
:100FE000410861F3820260F3C302800860F30412D7
:100FF0008DF800206088694600F0FCFA80F0010658
:10100000608801B032462946BDE8F0400123FAF776
:1010100059BD0125F4E70000A023002010B586B0DB
:10102000044614216846F6F748FA05208DF80000BA
:10103000ADF802406846F9F7EDFA06B010BD0000C1
:1010400002498969002900D008477047CC2900204F
:1010500030B585B00C460546142206496846F6F7B9
:1010600013FAADF8025068460294F9F7A1FA05B0F8
:1010700030BD00001428030030B585B00C4605468D
:10108000142206496846F6F7FFF9ADF802506846A3
:101090000294F9F7BFFA05B030BD00001C29030027
:1010A00070B50E4C0020D2B22070201D0C4D03787C
:1010B000EB5C1BB1001DFDF70FFB02E00C30FDF7F0
:1010C00009FA18B1074A5321F6F7A4F86078002806
:1010D00002D021780029FAD070BD0000A824002099
:1010E000BC2300200C410300034800220149C078C2
:1010F000F7F7CCBB450C0300F822002070B51F4960
:1011000088B01F4CD1E900014FF6FF76CDE905010B
:1011100030E0002205A9FEF7BDF8050026D0142115
:101120006846F6F7CAF9A088ADF80400112D17D06B
:10113000862D17D02846FCF7BBFF024611481249FE
:10114000A388401AC008012101EB00400F49FCF7B9
:10115000E6FA08208DF8000002956846F9F736FA9D
:1011600008B070BD07208DF80000F6E7A088FEF7F4
:1011700021F8A080A088B042CBD1F1E76828030015
:1011800008230020DC440300D4440300402F030064
:101190002DE9F04F8DB0054601270026FAF714F926
:1011A0000446112821D005DC68B3062870D0082C2D
:1011B00008D134E0A4F54050023816D0A0F54070B4
:1011C000FF386CD02046FCF773FF0246364837499B
:1011D0002B46401AC008012101EB004034A1FCF766
:1011E0009EFA21462846FFF733FF414C3A462846EF
:1011F000E178F7F7C9FB21790DB032462846BDE802
:10120000F04FF7F7C1BB14223A496846F6F73CF9AC
:10121000ADF8025001266846F9F7CAF9E5E70DF185
:1012200014084FF0000901A8B3DFDFF8C8B00124AB
:101230000DF1180AABF1440B42F6052E1FE0DBF866
:101240000C00CDE9030A002206A92046B4DF70B9DC
:10125000BDF81810B9F1000F0BD0A1F524500238D9
:101260000BD103AA21462846CDF81080ADDF58B136
:101270000EE0714501D14FF00109641CA4B2BDF824
:1012800004008442DBD303E0BDF814000028ACD195
:1012900000272846FAF748FAF9F776FFA5E7284627
:1012A000FAF7ACFCA1E70000D4440300D4440300E7
:1012B0006773636D5F736572766963655F636861A9
:1012C0006E6765645F696E645F73656E642829206C
:1012D00072657475726E656420257320666F722066
:1012E000636F6E6E5F68616E646C653A20256400A2
:1012F000F82200203C2803002DE9F0410746806ACF
:1013000014468846C8B3002531E000BFB96A05EB32
:10131000450001EB8006B088801CFE2802D90C2015
:10132000BDE8F0812288401C08F8020020881622BF
:10133000401C80B2208008F800202088401C80B229
:10134000208000EB0801308800F067FE2188084407
:1013500080B22080B28842B1B16871B14044F6F7E2
:1013600093F82088B188084420806D1CEDB297F86E
:101370002C00A842CAD80020D2E7FFE70720CFE719
:101380000A78062822F0FF020A7010D2DFE800F087
:10139000030507090B0D002008E0112006E02120BD
:1013A00004E0312002E0122000E0222008707047A3
:1013B00070B51A4D1A4C07E001682078884700285C
:1013C0002BD01648FCF71DFEA8680028F4D1FCF7C6
:1013D00053FA00BFFCF77CF80028FBD120780328E3
:1013E00007D0022805D0FCF7A1FD78B133DF20BF7C
:1013F000FDE7BFF34F8F0B4801680B4A01F4E06132
:1014000011430160BFF34F8F00BFFDE70749012083
:101410000860BFF34F8F20BFFDE770BDAC300020E8
:10142000A02400200CED00E00400FA0500050040B7
:1014300010B50020F8F700F920B10CA240F21121FC
:10144000F5F7E8FEF8F740F820B108A240F21521C0
:10145000F5F7E0FEFCF7F4FC002806D0BDE81040EC
:1014600002A240F21A21F5F7D5BE10BD2E2E5C2E39
:101470002E5C2E2E5C6D61696E2E630010B500F03F
:10148000FDF8074C002205492079F7F7FFF960784D
:10149000BDE8104000220349F7F7F8B9BBED0200A0
:1014A000A0230020D1BB02002DE9FC410C0007461F
:1014B00014D0F7F733FA060013D03846FAF734F9A8
:1014C00005462078022E0FD020F00100A5F57F41BF
:1014D0002070FF390BD040F008000AE00E20BDE874
:1014E000FC8143F20200FAE740F00100EEE720F051
:1014F000080020703846F7F7AFF9217860F3410112
:1015000021703846F7F7E8F9217860F382012170FD
:101510003846F7F7D1F970B93846F7F79DF970B149
:1015200028466A460721FDF7EFFC40B9019890F87C
:101530004400C00703D0207840F0100002E020787B
:1015400020F0100020700020C9E7000010B51148FD
:10155000F9F78DFA0F48401CF9F789FA0D48801CFD
:10156000F9F785FA0B48C01CF9F781FA09480121FF
:10157000401E0279182A02D04171002010BD064891
:10158000064A801AC00801EB00400549FCF7BCF888
:10159000032010BDA12300201C450300D4440300F8
:1015A0009C2D030000230A461946FAF78BBA000067
:1015B00010B500780B2809D004DC092806D00A28C9
:1015C00011D103E00C2801D014280CD1074C0022C3
:1015D00005492079F7F75AF96078BDE810400022F4
:1015E0000349F7F753B910BDBBED0200A02300205B
:1015F000D1BB020038B50C4607490968009169461D
:10160000FFF752FF21789DF800209143084301D055
:10161000002038BD012038BD7C29030070B50B4C7B
:1016200005004FF001060CD0FFF75EFC58B12868AA
:1016300020612879207504F11000A0602670002038
:1016400070BD0020F9E7072070BD0000A023002036
:1016500010B504460078062802D0132809D105E009
:101660006088A168BDE8104000F020B92046FFF76F
:10167000A7FC2046BDE81040F8F7DABF30B50446B5
:10168000008885B014284FD00ADC11282CD01328EC
:1016900028D134F8040FF7F72FF901282FD038E0BC
:1016A000192847D01A281DD1A088FDF72FFB002844
:1016B00018D1A088F7F7D0F80028A0884BD02A4985
:1016C00000220978F7F760F903208DF80000A08860
:1016D000ADF8020000208DF808008DF8090068467A
:1016E000F8F798FF05B030BD207A3D2804D04FF4BC
:1016F0008851A088002224E041F23D01F9E72079D9
:10170000C00701D0012200E0022220880121FFF75A
:1017100027FC34F8045B142214496846F5F7B4FE3C
:10172000ADF802500294DAE705B0201DBDE8304064
:10173000FFF7F4BA217A201D41B14279008802F006
:10174000030205B0BDE83040FAF724BA05B0BDE8A1
:101750003040F6F7B3BC05B00122BDE8304041F29D
:101760000601F8F7B6BD00009823002058290300B1
:1017700010B51548F9F772F91348401CF9F76EF9DE
:101780001148801CF9F76AF90F48C01CF9F766F98F
:101790000D4801210278182A0BD04278182A08D067
:1017A0008278182A05D0C278182A02D00171002048
:1017B00010BD0648064A801AC00801EB00400549E2
:1017C000FBF7A2FF032010BD98230020144503005F
:1017D000D44403009C2D030070B50C460546F7F772
:1017E0008BF8012802D043F2020070BD21004FF0B7
:1017F0000000FAD028467EDF0428F6D1112070BD03
:101800002DE9F04188B017460D468046F7F774F889
:101810000446002620216846F5F74FFE012C01D032
:101820008CB105E01F480022C1784046F7F7ACF8BC
:1018300075B14046F9F778FFA0F57F41FF3915D023
:10184000012C07D012E043F2020008B0BDE8F0819D
:10185000852618E04046F6F767F938B94046FFF7A5
:10186000DDFB4046F6F760F900B985262878C00709
:1018700011D0852E07D06B463A4621464046FFF7E9
:10188000B9FA0028E1D1012C09D000226B4631467B
:1018900040467FDFD9E7044803970790F3E72A46DD
:1018A000F4E7000098230020082D00203EB50546EF
:1018B0000C466846FAF7B4FC6A4621462846FDF70E
:1018C0007FFA09480099C2682846FFF799FF044645
:1018D000014601222846F9F7EDF821462846009AEC
:1018E000F8F796FD3EBD0000A0230020002805D19A
:1018F0000349012048700020F8F7C4B97047000080
:101900008C2D002010B51620F5F7A4FF48B10D4826
:1019100082684FF4800162B1016821F480010160A6
:1019200010BDBDE8104042F2010007A2AD21F5F75D
:1019300071BC4FF0E020C0F88011BFF34F8FBFF3B0
:101940006F8F10BD002F00202E2E5C2E2E5C2E2EB1
:101950005C2E2E5C2E2E5C2E2E5C636F6D706F6E77
:10196000656E74735C736F66746465766963655CD9
:10197000636F6D6D6F6E5C6E72665F7364682E630D
:101980000000000010B51620F5F764FFA0B1124862
:1019900090F800044009082811D20121814011F07B
:1019A000EC0F0CD00D4882684FF480017AB10168C9
:1019B00041F48001016010BD42F2010001E042F2F9
:1019C0000200BDE8104006A2A121F5F723BC4FF0AC
:1019D000E020C0F8001110BD16E000E0002F00204C
:1019E0002E2E5C2E2E5C2E2E5C2E2E5C2E2E5C2E31
:1019F0002E5C636F6D706F6E656E74735C736F6673
:101A0000746465766963655C636F6D6D6F6E5C6E43
:101A100072665F7364682E63000000000148FCF783
:101A200014BB0000BC290300C207002A03D000BF7A
:101A30004FF00F0201E04FF0F00201D04FEA011128
:101A4000044B03EB5003187800EA020040EA01005F
:101A500018707047582E00202DE9F84F074622488D
:101A60009146884605681E46012269461846F7F7E2
:101A700021FFDFF878A060B3009800210446801CA5
:101A80000AE000BF00EA050259F821C00AEB820211
:101A9000401C491CC2F80CC0B142F3D34FEA1749AD
:101AA000F8F7D4FA611C29400AEB810149EA0042A7
:101AB0002C40CA600AEB8401C86867F3C50066F36E
:101AC000891068F39F2020F00300401C20F00400E0
:101AD000C8609AF8000001E0FBF7FAFC0028FBD18F
:101AE000FAF772F9BDE8F88FC824002050320020C0
:101AF0007CB5054614480C460022D0E90510CDE916
:101B00000010124841792846F6F73EFF14B10E48FE
:101B1000001D01E00C48083001902846F9F704FE4A
:101B200000226946FDF7B6FB00280CD0FCF7C0FA8E
:101B3000024607480749401AC008022101EB00404D
:101B40000549FBF7E5FD7CBDF8270300F8220020DE
:101B5000D4440300D44403000C2E0300F8B504461B
:101B600022480026007878B374B3F9F7D5FAD4E99F
:101B70000232C01A91412DD300258DF800506846DD
:101B8000F6F7E6F9206910B9681EC4E902009DF86D
:101B90000000F6F701FAD4E9051088478DF80050E7
:101BA0006846F6F7D5F922697AB1D4E90210CB4339
:101BB00073EA000309D089186841C4E902109DF84E
:101BC0000000F6F7E9F909E00DE09DF80000F6F7EE
:101BD000E3F908E0D84370EA020004D02146044843
:101BE000FCF71FFA01263046F8BD0000182400203B
:101BF000BC29030038B51D4D69462868FAF77CFBFF
:101C00001B4C30E0017821B101290ED0022922D1EC
:101C100017E04168D1E90220D24372EA00021AD0EB
:101C200012480830FCF7FDF915E041686068814210
:101C300002D1002060600EE00C480830FCF70CFA7E
:101C400009E0FFF7EBFE20B14FF0FF31C0E90211D0
:101C5000F7E70120207069462868FAF742FB6946D9
:101C60002868FAF749FB0028CCD138BDB429030015
:101C700018240020F8B50B4C0D460646694620682E
:101C8000FAF724FB58B10670456069462068FAF7F8
:101C90003EFB10B10448F8F78DFA0020F8BD04208F
:101CA000F8BD0000B4290300202400200348806808
:101CB0004108034800224068F6F7FEB8E023002000
:101CC000AC29030070B50C4605464FF48E71FCF745
:101CD000FEF9216AA068415C206A401C2062C5F8B8
:101CE0001C1570BD1FB500228DF80020029181687F
:101CF00001914261D0E90012684690471FBD1FB5AF
:101D000000228DF800200291816801914261D0E9A2
:101D10000012684690471FBD1FB50A4601788DF82E
:101D2000001041680191017A8DF80810C068039095
:101D3000044850F82210083850F82220684690478E
:101D40001FBD0000C8230020014901200870704712
:101D5000A824002010B588B0044620220F49684608
:101D6000F5F792FB06200090C01F019002900390AF
:101D70004FF0EB7006900CB1094A00E00022694672
:101D80000848FAF7EDFD18B1074A4321F5F742FA82
:101D90000448001F447008B010BD0000002C030070
:101DA000491D0300AC2400200C4103002DE9FF472E
:101DB0000C4605464FF40071FCF78FF901274FF4EC
:101DC0000178002618B34FF4927949462846FCF76B
:101DD00079F9E0B149462846FCF779F9C5F8088356
:101DE00094F8290000B96F6002208DF80000D5F842
:101DF0008004C5F880040390A0690290E068019017
:101E0000A661E661D4E900126846904728E0042103
:101E10002846FCF762F918B34FF484712846FCF7A2
:101E200051F9E8B121462846FEF7DCFE616AA06957
:101E3000884215D1E06938B1E268616AA061206921
:101E4000E6616662E06008E094F8290000B96F601E
:101E5000C5F80883A661E268616A2046FEF7DBFEEA
:101E60004FF48E7841462846FCF72CF980B1606922
:101E7000216A814202D294F8280028B341462846BC
:101E8000FCF725F9606918B161692046FFF72AFF60
:101E90004FF4A27841462846FCF714F9002818D0E0
:101EA00041462846FCF713F994F8290000B12F6049
:101EB000A06900280DD0A661E268616A04B02046DE
:101EC000BDE8F047FEF7A7BE21462846FFF7FAFE19
:101ED000DEE7BDE8FF8700001FB50A4601788DF8F0
:101EE000001041680191017A8DF80810C0680390D4
:101EF000044850F82210083850F8222068469047CD
:101F00001FBD0000C82300202DE9FF410C464FF4FF
:101F1000927705463946FCF7E6F80026B8B139460F
:101F20002846FCF7E5F802208DF80000D5F880047B
:101F3000C5F880040390D5F83C050290E068019054
:101F4000A661E661D4E900126846904723E04FF4A9
:101F5000887739462846FCF7C6F8E0B13946284666
:101F6000FCF7C6F8D5F83C15A069884213D1E069A2
:101F700060B1E268D5F8000220F02000C5F8000248
:101F8000E069A0612069E661E06001E0A661E268C5
:101F90002046FEF74BFE4FF4A27739462846FCF761
:101FA000A2F868B139462846FCF7A2F8A06938B112
:101FB000A661E661D5F83C152046E268FEF736FEDC
:101FC0004FF4907631462846FCF78DF860B13146E3
:101FD0002846FCF78DF80120E860606920B1D5F84B
:101FE0004C152046FFF78BFE4FF4AC763146284661
:101FF000FCF779F800280ED031462846FCF778F82F
:102000006069002807D0D5F84C1504B02046BDE81B
:10201000F041FFF774BEBDE8FF810870000A487008
:102020000220704710B514210448F5F746FA044819
:102030000068FAF730F9002010BD00009830002049
:10204000602A03002DE9F05F8346DDE90A4A9946DC
:1020500090460D460846012703E000BFB0FBF8F0AC
:102060007F1C4045FAD2B94500D94F465FEACA7095
:1020700012D18CB15FEA8A7002D5B9F1000F01D09C
:10208000202607E0302605E031465846641EF7F763
:102090005BFC0CB1A742F7D35FF00106B9F1010F69
:1020A00002D9A9F1010903E0B5FBF6F0404502D3DE
:1020B00006FB08F6F2E7DFF83C9000BFB5FBF6F050
:1020C00000FB165519F800105846F7F73DFCB6FB13
:1020D000F8F6002EF2D15FEACA7009D0002C07D0C2
:1020E000A74205D220215846641EF7F72DFCF5E7DC
:1020F000BDE8F09FF029030010B5094C0022074904
:102100006078F6F7C3FB002806D16079BDE810407F
:1021100000220449F6F7BABB10BD0000159F02006B
:10212000F8220020019A0200F8B5054680B2F9F7BE
:10213000A7FB040013D0154E207A0027317B88427C
:102140000ED2A8B204F10A0175DF28B1112806D019
:10215000BDE8F840FEF774BF207A401C2072F8BD3D
:102160002772307C38B1A8B23B2176DF18B108283D
:1021700001D0FEF765FF71690029F0D08DF800707D
:10218000ADF8025068468847F8BD0000CC29002011
:10219000417939B190F82E1421B990F8300408B182
:1021A000012070470020704701460148FAF7FAB84D
:1021B000E829002030B40446007A00280AD060885C
:1021C000002166DF28B1112802D0616830BC0847C1
:1021D0000120207230BC704770B50C460546F7F7F9
:1021E000D7FB002807D04268002A04D021462846A1
:1021F000BDE87040104770BD2DE9FC411646DDE991
:102200000854CDE900541F468046022200F00CF825
:10221000002807D1CDE900543B4610223146404604
:1022200000F002F8BDE8FC812DE9FC5F0026DDE945
:102230000C4B994692468E4680462788354630E0BC
:10224000D8F80400002200EB850069460068019080
:1022500001A864DF002830D19DF8000050451FD14F
:102260000EB1002100E002212288084411185945CE
:1022700022D846B9521C90B2208009F800E020888C
:10228000401C20800126218801A801EB0902694633
:1022900064DF002811D120889DF8001008442080B8
:1022A0006D1CB8F80000A842CADC56B12088C01BDB
:1022B000401E80B2FF2802D90C20BDE8FC9F09F81F
:1022C00007000020F9E7000010B504281DD209B16D
:1022D000032400E00024F7F739F8202802D24FF059
:1022E000A04102E00A4900F01F0001EB8000D0F895
:1022F000001721F44031C0F80017D0F8001741EA68
:102300000441C0F80017002010BD062010BD0000D9
:1023100000030050002070472DE9F84F114D88460A
:1023200081461E4617466946DDF828A02868F9F759
:10233000CDFF040013D01C21F5F7BFF80020207159
:10234000C4F80090C4E90486C4E902A76946286875
:10235000F9F7DDFFFEF7D6F90020BDE8F88F04207D
:10236000FBE70000602A03002DE9FC410446002041
:1023700000900190A0788DF80200617A2D48FDF759
:1023800097F92D492D4A891AC908012606EB0145FE
:1023900080B10246A178237A6846FDF765F89DF87A
:1023A000020001280ED006280CD0072808D00828E3
:1023B00011D10AE0627A284621A1FBF7A9F91FE0B2
:1023C000142006E0ADF8006005E00198808809302F
:1023D0008008ADF800002088221D6946FCF75AFFEE
:1023E00088B107280DD02649112811D0862818D089
:1023F000FBF75EFE02462388284622A1FBF78FF9F1
:102400000320BDE8FC81A17A21F00301A172F8E765
:10241000A07A20F0010040F00200A0720E700020AF
:10242000EFE7A27A22F0020242F00102A2720E70DD
:10243000E7E700007C2C0020FC440300D4440300A8
:10244000706D5F6275666665725F7074725F6765F6
:1024500074282920636F756C64206E6F7420726518
:102460007472696576652052414D206275666665B5
:10247000722E20626C6F636B5F69643A2025640082
:10248000202300207064735F706565725F646174FF
:10249000615F73746F726528292072657475726E3E
:1024A00065642025732E20706565725F69643A202B
:1024B0002564000038B505460C46002001E0009870
:1024C000401C00906946284600F00EF800280AD00B
:1024D0008178A142F3D1817A8A07F0D4C907EED17D
:1024E00041680029EBD138BD10B50A4B0A680CE0F1
:1024F00002EB420433F82440844205D102EB42004F
:1025000003EB80000A6010BD521C042AF0D30020A7
:1025100010BD00008C2C00204FF6FF710180FF21C0
:1025200081704172817A21F0030181720021017270
:102530004160704770B50546002406E0687A204483
:10254000C1B20648FDF7C8F8641C287AA042F5D845
:102550002846BDE87040FFF7DFBF00007C2C00205C
:102560002DE9FC47064639489846144600780D4642
:102570004FF0000978B37DB32888A0F57F41FF397B
:1025800033D0688848B36868F9F76AFA80B384B3CF
:102590002088ADF80000678801A8FDF7E3FF04007C
:1025A00034D084F800804FF0000A84F816A0BDF8FB
:1025B0000000A08268682061244801210C38F9F7E6
:1025C0000FFFE060288820816888A080E780B8F14C
:1025D000030F23D026E001E004E006E048F20160AA
:1025E000BDE8FC8748F20460FAE748F20360F7E7C9
:1025F00000E002E048F20260F2E72889694687B20B
:10260000384600F0AFF80028EAD1C5E7BDF8001061
:10261000384600F09BF848F20760E1E70420A07517
:102620003068A061A4F80A9001A8FDF7A9FF46B19F
:10263000C6F804A0E1680648316086F80AA000895F
:102640003081FEF751F80020CAE70000682400201E
:10265000EC2F00202DE9F8430D46898A384A01EB1A
:10266000810102EB810638B129463046FCF752FA67
:102670004FF40640BDE8F88331897068002400EB10
:1026800081072F48A97DA83848F20D6807294FD245
:10269000DFE801F00D2E172504414B004460A969C5
:1026A000016027482749A838FEF708F930B1022011
:1026B000A875042339462A1D009424E048F20960D5
:1026C000D8E728692A4608B1032000E00120907568
:1026D000042305F10C0207F10801009413E0012026
:1026E000A8750094E88807F10C0183002A690AE0C4
:1026F00028782A4603280CD006209075042305F17B
:102700000802391D00941048FAF7B8FBB0B14446EE
:1027100010E00520F1E70621A9750A4940680988FB
:10272000FEF74AF9040005D108E041F61D5401E026
:1027300048F20E6429463046FCF7ECF9204699E74A
:10274000C42F0020482400202425002001EB810212
:10275000034901EB82014A89101AC01E4881704763
:10276000C42F002070B5C01C82B240F2FE308242FD
:1027700002D948F2086070BD114B00204FF480650B
:1027800000EB800413F8246096B903EB84063489C7
:10279000768914443444A4B2AC4209D8088000EBD2
:1027A000800003EB8000418911444181002070BD0D
:1027B000401C80B20228E3D348F2066070BD0000DE
:1027C000C42F00200D0E0F100B0C181988220020AA
:1027D000A8220020C82200200B000300E994020078
:1027E0000C000300E994020018000300E9940200C1
:1027F00019000300E99402000100FFFF010000003E
:1028000000000000020000000000000001000900BC
:1028100000000000080000000000000000000000B0
:1028200000000000000000000700000000000000A1
:102830000000000000000000000000001100000087
:102840000000000000000000000000000000000088
:102850001200000000000000000000000000000066
:1028600000000000010000000100010064280300D6
:10287000010001007828030000000000C5FD0200EF
:10288000C1AF0200770A000000000000770A0000D4
:10289000000000007ADA0000000000008DEE020067
:1028A0000800000000000000000000000000000020
:1028B0000000000089FF0200B115030091B302007F
:1028C00091B00200706D5F696E69740001000600CE
:1028D00034230020706D5F706565725F6E657700F0
:1028E000706D5F70656572735F64656C65746500BB
:1028F00007000000000000000000000000000000D1
:10290000000000005116030002000000000000005B
:1029100000000000000000000000000008000000AF
:1029200000000000000000000000000000000000A7
:102930000700000000000000000000000000000090
:102940000000000004000000000000000000000083
:102950000000000000000000060000000000000071
:102960000000000000000000000000007365635FCD
:102970006B65797365745F66696C6C00E0000000DC
:102980008D030300020000000000000050EADA306E
:102990008883B89F604F15F30000C98E0000005077
:1029A00000030050F1E302005DE6020003000000B6
:1029B000F8230020982E00200100060000000000EF
:1029C00038240020C99C0200000000000000000024
:1029D0000338FDD8704700000C2F00200000FFFFD7
:1029E000DEC0ADDEFF011EF1DEC0ADDEFE011EF178
:1029F0003031323334353637383941424344454635
:102A00006E72665F6673746F726167655F696E6927
:102A100074006E72665F6673746F726167655F756E
:102A20006E696E6974006E72665F6673746F726150
:102A300067655F72656164006E72665F6673746F6E
:102A4000726167655F7772697465006E72665F6652
:102A500073746F726167655F657261736500000012
:102A6000FC2F002000100000040000000100000006
:102A700089B702002520030075070300192303000E
:102A8000DDA202008D0A030015230300F9B902003C
:102A9000B0450300B4450300000000000000000042
:102AA000000000000000000080240020902A0300A5
:102AB000A82A030004000000556E6B6E6F776E202D
:102AC0006572726F7220636F646500000000000021
:102AD0009840030001000000443F03000200000092
:102AE000383D030003000000B83F0300040000006D
:102AF0000C40030005000000EC3E0300060000004F
:102B0000883E030007000000F43F030008000000B7
:102B1000003F030009000000643F03000A000000BA
:102B2000804003000B000000203D03000C0000006B
:102B3000183F03000D000000E84003000E000000F5
:102B4000E43F03000F0000002040030010000000DD
:102B50005440030011000000FC400300120000007C
:102B6000D0400300130000006C4003008000000010
:102B7000A03E030081000000DC3D03008200000055
:102B80009C3D0300830000007C3D030084000000A6
:102B9000B83D030085000000C43E0300860000002D
:102BA000CC3F030090000000683E0300910000004D
:102BB0005C3D0300920000002C3F030000820000F7
:102BC0003440030001820000803F030002820000C5
:102BD0009C3F030000840000F83D030001840000D6
:102BE000A440030002840000403E03000384000070
:102BF0001C3E03006DD4020041D4020039D402000F
:102C0000FFFFFFFFFFFFFFFFFFFFFFFFFFFFFFFFD4
:102C100000000000000000000000D60106010000D6
:102C2000B83100207F00000038320020FC4503004E
:102C3000044603000000000000000000010000073F
:102C40002C2C03003C2C030008000000642C030023
:102C5000742C030008000000742C0300842C030073
:102C6000080000002C46030044460300000000005A
:102C7000000000001C4603002C460300000000007A
:102C800000000000B4450300BC450300BC45030040
:102C9000E4450300E4450300F4450300F445030064
:102CA000FC45030070220020842C0300A42C0300A8
:102CB0000800000004460300144603001446030005
:102CC0001C460300B42C0300C42C030008000000C1
:102CD000004040404040404040404141414141402F
:102CE00040404040404040404040404040404040E4
:102CF0004005020202020202020202020202020273
:102D00000220202020202020202020020202020277
:102D100002029090909090901010101010101010CF
:102D200010101010101010101010101002020202DB
:102D3000020288888888888808080808080808081F
:102D4000080808080808080808080808020202021B
:102D500040000000D12C03004661696C656420745A
:102D60006F20646973636F6E6E65637420636F6E4A
:102D70006E656374696F6E2E20436F6E6E6563744B
:102D8000696F6E2068616E646C653A202564204529
:102D900072726F723A20256400000000436F756CF8
:102DA00064206E6F74206163717569726520636F52
:102DB0006E6E5F7374617465207573657220666CE6
:102DC0006167732E20496E63726561736520424CA2
:102DD000455F434F4E4E5F53544154455F555345F5
:102DE000525F464C41475F434F554E5420696E2019
:102DF00074686520626C655F636F6E6E5F7374618B
:102E00007465206D6F64756C652E0000434152201F
:102E1000636861722076616C756520636F756C64A0
:102E20006E27742062652073746F72656420286554
:102E300072726F723A202573292E20526561747464
:102E4000656D70742077696C6C2068617070656E58
:102E5000206F6E20746865206E65787420636F6ED5
:102E60006E656374696F6E2E000000006773636D9A
:102E70005F6C6F63616C5F64625F63616368655F11
:102E80006170706C7928292072657475726E656442
:102E90002025732077686963682073686F756C6498
:102EA000206E6F742068617070656E2E20636F6E87
:102EB0006E5F68616E646C653A20256400000000F6
:102EC000546865206C6F63616C2064617461626139
:102ED000736520686173206368616E6765642C2088
:102EE000736F20736F6D65207375627363726970A1
:102EF00074696F6E7320746F206E6F746966696396
:102F00006174696F6E7320616E6420696E646963B9
:102F10006174696F6E7320636F756C64206E6F747B
:102F200020626520726573746F72656420666F72CB
:102F300020636F6E6E5F68616E646C65202564004F
:102F40007064735F706565725F646174615F7374F0
:102F50006F726528292072657475726E656420250C
:102F600073207768696C652073746F72696E67206F
:102F700073657276696365206368616E6765647303
:102F80007461746520666F72207065657220696473
:102F90002025642E0000000073645F626C655F672B
:102FA000617474735F696E697469616C5F75736570
:102FB000725F68616E646C655F6765742829207252
:102FC000657475726E65642025732077686963681F
:102FD0002073686F756C64206E6F74206861707008
:102FE000656E2E0044696420616E6F74686572209E
:102FF000746872656164206D616E6970756C61746E
:103000006520504D5F504545525F444154415F49F2
:10301000445F474154545F4C4F43414C20666F72AC
:1030200020706565725F6964202564206174207476
:1030300068652073616D652074696D653F207064FB
:10304000625F77726974655F6275665F72656C65F1
:1030500061736528292072657475726E6564202518
:10306000732E000073645F626C655F6761747473D4
:103070005F7379735F617474725F7365742829205C
:1030800072657475726E6564204E52465F45525289
:103090004F525F494E56414C49445F444154412090
:1030A000666F72204E554C4C20706F696E7465725D
:1030B0002077686963682073686F756C64206E653B
:1030C0007665722068617070656E2E20636F6E6E1B
:1030D0005F68616E646C653A2025640073645F62AA
:1030E0006C655F6761705F646174615F6C656E677A
:1030F00074685F7570646174652829202872657131
:103100007565737429206F6E20636F6E6E656374CE
:10311000696F6E20307825782072657475726E65DF
:10312000642025732E000000546865207265717557
:10313000657374656420636F6D62696E6174696F35
:103140006E206F6620545820616E642052582070A3
:1031500061636B6574206C656E6774687320697356
:1031600020746F6F206C6F6E672062792025752048
:103170006D6963726F7365636F6E64732E00000018
:10318000436F756C64206E6F7420696E6974696139
:103190006C697A6520666C6173682073746F726104
:1031A00067652E206664735F726567697374657204
:1031B00028292072657475726E65642030782578D0
:1031C0002E000000436F756C64206E6F7420777260
:1031D000697465206461746120746F20666C61732A
:1031E000682E206664735F7265636F72645F7B77BD
:1031F000726974657C7570646174657D28292072BC
:10320000657475726E656420307825782E2070653F
:1032100065725F69643A202564000000436F756C35
:1032200064206E6F742064656C65746520706565DC
:103230007220646174612E206664735F66696C65D8
:103240005F64656C65746528292072657475726E9B
:103250006564203078257820666F7220706565720D
:103260005F69643A2025640043616E6E6F74207359
:10327000746F7265206461746120746F20666C6184
:103280007368206265636175736520706D5F627538
:10329000666665725F7074725F6765742829206363
:1032A0006F756C64206E6F742072657472696576D8
:1032B000652052414D206275666665722E20497305
:1032C00020626C6F636B5F6964202564206E6F748D
:1032D00020616C6C6F63617465643F007064625F51
:1032E00077726974655F6275665F72656C6561733C
:1032F0006528292072657475726E656420257320B7
:1033000077686963682073686F756C64206E6F748A
:103310002068617070656E2E20706565725F6964EB
:103320003A2025642C20646174615F69643A202529
:1033300064000000506565722049442025642077B0
:103340006173206E6F742070726F7065726C79207B
:1033500072656C65617365642E207064735F70655F
:1033600065725F69645F667265652829207265749D
:1033700075726E65642025732E20706565725F69B5
:10338000643A202564000000536F6D652070656508
:1033900072206461746120776173206E6F74207095
:1033A000726F7065726C79207772697474656E20C3
:1033B000746F20666C6173682E2077726974655F24
:1033C0006275665F73746F72652829207265747503
:1033D000726E656420257320666F72207065657259
:1033E0005F69643A20256400436F756C64206E6FDA
:1033F000742072657472656976652072616E6B7394
:103400002E207064625F706565725F646174615FD5
:103410006C6F616428292072657475726E65642012
:1034200025732E20706565725F69643A20256400FB
:1034300025732829206661696C6564206265636173
:1034400075736520612063616C6C20746F20706DF2
:103450005F706565725F64656C65746528292072AC
:10346000657475726E65642025732E2070656572B3
:103470005F69643A202564004F7574646174656403
:1034800020283029000000004F7574646174656461
:1034900020283229000000004F757464617465644F
:1034A0002028332900000000706D5F636F6E6E5F2F
:1034B0007365637572652829206661696C6564208F
:1034C0006265636175736520616E20534D50207491
:1034D000696D656F75742069732070726576656EAD
:1034E00074696E67207365637572697479206F6E95
:1034F00020746865206C696E6B2E20446973636F5D
:103500006E6E656374696E6720636F6E6E5F68616F
:103510006E646C652025642E00000000706D5F6392
:103520006F6E6E5F736563757265282920666169C9
:103530006C6564206265636175736520636F6E6E90
:103540005F68616E646C65202564206973206E6F0E
:103550007420612076616C696420636F6E6E6563B0
:1035600074696F6E2E000000706D5F636F6E6E5F2A
:103570007365637572652829206661696C656420CE
:1035800062656361757365207468652073746F721A
:103590006564206461746120666F7220636F6E6E73
:1035A0005F68616E646C6520256420646F657320BC
:1035B0006E6F74206861766520612076616C696445
:1035C000206B65792E000000426F6E64696E672083
:1035D00064617461000000004170706C6963617423
:1035E000696F6E2064617461000000002E2E5C2EF5
:1035F0002E5C2E2E5C2E2E5C2E2E5C2E2E5C636F8F
:103600006D706F6E656E74735C626C655C70656521
:10361000725F6D616E616765725C706565725F6D2A
:10362000616E616765725F68616E646C65722E635E
:1036300000000000436F6E6E656374696F6E2073E7
:1036400065637572697479206661696C65643A2096
:10365000726F6C653A2025732C20636F6E6E5F6805
:10366000616E646C653A20307825782C2070726F1A
:103670006365647572653A2025732C206572726FDC
:10368000723A202564000000496E76616C696420FE
:10369000526F6C650000000052656D6F74652064A8
:1036A00061746162617365004C6F63616C20646179
:1036B0007461626173650000557064617465000037
:1036C00044656C65746500005365727669636520B6
:1036D0006368616E6765642070656E64696E6720FB
:1036E000666C616700000000426F6E64696E67007F
:1036F00050616972696E6700506565722072616E13
:103700006B0000005065726970686572616C000042
:1037100043656E7472616C00456E63727970746992
:103720006F6E000043656E7472616C206164647238
:10373000657373207265736F6C7574696F6E0000CA
:103740005065657220646174612075706461746590
:1037500064206661696C65643A20706565725F69B2
:10376000643A2025642C20646174615F69643A20A6
:1037700025732C20616374696F6E3A2025732C20A9
:103780006572726F723A2025730000005065657291
:103790002064617461207570646174656420696E71
:1037A00020666C6173683A20706565725F69643A7F
:1037B0002025642C20646174615F69643A2025735C
:1037C0002C20616374696F6E3A20257325730000A5
:1037D000436F756C64206E6F7420636F6D706C65E1
:1037E000746520656E6372797074696F6E20707293
:1037F0006F6365647572652E2073645F626C655FCC
:103800006761705F7365635F696E666F5F72657035
:103810006C7928292072657475726E656420257331
:103820002E20636F6E6E5F68616E646C653A202552
:10383000642C20706565725F69643A2025642E00EF
:10384000436F756C64206E6F7420636C65616E20CD
:103850007570206166746572206661696C656420AC
:10386000626F6E64696E672070726F6365647572F3
:10387000652E207064625F77726974655F62756639
:103880005F72656C65617365282920726574757255
:103890006E65642025732E20636F6E6E5F68616EA7
:1038A000646C653A2025642E0000000052414D20D2
:1038B00062756666657220666F72206E657720623B
:1038C0006F6E642077617320756E617661696C61DB
:1038D000626C652E207064625F77726974655F62E6
:1038E00075665F67657428292072657475726E65E8
:1038F000642025732E20636F6E6E5F68616E646C4A
:10390000653A2025642E0000696D5F626C655F6119
:103910006464725F67657428292072657475726EBD
:1039200065642025732E20636F6E6E5F68616E6420
:103930006C653A2025642E204C696E6B207761738C
:10394000206C696B656C7920646973636F6E6E655A
:10395000637465642E00000073645F626C655F676A
:1039600061705F7365635F696E666F5F7265706CCF
:103970007928292072657475726E6564204E5246EE
:103980005F45524F525F494E56414C49445F535434
:103990004154452C20776869636820697320616E03
:1039A0006572726F7220756E6C65737320746865D2
:1039B000206C696E6B20697320646973636F6E6E2F
:1039C000656374696E672E00436F756C64206E6F5B
:1039D000742073746F726520626F6E642E20706441
:1039E000625F77726974655F6275665F73746F7228
:1039F0006528292072657475726E65642025732EA2
:103A000020636F6E6E5F68616E646C653A2025643A
:103A10002C20706565725F69643A2025640000009F
:103A2000436F756C64206E6F742072657472696583
:103A300076652052414D2062756666657220666F1C
:103A40007220696E636F6D696E6720626F6E642E9F
:103A5000207064625F77726974655F6275665F6724
:103A6000657428292072657475726E6564202573EB
:103A70002E20636F6E6E5F68616E646C653A202500
:103A80006400000043616E6E6F742073656375722D
:103A900065206C696E6B206265636175736520617A
:103AA0002070726576696F757320736563757269CE
:103AB00074792070726F63656475726520656E64D9
:103AC000656420696E2074696D656F75742E20447D
:103AD0006973636F6E6E65637420616E64207265D6
:103AE0007472792E20736D645F706172616D735FA3
:103AF0007265706C792829206F7220736D645F6C19
:103B0000696E6B5F736563757265282920726574D1
:103B100075726E6564204E52465F4552524F525F39
:103B200054494D454F55542E20636F6E6E5F68614A
:103B30006E646C653A20256400000000436F756C6C
:103B400064206E6F7420706572666F726D2073658D
:103B50006375726974792070726F636564757265DC
:103B60002E20736D645F6C696E6B5F736563757235
:103B70006528292072657475726E65642025732E20
:103B800020636F6E6E5F68616E646C653A202564B9
:103B900000000000436F756C64206E6F74207065C8
:103BA00072666F726D2073656375726974792070C7
:103BB000726F6365647572652E20736D645F7061EA
:103BC00072616D735F7265706C792829206F722045
:103BD000736D645F6C696E6B5F7365637572652886
:103BE000292072657475726E65642025732E2063BA
:103BF0006F6E6E5F68616E646C653A2025640000CC
:103C000054686520626F6F746C6F616465722068C0
:103C100061732077726974652070726F7465637464
:103C20006564206974732073657474696E677320AA
:103C3000706167652E20546869732070726F6869BF
:103C4000626974732073657474696E672074686543
:103C5000206164766572746973696E67206E616D48
:103C6000652E2054686520626F6F746C6F616465A7
:103C700072206D75737420626520636F6D70696C5E
:103C800065642077697468204E52465F424C5F53EA
:103C9000455454494E47535F504147455F50524F3A
:103CA000544543543D3020746F20616C6C6F772015
:103CB00073657474696E67207468652061647665E5
:103CC00072746973696E67206E616D652E00000005
:103CD000616464725F69735F77697468696E5F625B
:103CE0006F756E647328705F66732C2070616765F2
:103CF0005F616464722C20286C656E202A20705FDE
:103D000066732D3E705F666C6173685F696E666F87
:103D10002D3E65726173655F756E697429290000B7
:103D20004E52465F4552524F525F494E56414C49A2
:103D3000445F4441544100004E52465F4552524F49
:103D4000525F534F46544445564943455F4E4F5486
:103D50005F454E41424C4544000000004E52465FD4
:103D60004552524F525F464541545552455F4E4F62
:103D7000545F454E41424C45440000004E52465F60
:103D80004552524F525F4D555445585F554E4C4F1A
:103D9000434B5F4641494C45440000004E52465F4C
:103DA0004552524F525F4D555445585F4C4F434B0F
:103DB0005F4641494C4544004E52465F4552524F82
:103DC000525F4D555445585F434F4E445F494E49ED
:103DD000545F4641494C4544000000004E52465F46
:103DE0004552524F525F4D555445585F494E4954C4
:103DF0005F4641494C4544004E52465F4552524F42
:103E0000525F424C455F495053505F52585F504B90
:103E1000545F5452554E4341544544004E52465F00
:103E20004552524F525F424C455F495053505F508C
:103E30004545525F52454A45435445440000000001
:103E40004E52465F4552524F525F424C455F495079
:103E500053505F4C494E4B5F444953434F4E4E4580
:103E600043544544000000004E52465F4552524FB5
:103E7000525F4150495F4E4F545F494D504C454D44
:103E8000454E5445440000004E52465F4552524F45
:103E9000525F4E4F545F535550504F52544544005B
:103EA0004E52465F4552524F525F4D4F44554C451E
:103EB0005F4E4F545F494E495449414C495A45441D
:103EC000000000004E52465F4552524F525F4D4F28
:103ED00044554C455F414C52454144595F494E4918
:103EE0005449414C495A4544000000004E52465F37
:103EF0004552524F525F4E4F545F464F554E44000D
:103F00004E52465F4552524F525F494E56414C49C0
:103F1000445F5354415445004E52465F4552524F00
:103F2000525F444154415F53495A45004E52465FE7
:103F30004552524F525F494F5F50454E44494E479C
:103F4000000000004E52465F4552524F525F53569A
:103F5000435F48414E444C45525F4D495353494E8F
:103F6000470000004E52465F4552524F525F494E45
:103F700056414C49445F4C454E47544800000000B0
:103F80004E52465F4552524F525F4452565F54570D
:103F9000495F4552525F414E41434B004E52465F8E
:103FA0004552524F525F4452565F5457495F4552F3
:103FB000525F444E41434B004E52465F4552524F72
:103FC000525F494E5445524E414C00004E52465F9E
:103FD0004552524F525F53544F524147455F4655E9
:103FE0004C4C00004E52465F4552524F525F4E5568
:103FF0004C4C00004E52465F4552524F525F494E64
:1040000056414C49445F504152414D004E52465F2B
:104010004552524F525F4E4F5F4D454D00000000DC
:104020004E52465F4552524F525F464F52424944AC
:1040300044454E004E52465F4552524F525F4452E5
:10404000565F5457495F4552525F4F56455252553D
:104050004E0000004E52465F4552524F525F494E4D
:1040600056414C49445F4144445200004E52465F21
:104070004552524F525F5245534F5552434553009C
:104080004E52465F4552524F525F494E56414C493F
:10409000445F464C414753004E52465F535543439D
:1040A000455353004E52465F4552524F525F424C69
:1040B000455F495053505F4348414E4E454C5F4128
:1040C0004C52454144595F455849535453000000F0
:1040D0004E52465F4552524F525F434F4E4E5F43E2
:1040E0004F554E54000000004E52465F4552524F0D
:1040F000525F54494D454F55540000004E52465FA3
:104100004552524F525F4255535900002E2E5C2E9D
:104110002E5C2E2E5C2E2E5C2E2E5C2E2E5C636F63
:104120006D706F6E656E74735C6C696272617269DA
:1041300065735C6C6F675C7372635C6E72665F6CF8
:104140006F675F6261636B656E645F756172742E29
:10415000630000007761726E696E67006465627566
:10416000670000001B5B313B33306D001B5B306D23
:10417000000000001B5B313B33316D001B5B313BAA
:1041800033326D001B5B313B33336D001B5B313BC6
:1041900033346D001B5B313B33356D001B5B313BB2
:1041A00033366D001B5B313B33376D00696E666FD4
:1041B000000000006572726F7200000073645F623D
:1041C0006C655F6366675F73657428292072657428
:1041D00075726E6564202573207768656E20617442
:1041E00074656D7074696E6720746F2073657420D8
:1041F000424C455F47415454535F4346475F5345E4
:1042000052564943455F4348414E4745442E0000BE
:1042100073645F626C655F6366675F7365742829AA
:104220002072657475726E656420257320776865E9
:104230006E20617474656D7074696E6720746F2090
:1042400073657420424C455F434F4D4D4F4E5F4365
:1042500046475F56535F555549442E0073645F626D
:104260006C655F6366675F73657428292072657487
:1042700075726E6564202573207768656E206174A1
:1042800074656D7074696E6720746F207365742037
:10429000424C455F47415454535F4346475F415446
:1042A00054525F5441425F53495A452E000000006A
:1042B00073645F626C655F6366675F73657428290A
:1042C0002072657475726E65642025732077686549
:1042D0006E20617474656D7074696E6720746F20F0
:1042E00073657420424C455F434F4E4E5F434647D3
:1042F0005F4741502E00000073645F626C655F632E
:1043000066675F73657428292072657475726E65BF
:1043100064202573207768656E20617474656D7004
:1043200074696E6720746F2073657420424C455F1A
:104330004741505F4346475F524F4C455F434F559F
:104340004E542E00706565725F6D616E61676572B7
:104350005F67636D00000000706565725F6D616E80
:10436000616765725F6773636D00000070656572F9
:104370005F6D616E616765725F696D006E72665F29
:10438000626C655F6761747400000000706565723F
:104390005F6D616E616765725F706473000000003D
:1043A000706565725F6D616E616765725F70646292
:1043B00000000000706565725F6D616E6167657217
:1043C00000000000706565725F6D616E6167657207
:1043D0005F68616E646C65720000000070656572F4
:1043E0005F6D616E616765725F736D6400000000F0
:1043F000706565725F6D616E616765725F736D0098
:10440000636C6F636B000000434C4F434B00000034
:104410004750494F544500005052530055415254A3
:104420000000000055415254450000006170705F6B
:10443000627574746F6E00006170705F74696D6591
:10444000720000006E72665F6673746F72616765FA
:10445000000000007077725F6D676D7400000000EF
:10446000736F72746C69737400000000756172740C
:104470005F6C6F675F6261636B656E640000000074
:10448000617070006E72665F736468006E72665F62
:104490007364685F626C65006E72665F7364685F08
:1044A000736F63004446030070220020C8020000BE
:1044B0003C750200F4460300382500203831000026
:1044C00044780200F42B0300000000006C44030059
:1044D000C0240020444303000000030358430300AA
:1044E000000003036C430300000003037C4303004C
:1044F000000003038C43030000000303A0430300F8
:1045000000000303B443030000000303C44303009B
:1045100000000303DC43030000000303F043030037
:1045200000000303004403000000000008440300EF
:1045300000000000104403000000000018440300C5
:10454000000000001C44030000000000244403009D
:10455000000000002C440300000000003844030069
:10456000000000004444030000000303544403001F
:1045700000000000604403000000000080440300CD
:104580000000030384440300000003038C44030081
:10459000000003039844030000000303D424002018
:1045A000CC240020D4240020F83000201800000083
:1045B000A17D02001D9102000000000011C5020053
:1045C000382500201B85020058250020B18F0200ED
:1045D000000000002190020000000000759202001F
:1045E000000000009BC602004C250020718B0200D9
:1045F000482D0020118F020000000000A1CD020014
:1046000000000000ED18030000000000D9CD0200FA
:1046100000000000CD8C020000000000A1DD0200BF
:104620000000000055DF020000000000C1990200F8
:1046300000000000690C030000000000B9CD02007A
:1046400000000000061BFFFF0A18015AFF0109566F
:10465000200110D455F702DA59108102101859C5FB
:1046600014B836031AC0041A8804140437031A1045
:10467000041A18041AE8101AF004147834032AC82B
:104680002019081A98041BD8350819101AF8041AAA
:10469000C80C1AA8081A243069B869011A18014907
:1046A00079690901566970011915100140110261FB
:1046B00004091F88811220BA4008293C5904011CB2
:1046C00014B441031A54041AAC041A5C041A6C049E
:1046D0001A64041A74041A7C041A84041A8C041AC6
:1046E00094041A9C041AA404515B90D009219415D7
:0446F000AB02000019
:040000050002720182
:00000001FF
